:020000040800F2
:1000000000070020F1010008AD2D0008652D000853
:100010008D2D0008652D0008852D0008F3010008CE
:10002000F3010008F3010008F3010008453E000851
:10003000F3010008F3010008F3010008F3010008D0
:10004000F3010008F3010008F3010008F3010008C0
:10005000F3010008F30100084D4300087543000850
:100060009D430008C5430008ED430008F301000864
:10007000F3010008F3010008F3010008F301000890
:10008000F3010008F3010008F3010008F301000880
:10009000F3010008452D0008552D000815440008FF
:1000A000F3010008F3010008F3010008F301000860
:1000B000FD440008F3010008F3010008F301000803
:1000C000F3010008F3010008F3010008F301000840
:1000D000F3010008F3010008E9440008F3010008F7
:1000E00079440008F3010008F3010008F301000857
:1000F000F3010008F3010008F3010008F301000810
:10010000F3010008F3010008F3010008F3010008FF
:10011000F3010008F3010008F3010008F3010008EF
:10012000F3010008F3010008F3010008F3010008DF
:10013000F3010008F3010008F3010008F3010008CF
:10014000F3010008F3010008F3010008F3010008BF
:10015000F3010008F3010008F3010008F3010008AF
:10016000F3010008F3010008F3010008F30100089F
:10017000F3010008F3010008F3010008F30100088F
:10018000F3010008F3010008F3010008F30100087F
:10019000F3010008F3010008F3010008F30100086F
:1001A000F3010008F3010008F3010008F30100085F
:1001B000F3010008F3010008F3010008F30100084F
:1001C000F3010008F3010008F3010008F30100083F
:1001D000F3010008F3010008F3010008F30100082F
:1001E000DD14000800000000000000000000000016
:1001F00002E000F000F8FEE772B6374880F30888A6
:10020000364880F3098836483649086040F20000D5
:10021000CCF200004EF63471CEF200010860BFF35C
:100220004F8FBFF36F8F40F20000C0F2F0004EF628
:100230008851CEF200010860BFF34F8FBFF36F8F7C
:100240004FF00000E1EE100A4EF63C71CEF20001D4
:100250000860062080F31488BFF36F8F04F0D6FF88
:1002600005F0B6F84FF055301F491B4A91423CBF8C
:1002700041F8040BFAE71D49184A91423CBF41F886
:10028000040BFAE71A491B4A1B4B9A423EBF51F82E
:10029000040B42F8040BF8E700201849184A914271
:1002A0003CBF41F8040BFAE704F0B4FF05F0D6F8C0
:1002B000144C154DAC4203DA54F8041B8847F9E797
:1002C00000F042F8114C124DAC4203DA54F8041B12
:1002D0008847F9E704F09CBF0007002000230020B6
:1002E0000000000808ED00E00001002000070020E9
:1002F0004857000800230020B4230020B823002022
:10030000FC540020E0010008E4010008E4010008BA
:10031000E40100082DE9F04F2DED108AC1F80CD052
:10032000C3689D46BDEC108ABDE8F08F002383F3BF
:1003300011882846A047002004F0E8FBFEE704F0FF
:1003400071FB00DFFEE70000F8B501F035F904F0BD
:10035000FFFE074604F050FF0546A8BB1F4B9F4217
:1003600032D001339F4232D01D4B27F0FF029A4218
:1003700030D1F8B200F008FF2E4642F2107400F0BF
:1003800009FF08B10024264601F082FC20B10320B9
:1003900000F07AF80024264635B1124B9F4203D074
:1003A00004F022FF00242646002004F0DBFE0EB1FC
:1003B00000F080F801F014FA00F020FF204600F071
:1003C000D1F800F077F8F9E72E460024D7E7044685
:1003D0000126D4E7064640F6C414D0E7010007B072
:1003E000000008B0263A09B008B501F0B1F8A0F154
:1003F00020035842584108BD07B541F212030221BB
:1004000001A8ADF8043001F0C1F803B05DF804FBB9
:1004100038B5302383F31188174803680BB104F013
:1004200033FC164A144800234FF47A7104F022FC7E
:10043000002383F31188124C236813B12368013B16
:100440002360636813B16368013B63600D4D2B78D3
:1004500033B963687BB9022001F050F9322363603D
:100460002B78032B07D163682BB9022001F046F9E2
:100470004FF47A73636038BDB8230020110400087C
:10048000D8240020D0230020084B187003280CD853
:10049000DFE800F008050208022001F025B902207B
:1004A00001F018B9024B00225A607047D023002097
:1004B000D824002010B501F0EBFB30B1234B032210
:1004C0001A70234B00225A6010BD224B224A1C4650
:1004D00019680131F8D004339342F9D16268A2421D
:1004E000F2D31E4B9B6803F1006303F510439A425D
:1004F000EAD204F04BFE04F05DFE002001F076F835
:100500000220FFF7C1FF164B9A6D00229A65996F82
:100510009A67996FD96DDA65D96FDA67D96F196EF5
:100520001A66D3F88010C3F88020D3F8803072B6F2
:100530004FF0E0233021C3F8084DD4E9003281F3B5
:1005400011889D4683F308881047BDE7D02300201B
:10055000D8240020009000082090000800230020EC
:10056000001002402DE9F04F93B0AC4B00902022D8
:10057000FF210AA89D6801F0DDF8A94A1378A3B904
:10058000A848012103601170302383F311880368A8
:100590000BB104F079FBA44AA24800234FF47A710E
:1005A00004F068FB002383F31188009B13B19F4B79
:1005B000009A1A609E4A009C1378032B1EBF0023EA
:1005C00013709A4A4FF0000A18BF5360D34656463C
:1005D000D146012001F088F824B1944B1B68002B10
:1005E00000F01582002000F0B3FF0390039B002B66
:1005F00001DA00F04BFE039B002BEDDB012001F044
:1006000069F8039B213B162BE3D801A252F823F093
:100610006D0600089506000829070008D3050008A4
:10062000D3050008D3050008B307000883090008B4
:100630009D080008FF080008270900084D09000868
:10064000D30500085F090008D3050008D109000898
:100650000D070008D3050008150A000879060008F0
:100660000D070008D3050008FF0800080220FFF767
:10067000BBFE002840F0F581009B0221BAF1000F7B
:1006800008BF1C4605A841F21233ADF8143000F043
:100690007DFF9EE74FF47A7000F05AFF071EEBDBF8
:1006A0000220FFF7A1FE0028E6D0013F052F00F24F
:1006B000DA81DFE807F0030A0D10133605230593EE
:1006C000042105A800F062FF17E054480421F9E76F
:1006D00058480421F6E758480421F3E74FF01C0876
:1006E000404600F085FF08F104080590042105A8A4
:1006F00000F04CFFB8F12C0FF2D1012000FA07F7FF
:1007000047EA0B0B5FFA8BFB4FF0000901F05EF834
:1007100026B10BF00B030B2B08BF0024FFF76CFE78
:1007200057E746480421CDE7002EA5D00BF00B0378
:100730000B2BA1D10220FFF757FE074600289BD0C4
:10074000012000F053FF0220FFF79EFE00261FFA53
:1007500086F8404600F05AFF044690B1002140461A
:1007600000F06CFF01360028F1D1BA46044641F290
:100770001213022105A8ADF814303E4600F006FF22
:1007800027E70120FFF780FE2546244B9B68AB42FC
:1007900007D9284600F02CFF013040F0678104356E
:1007A000F3E7234B00251D70204BBA465D603E46A3
:1007B000ACE7002E3FF460AF0BF00B030B2B7FF484
:1007C0005BAF0220FFF760FE322000F0C1FEB0F107
:1007D0000008FFF651AF18F003077FF44DAF0F4A42
:1007E000926808EB050393423FF646AFB8F5807F69
:1007F0003FF742AF124B0193B84523DD4FF47A70B7
:1008000000F0A6FE0390039A002AFFF635AF019B85
:10081000039A03F8012B0137EDE700BF0023002006
:10082000D4240020B823002011040008D82400207C
:10083000D023002004230020082300200C230020C4
:10084000D4230020C820FFF7CFFD074600283FF43F
:1008500013AF1F2D11D8C5F1200242450AAB25F078
:10086000030028BF424683490192184400F050FF1C
:10087000019A8048FF2100F05DFF4FEAA8037D49FF
:100880000193C8F38702284600F05CFF0646002863
:100890003FF46DAF019B05EB830537E70220FFF7BF
:1008A000A3FD00283FF4E8AE00F0DAFE00283FF494
:1008B000E3AE0027B846704B9B68BB4218D91F2F88
:1008C00011D80A9B01330ED027F0030312AA134458
:1008D00053F8203C05934046042205A901F0C2F9D3
:1008E00004378046E7E7384600F082FE0590F2E7DD
:1008F000CDF81480042105A800F048FE06E7002387
:10090000642104A8049300F037FE00287FF4B4AEFD
:100910000220FFF769FD00283FF4AEAE049800F016
:1009200095FE0590E6E70023642104A8049300F0F7
:1009300023FE00287FF4A0AE0220FFF755FD00281B
:100940003FF49AAE049800F083FEEAE70220FFF736
:100950004BFD00283FF490AE00F092FEE1E702204C
:10096000FFF742FD00283FF487AE05A9142000F0F0
:100970008DFE04210746049004A800F007FE3946C6
:10098000B9E7322000F0E4FD071EFFF675AEBB07A5
:100990007FF472AE384A926807EB090393423FF640
:1009A0006BAE0220FFF720FD00283FF465AE27F074
:1009B00003074F44B9453FF4A9AE484600F018FE7E
:1009C0000421059005A800F0E1FD09F10409F1E713
:1009D0004FF47A70FFF708FD00283FF44DAE00F0A9
:1009E0003FFE002844D00A9B01330BD008220AA9FD
:1009F000002000F0A7FE00283AD02022FF210AA8FC
:100A000000F098FEFFF7F8FC1C4804F085F813B0DE
:100A1000BDE8F08F002E3FF42FAE0BF00B030B2B35
:100A20007FF42AAE0023642105A8059300F0A4FDFD
:100A3000074600287FF420AE0220FFF7D5FC804651
:100A400000283FF419AEFFF7D7FC41F2883004F0DC
:100A500063F8059800F0D0FE464600F0B7FE3C462D
:100A6000B7E5064652E64FF0000905E6BA467EE6CF
:100A700037467CE6D423002000230020A086010016
:100A8000094A136849F2690099B21B0C00FB013353
:100A90001360064B186844F2506182B2000C01FBEF
:100AA0000200186080B27047142300201023002039
:100AB00010B500211022044600F03CFE034B03CB8E
:100AC000206061601868A06010BD00BF9075FF1FB6
:100AD000F0B5ADF5517D6EAC4FF4C47207460D46CE
:100AE0002046002100F026FE02F068F9264B4FF464
:100AF0007A72B0FBF2F0186093E80700022384E8F2
:100B000007000DF5ED702382FFF7D2FF44F20403D6
:100B10001E49238407A804F009FD1F2384F83231FD
:100B20000DF2EB2207AB0DF1340C1E4603CE6645E9
:100B300010605160334602F10802F6D1306810604F
:100B4000B188B37993710FAE91802046314601226E
:100B500000F06CFE00230393AB7E029305F11903B2
:100B6000019380B20123CDE904600093E97E04A3E0
:100B7000D3E90023384602F035FD0DF5517DF0BD77
:100B80009E6AC421818A46EEE02400203C5500087C
:100B90002DE9F0412C4C237ADAB080460D465BBB40
:100BA00027A9284600F068FF0746002842D19DF893
:100BB0009D60C82E3ED801464FF4A662204600F044
:100BC000B9FD4FF48073C4F8F8314FF40073C4F8E2
:100BD0000C334FF44073C4F8203432460DF19E01BB
:100BE00004F1090000F094FD26449DF89C307772D2
:100BF00023720BB9EB7E23728122002106AC27A859
:100C000000F098FD0122214627A800F07BFF002379
:100C10000393AB7E029305F1190380B2019328235D
:100C2000CDE904400093E97E05A3D3E900234046C3
:100C300002F0D8FC5AB0BDE8F08100BFAFF30080ED
:100C400026417272DF25D7B728350020F0B5254E32
:100C50004FF48A7505FB0065F1B096F8D83085F839
:100C6000DC300024D822214685F8E8403AA800F07C
:100C700061FD06F1090000F055FDD5F8E4308DF86E
:100C8000F000C2B206AF06F109010DF1F100CDE9A5
:100C90003A3400F03DFD394601223AA800F068FFE1
:100CA00080B2CDE9047008230127CDE9023706F1AF
:100CB000D803019330230093317A0B4807A3D3E97B
:100CC000002302F08FFCA04206DD02F077F8C5F8A1
:100CD000E000384671B0F0BD2046FBE778F6339F60
:100CE00093CACD8D28350020F83400202DE9F0413D
:100CF0001D4D1E4E1E4F86B0284602F09FFC034637
:100D000058B30024CDE90344ADF81440027B8DF8BC
:100D1000142099684068029403AA03C21B68DFF894
:100D2000548043F00043029302F04AF8821941F1E3
:100D30000003009402A9384601F0A2F9A04205DDA3
:100D4000284602F07FFC88F80040D5E798F800308C
:100D5000072B05D8013388F8003006B0BDE8F081D4
:100D6000014802F06FFCF8E7F834002040420F0021
:100D7000603A00205D3A002070B50D4614461E46CC
:100D800002F08CFB50B9022E10D1012C0ED112A30F
:100D9000D3E90023C5E90023012007E0282C10D067
:100DA00005D8012C09D0052C0FD0002070BD302CA7
:100DB000FBD10BA3D3E90023ECE70BA3D3E900237A
:100DC000E8E70BA3D3E90023E4E70BA3D3E900236F
:100DD000E0E700BFAFF30080401DA12026812A0B71
:100DE00078F6339F93CACD8D9E6AC421818A46EEE0
:100DF00026417272DF25D7B7F017304A39059E5663
:100E000038B505460E4C0021013500F017FCA4F85A
:100E10002C55B4F82C0500F0F9FB78B1B4F82C058A
:100E200000F004FC014648B9B4F82C0500F006FCBB
:100E3000B4F82C350133A4F82C35EAE738BD00BFEF
:100E40002835002010B50A4B0A4A1A6003F5805372
:100E500093F858203AB95C6D2CB1204600F092FF0F
:100E6000204601F0C9F8BDE81040034800F08ABFF1
:100E7000603A002098550008A04A00202DE9F04F64
:100E80008FB000AF05460C4602F008FB00284BD19E
:100E9000237E022B1BD1E38A012B18D101F08EFF98
:100EA0000646FFF7EDFD03464FF4C870DFF8D48225
:100EB000B3FBF0F206F5167602FB103316FA83F355
:100EC000C8F80030E37E33B9A74B00221A703C37D4
:100ED000BD46BDE8F08F07F12401204600F080FDFB
:100EE0000028F4D107F11400FFF7E2FD97F826403F
:100EF00007F11401224607F1270004F0E5FA002863
:100F0000E2D10F2C08D8984B1C70D8F80030A3F50C
:100F10001673C8F80030DAE797F824100029D6D005
:100F2000284602F0B3FAD2E7E38A282B33D010D850
:100F3000012B2BD0052BCAD1BFF34F8F8B498C4B84
:100F4000CA6802F4E0621343CB60BFF34F8F00BF67
:100F5000FDE7302BBBD1874EE17E327A9142B6D18C
:100F6000607E3146002291F8DC50854200F0AD8071
:100F70000132042A01F58A71F5D1326840F6B831A0
:100F8000FA328A4294BF32603160A0E72146284697
:100F9000FFF79EFD9BE721462846FFF7F9FD96E700
:100FA000B2F8EC507B6005F103094FEA99094FEA6A
:100FB0008902D11DC908A8EBC1039D46EB4600215B
:100FC000584600F0B7FB04F1EE012A46314458467A
:100FD00000F09EFB7B6813B9012000F007FB96F838
:100FE000D20000F013FB044630B9307200F038FB39
:100FF000204600F0FBFAB0E0D6F8D4203AB996F8D3
:10100000D200B6F82C25824201D8FFF7F9FED6F8B7
:10101000D4202A44944208D296F8D200B6F82C255F
:101020000130824201D8FFF7EBFE70685FFA89F267
:10103000594600F087FB08B9C54679E0726896F812
:10104000D2002A447260D6F8D42005EB0209C6F813
:10105000D49000F0DBFA814509D396F8D220D6F877
:10106000D4000132001B86F8D220C6F8D400FF2D30
:101070000FD80024347200F0F3FA204600F0B6FADC
:1010800000F006FE3C4B188108B9FFF713FAC5467D
:101090001DE7BB6896F8D9000AFB0362FB68D2F82B
:1010A000E41082F8E83001F58061C2F8E030C2F85F
:1010B000E410FFF7CBFDFFF719FE96F8D9200132B7
:1010C00002F0030286F8D920B6E74FF48A7A0AFBC9
:1010D00002F505F1EA013144204600F07DFDF8609B
:1010E00000287FF4F4AE3544012285F8E82001F0B1
:1010F00065FED5F8E020D6ED007ADFED206A801A93
:10110000192838BF192040F6B832904228BF10463F
:10111000B8EE677A07EE900AF8EEE77A67EEA67AFD
:10112000DFED176AE7EE267AFCEEE77AC6ED007A85
:1011300096F8D9307168BB600AFB03F4321992F853
:10114000E8505DB1D2F8E4308B42E8463FF428AF76
:10115000002182F8E810C2F8E010C5467368064A1C
:101160009B0A01331381B2E6F134002000ED00E068
:101170000400FA0528350020E0240020CDCCCC3D29
:101180006666663FF4340020014B1870704700BF5C
:10119000EC24002038B54FF00054144B22689A42DA
:1011A00021D1607DF0B1124B124918701248237D95
:1011B00003724FF48073C0F8F8314FF40073C0F835
:1011C0000C3300254FF44073C0F82034C0F8E450CD
:1011D000C922093000F09CFAE0222946204600F09E
:1011E000A9FA012038BD0020FCE700BF9AAD44C534
:1011F000EC240020160000202835002037B500F030
:1012000047FD194D1949288102236B7100220123E2
:10121000174801F0AFF900230193164B16490093CC
:101220001648174B4FF4805202F008F9154B197805
:1012300011B1124802F02AF901F0C0FD0446FFF78F
:101240001FFC4FF4C873B0FBF3F202FB130304F569
:10125000167010FA83F00C4B186003F0CDFF08B144
:101260000F232B8103B030BDE024002040420F004B
:10127000603A0020790D0008F0240020F8340020A6
:101280007D0E0008EC240020F43400202DE9F04FFE
:101290002DED028B0FF23829D9E90089834C93B0E8
:1012A0000BAE9FED7E8BFFF721FD814FDFF828A26B
:1012B00000230A93ADF834300B9373604FF0000BAA
:1012C0005B468DED008B01250DF11D0207A9384607
:1012D0008DF81C508DF81DB001F0D8FC9DF81C3025
:1012E000002B40F0A580204602F0D8F806460028E2
:1012F00045D1704F01F062FD3B6898423FD301F049
:101300005DFD8246FFF7BCFB4FF4C873B0FBF3F200
:1013100002FB13030AF5167010FA83F03860664F6B
:1013200097F800B0CBF1100ABBF1000F14BF3346A1
:101330002B465FFA8AFA0EA88DF82830FFF7B8FB23
:10134000BAF1060F28BF4FF0060A0EAB03EB0B01F4
:1013500052460DF1290000F0DBF90AAB0393182384
:1013600002930AF10102554BD2B2CDE90053049227
:1013700020464CA3D3E9002302F0D6F83E7001F0DA
:101380001DFD4F4A4F4D1368C31AB3F57A7F2ED314
:10139000106001F015FD02460B46204602F05CF994
:1013A000204602F07BF810B32B7A474E002B14BF77
:1013B00003230223737101F001FD0EAF4FF47A7322
:1013C0000122B0FBF3F039463060304600F0E0FA1D
:1013D000182302933D4B019380B240F25513CDE99F
:1013E0000370009342464B46204602F09DF82B7A4C
:1013F00093B101F0E3FC002607464FF48A7A95F892
:10140000D900304400F003000AFB005393F8E820B1
:1014100092B30136042EF2D1C82003F07DFB2B7A63
:10142000002B7FF43DAF13B0BDEC028BBDE8F08F15
:10143000DAF8143083F48063CAF814305946102265
:101440000EA800F077F90DF11E0308AA0AA9384684
:1014500000F03CFF96E803000FAB83E803009DF823
:1014600034308DF844300A9B0E930EA9DDE9082331
:10147000204602F0C5FA21E7D3F8E02042B12B68FC
:10148000FA2B38BFFA23BA1A0533B2EB430FC0D395
:10149000FFF7DCFB0028BCD1BEE700BF0000000066
:1014A00000000000401DA12026812A0BF8340020F6
:1014B000603A0020F4340020F1340020F0340020A1
:1014C000583A002028350020E02400205C3A002013
:1014D000F1C6A7C1D068080F0008004808B5054844
:1014E00000F098FFBDE80840034A0449002003F0DB
:1014F000CFBF00BF603A0020804F0020450E00089B
:1015000070B5104B1B780133DBB2012B0C4612D89F
:101510000D4B1D6829684FF47A730E6AA2FB0332E3
:10152000014622462846B047844204D1074B002298
:101530001A70012070BD4FF4FA7003F0EDFA00202C
:10154000F8E700BF182300201C230020744F002060
:1015500007B50023024601210DF107008DF8073081
:10156000FFF7CEFF20B19DF8070003B05DF804FB44
:101570004FF0FF30F9E700000A4608B50421FFF7F5
:10158000BFFF80F00100C0B2404208BD30B4074B3D
:101590000A461978064B53F821402368DD69054B4C
:1015A0000146AC46204630BC604700BF744F002067
:1015B0001C230020A086010070B503F065FC094ED5
:1015C000094D3080002428683388834208D903F00D
:1015D00057FC2B6804440133B4F5104F2B60F2D351
:1015E00070BD00BF764F0020304F002003F006BDD5
:1015F00000F1006000F510400068704700F10060E5
:10160000920000F5104003F083BC0000054B1A68FF
:10161000054B1B889B1A834202D9104403F030BC4F
:1016200000207047304F0020764F0020024B1B688F
:10163000184403F02DBC00BF304F0020024B1B6844
:10164000184403F037BC00BF304F00200020704723
:1016500000F10050A0F51040D0F890057047000050
:10166000064991F8243033B10023086A81F8243008
:101670000822FFF7C3BF0120704700BF344F00208E
:10168000014B1868704700BF002004E030B50F4BD5
:101690000F4C1B682288C3F30B03013893420844A4
:1016A0000BD164680A46013C824213460BD214F9FE
:1016B000015F2DB102F8015BF6E781420B4602D2D1
:1016C0002C2203F8012B581A30BD00BF002004E083
:1016D00020230020022802BF024B4FF080629A6153
:1016E000704700BF00080048022802BF024B4FF4B9
:1016F00080629A61704700BF00080048022801BF5D
:10170000024A536983F480635361704700080048BC
:1017100010B50023934203D0CC5CC4540133F9E7E5
:1017200010BD000003460246D01A12F9011B002921
:10173000FAD1704702440346934202D003F8011BDA
:10174000FAE770472DE9F8431F4D144695F8242019
:101750000746884652BBDFF870909CB395F824305A
:101760002BB92022FF2148462F62FFF7E3FF95F8AF
:101770002400C0F10802A24228BF2246D6B2414648
:10178000920005EB8000FFF7C3FF95F82430A41BFF
:101790001E44F6B2082E17449044E4B285F8246043
:1017A000DBD1FFF75DFF0028D7D108E02B6A03EB00
:1017B00082038342CFD0FFF753FF0028CBD1002014
:1017C000BDE8F8830120FBE7344F0020024B1A7874
:1017D000024B1A70704700BF744F0020182300207E
:1017E00003494FF461430B60024B186803F080B863
:1017F0005C4F00201C230020094B10B51822044622
:1018000000211846FFF796FF064A074B127804603E
:101810000146BDE8104053F8220003F069B800BF4C
:101820005C4F0020744F00201C2300202DE9F3475B
:101830000D46044600219046284640F27912FFF7F3
:1018400079FF234620220021284602F07BF8231D41
:1018500002222021284602F075F8631D032222216E
:10186000284602F06FF8A31D03222521284602F026
:1018700069F804F1080310222821284602F062F8D2
:1018800004F1100308223821284602F05BF804F125
:10189000110308224021284602F054F804F11203F3
:1018A00008224821284602F04DF804F114032022B2
:1018B0005021284602F046F804F118034022702116
:1018C000284602F03FF804F120030822B021284600
:1018D00002F038F804F121030822B821284602F06A
:1018E00031F804F12207C0263B463146082228463B
:1018F000083602F027F8B6F5A07F07F10107F3D10B
:1019000094F832308DF8073031460DF10703082284
:10191000284602F017F8002604F1330A9DF8073034
:101920004FEAC6099E4209F5A47720D394F83231D4
:10193000502B28BF50238DF80730B8F1000F08D185
:1019400039460DF107030722284601F0FBFF09F293
:101950004F17002604F233149DF807309E4207EB20
:10196000C6010DD30731C80802B0BDE8F0870AEB05
:10197000060308223946284601F0E4FF0136CDE788
:10198000A3190822284601F0DDFF0136E4E7000034
:1019900013B504460846002101602346C0F8031031
:1019A0002022019001F0CEFF0198231D0222202168
:1019B00001F0C8FF0198631D0322222101F0C2FF3C
:1019C0000198A31D0322252101F0BCFF019804F119
:1019D00008031022282101F0B5FF072002B010BD36
:1019E000F7B5047F05460E462CB1838A122B02D927
:1019F000012003B0F0BD00231946072200962846B7
:101A000001F064FE731C0093012200230721284685
:101A100001F05CFED4B9B31C0093052223460821D3
:101A2000284601F053FE0D24B378102BE0D837463A
:101A3000B278BB1B934210D32B7FA88A0734E408EB
:101A4000B3B9844294BF00200120D2E7AB8ADB0007
:101A5000083BDB08B3700824E6E7FB1C0093214633
:101A600000230822284601F031FE08340137DFE761
:101A7000201A18BF0120BCE7F7B5047F05460E46C3
:101A80002CB1838ACA2B02D9012003B0F0BD0023F8
:101A9000194600960822284601F018FE731CD4B996
:101AA0000822009311462346284601F00FFE102419
:101AB0007378C82BE8D8012372785F1C013B9342EE
:101AC00010D32B7FA88A0734E408B3B9844294BFAB
:101AD00000200120D9E7AB8ADB00083BDB087370EC
:101AE0000824E5E7F319009321460023082228463D
:101AF00001F0ECFD08343B46DEE7201A18BF012058
:101B0000C3E70000F7B50D460446002116462846F7
:101B10008122FFF70FFE234608220021284601F00C
:101B200011FF94F901206378002AB8BF7F238DF854
:101B300007309EB90DF1070307220821284601F05E
:101B400001FF0F27002602349DF807309E4207EB65
:101B5000C60105D30731C80803B0F0BD0827F1E777
:101B6000A3190822284601F0EDFE0136ECE700003B
:101B7000F7B50E460546002114463046CE22FFF743
:101B8000D9FD2B4628220021304601F0DBFE2B7ABE
:101B9000C82B28BFC8238DF807308CB90DF1070377
:101BA00008222821304601F0CDFE30242F469DF832
:101BB00007207B1B934205D3E01DC00803B0F0BD96
:101BC0002824F3E707F1090321460822304601F0F3
:101BD000B9FE08340137EAE7F7B5047F05460E463B
:101BE00034B1838AB3F5827F02D9012003B0F0BDFE
:101BF0000096012310220021284601F067FDDCB980
:101C0000B31C0093092223461021284601F05EFDF3
:101C100019247388B3F5807FE7D837467288BB1BD9
:101C2000934210D32B7FA88A0734E408B3B98442C7
:101C300094BF00200120D9E7AB8ADB00103BDB0812
:101C400073801024E5E73B1D009321460023082202
:101C5000284601F03BFD08340137DFE7201A18BFA2
:101C60000120C3E730B5094D0A4491420DD011F867
:101C7000013B5840082340F30004013B2C4013F083
:101C8000FF0384EA5000F6D1EFE730BD2083B8EDC2
:101C9000F7B5364A106851686B4603C36A46344943
:101CA0003448082303F020FC044690BB0A25324A3E
:101CB000106851686B4603C36A4630492D480823B3
:101CC00003F012FC0446002847D00369B3F5EE2F59
:101CD00043D8B0F86620B2F5886F3ED1284A024456
:101CE00002F15C018B4238D35C3B224900209E1AF2
:101CF000FFF7B8FF3246074604F164010020FFF702
:101D0000B1FFA3689F4228D1E368984208BF00252D
:101D100023E00369B3F5EE2F26D8428BB2F5886F26
:101D200020D1174A024402F110018B4218D3103B14
:101D3000104900209D1AFFF795FF2A46064604F138
:101D400018010020FFF78EFFA3689E4202D1E368CE
:101D5000984201D00D25AAE70025284603B0F0BD22
:101D60001025A4E70C25A2E70B25A0E7685500087D
:101D7000DC6F07000090000871550008906F0700A5
:101D80000870FFF710B5037C044613B9006803F030
:101D900093FB204610BD00000023BFF35B8FC360A0
:101DA000BFF35B8FBFF35B8F8360BFF35B8F7047C5
:101DB000BFF35B8F0068BFF35B8F704770B505465C
:101DC0000C30FFF7F5FF05F1080604463046FFF733
:101DD000EFFFA04206D930466D68FFF7E9FF2544C2
:101DE000281A70BD3046FFF7E3FF201AF9E700001C
:101DF00070B50546406898B105F10800FFF7D8FFB7
:101E000005F10C0604463046FFF7D2FF8442304607
:101E100094BF6D680025FFF7CBFF013C2C44201ACE
:101E200070BD000038B50C460546FFF7C7FFA0425D
:101E300010D305F10800FFF7BBFF04446868B4FB4A
:101E4000F0F100FB1144BFF35B8F0120AC60BFF3E6
:101E50005B8F38BD0020FCE72DE9F04114460746B2
:101E60000D46FFF7C5FF844228BF0446D4B1B846EB
:101E700058F80C6B4046FFF79BFF30442860404603
:101E80007E68FFF795FF331A9C4203D86C600120EF
:101E9000BDE8F0816B60A41B3B68AB602044E86048
:101EA0000220F5E72046F3E738B50C460546FFF774
:101EB0009FFFA04210D305F10C00FFF779FF044407
:101EC0006868B4FBF0F100FB1144BFF35B8F0120A5
:101ED000EC60BFF35B8F38BD0020FCE72DE9FF41CC
:101EE000884669460746FFF7B7FF6C4606B204EB23
:101EF000C6060025B44209D06268206808EB0501D7
:101F0000FFF706FC636808341D44F3E729463846AA
:101F1000FFF7CAFF284604B0BDE8F081F8B50546D2
:101F20000C300F46FFF744FF05F108060446304623
:101F3000FFF73EFFA042304688BF6C68FFF738FFCE
:101F4000201A386020B130462C68FFF731FF20445A
:101F5000F8BD000073B5144606460D46FFF72EFF88
:101F6000844228BF04460190DCB101A93046FFF746
:101F7000D5FF019B33B93268C5E90233C5E90024B6
:101F800001200CE09C4238BF0194286001986860F1
:101F90008442F5D93368AB60241AEC60022002B0A9
:101FA00070BD2046FBE700002DE9FF410F46694662
:101FB000FFF7D0FF6C4600B204EBC0050026AC4230
:101FC00009D0D4F8048054F8081BB8194246FFF72A
:101FD0009FFB4644F3E7304604B0BDE8F0810000C3
:101FE00038B50546FFF7E0FF044601462846FFF7EF
:101FF00019FF204638BD000008B103F05DBA7047F4
:102000007047000010B41346026814680022A4460A
:102010005DF8044B6047000000F5805090F86904BB
:102020007047000000F5805090F86204704700008F
:1020300000F5805090F96804704700005020704708
:10204000302383F3118800F58052D2F8AC34D2F8F3
:10205000A8041844D2F8A4341844D2F88C34184494
:10206000D2F89C341844D2F898341844002383F3EF
:102070001188704700F58050C0F864140120704743
:102080002DE9FF470C4600F58051054691F86204A2
:10209000BDF8308098B1D1F888040130C1F88804C7
:1020A0002068860006D4207B08280BD9667B0EB1F9
:1020B0000F2807D9D1F88C340133C1F88C344FF094
:1020C000FF30AAE0302080F31188E86BD0F8C470AC
:1020D00017F4001713D0D1F890040130C1F8900420
:1020E000D1F89414002940F09B80CDF8008021465F
:1020F000284600F0B3FE002383F311888DE0D0F86A
:10210000C460686BC6F301464FF0480919FB060925
:1021100020680028B4BF40F0804C4FEA804CC9F8DA
:1021200000C02068400044BF4CF00050C9F80000D7
:1021300094F80CC0300640EA0C40C9F8040094F84A
:102140000DC04FEA461ABCF1000F27D040F44010F2
:10215000C9F80400D1F8C0040130C1F8C00405EB8F
:102160000A0101F58351087F40F020000877207BA9
:10217000CDE9022300F0C6FEDDE902230330801022
:10218000F9B2814207F1010710DA04EB810C09EB87
:102190008101DCF804C0C1F808C0F1E705EB0A01D1
:1021A00001F58351087F6CF34510DFE7E96B0120EF
:1021B000B040C1F8CC0006F1830105EB4111C1E943
:1021C000002305EB461101F583512046083104F147
:1021D0000C0750F804CB41F804CBB842F9D1008881
:1021E0000880AA4441F278014AF801600AF5805A51
:1021F00008F003019AF87C0041F0100120F01F0064
:1022000001438AF87C10002181F31188CDF8008009
:102210002146284600F022FE012004B0BDE8F087E8
:10222000002068E738B5C26B936923F0010393611E
:10223000044600F0C3FD0546E36B9B69DB0706D54A
:1022400000F0BCFD431BFA2BF6D9002004E004F596
:102250008054012084F8620438BD000013B500F5F5
:1022600080540191606DFFF7C3FD1F280AD90199C1
:10227000606D2022FFF732FEA0F120035842584142
:1022800002B010BD0020FBE708B5302383F31188AE
:1022900000F58050406DFFF77FFD002383F3118828
:1022A00008BD0000002202608281426082607047A7
:1022B00010B500220023C0E9002300230446038157
:1022C0000C30FFF7EFFF204610BD00002DE9F0476E
:1022D0009A4688B0074688469146302383F3118892
:1022E00007F580546846FFF7E3FF606DFFF766FD72
:1022F0001F282DD9606D20226946FFF771FE202826
:1023000026D194F862341BB303AD444605AB2E4688
:1023100003CE9E4220606160354604F10804F6D188
:1023200030682060B388A380DDE90023C9E9002379
:10233000BDF80830AAF80030002383F31188534613
:102340004A464146384608B0BDE8F04700F044BD73
:10235000002080F3118808B0BDE8F0872DE9F84F20
:10236000064635468846182200210430FFF7E2F978
:10237000254B45F8403B06F582572C462046203435
:10238000FFF796FFA742F9D106F580544FF480532A
:1023900025640025C4E9113501236765E56484F8E7
:1023A000503084F8583006F5845706F5A4594FF09C
:1023B000000A4FF0000B47E908ABA7F11800FFF740
:1023C00071FF203747F8285C4F45F4D184F86884C2
:1023D000A4F86A54A4F86C54A4F86E5484F87054A9
:1023E000A4F87254A4F87454A4F8765484F8785479
:1023F000B8F1000F02D0054800F0DAFC044BF3639B
:102400003046BDE8F88F00BF985500087C5500089D
:102410000064004010B5044B197804464A1C1A7039
:10242000FFF79CFF204610BD7D4F00202DE9F843AB
:1024300015460C4600295CD0022001F081FF2E4990
:10244000B0FBF4F78C428CBF0A2111214B1EB7FB65
:10245000F1F601FB1671DAB221B1022B1946F5D85B
:10246000002032E0731EB3F5806FF9D2C2EBC208D0
:1024700008F103014FEAE10EC1F3C701A2EB010C21
:102480000EF101094FF47A735FFA8CF70EFB033EED
:1024900059FA8CFCBEFBFCFCBCF5617F17DC1FFA13
:1024A0008CF34A1C57FA82F27243B0FBF2F084427A
:1024B000D6D14A1E0F2AD3D87A1E072AD0D8012097
:1024C0002B806E8028716971AF71BDE8F88308F1C7
:1024D000FF314FEAE10CC1F3C701521A0CF1010EB2
:1024E000D7B20CFB03335EFA82F2B3FBF2F39BB27A
:1024F000D7E70846E9E700BF3F420F0030B50D4B74
:102500000D4D05201C786C438C420ED159785180BA
:1025100099785171D9789171197911715B7903EBBF
:1025200083035B001380012030BD013803F10603F3
:10253000E8D1F9E7DC55000840420F000B4B10B51D
:102540004FF45472044600211846FFF7F3F8084B85
:10255000A3624033E362D8332363F0336363E36BF6
:1025600060620022C3F8C02010BD00BF00A400407C
:1025700070A400402DE9F04700F580551F4695F8FE
:102580006834012B88B004468946904604D9002659
:10259000304608B0BDE8F087994A52F8231009B9CF
:1025A00042F823009748C4F81C90017884F8207002
:1025B00099B9302383F31188934B9A6D42F00072DE
:1025C0009A659A6B42F000729A639A6B22F00072DD
:1025D0009A630123037081F3118895F861647EB9D1
:1025E000302383F311880321152001F0CBFF032151
:1025F000162001F0C7FF012385F8613486F31188A6
:10260000302383F31188E26B936923F01003936105
:1026100000F0D4FB8246E36B9E6916F0080609D0F1
:1026200000F0CCFBA0EB0A03FA2BF4D9002686F3CA
:102630001188ADE79A6942F001029A6100F0BEFB91
:102640008246E36B9A69D00706D400F0B7FBA0EB93
:102650000A03FA2BF5D9E9E79A6942F002029A6176
:10266000E36B4FF0000AC3F854A08AF31188686D39
:10267000FFF792FB202200216846FFF75BF802A8D3
:10268000FFF710FE04F58353CDF818A06A463344D3
:102690000DF1180E9446BCE80300F445186059602B
:1026A000624603F10803F5D1DCF80000186020361B
:1026B0009CF804201A71B6F5806FDBD1002304F575
:1026C000A35285F8603485F863340A3249462046BF
:1026D000FFF7ACFE064690B9E26B936923F0010365
:1026E000936100F06BFB0546E36B9B69D9077FF5AF
:1026F0004EAF00F063FB431BFA2BF5D947E795F883
:102700006E34C5F87C94591E95F86F34E26B013B2A
:102710001B0243EA416395F8701401390B43B5F885
:102720006C14013943EA0143D361B8F1000F36D08C
:1027300004F5A352123241462046FFF7DFFE90B95E
:10274000E26B936923F00103936100F037FB0546C8
:10275000E36B9B69DA077FF51AAF00F02FFB431B91
:10276000FA2BF5D913E795F87724C5F88084511E24
:1027700095F87824E36B013A120142EA012295F8B8
:10278000761401390A43B5F87414013942EA01425A
:1027900042F40002DA60E36B4FF420629A64204650
:1027A000FFF7CCFE002385F86934E36B6FF04042FD
:1027B0001A65E36B154A5A65E36B44229A65E36B2D
:1027C0000722C3F8DC20E36B03229742DA653FF46B
:1027D000DFAEE26B936923F00103936100F0EEFA40
:1027E0000746E36B9B69DB0705D500F0E7FAC31BDF
:1027F000FA2BF6D9CBE6012385F86234C8E600BF90
:10280000784F00207C4F0020001002409B00080001
:102810002DE9F04F00F5A5578BB005469046994637
:102820004FF0000B41F2780A1037EB6BD3F8D4303D
:1028300023FA0BF3DC0753D505EB4B1151444FEA58
:102840004B120B7918074BD405F58056D6F8943403
:102850000133C6F89434C7E900890B79990648BF5B
:10286000D6F8C43405EB020148BF0133514448BFD8
:10287000C6F8C4340B7943F008030B71DB0724D589
:1028800096F863340BB302A8019205F58354FFF761
:102890000FFD019A0834144405AB04F1080C2068BC
:1028A00061681A4603C2083464451346F7D12068AC
:1028B0001060A2889A800123ADF810302B68CDE912
:1028C00002891B6C02A928469847D6F8B834D6F876
:1028D00064040133C6F8B83410B103681B69984723
:1028E0000BF1010BBBF1200F9FD10BB0BDE8F08FB6
:1028F0002DE9F04F8DB004460F4600F061FA824694
:102900008946002F56D1E36BD3F89020920141BF46
:1029100004F58051D1F8A8240132C1F8A824D3F8D5
:102920009020160703D100200DB0BDE8F08FD3F83A
:102930009050E66AC5F30125482303FB0566E84687
:102940004046FFF7AFFC326851004ABF22F06043B7
:10295000C2F38A4343F00043920048BF43F08043F0
:102960000093736813F400131FBF04F58052012312
:102970008DF80D30D2F8C8340EBF8DF80D3001330C
:10298000C2F8C834F38803F00F038DF80C304FF011
:10299000000B9DF80C0000F0B5FA5FFA8BF398423B
:1029A00020D9F2180CA90B44127A03F82C2C0BF145
:1029B000010BEEE7012FB6D1E36BD3F89820950118
:1029C00041BF04F58051D1F8A8240132C1F8A824F0
:1029D000D3F898201007A6D0D3F89850266BC5F3EB
:1029E0000125A9E7EFB9E36BC3F8945004A8FFF7FA
:1029F0005FFC98E80F0007AD07C52B800023ADF8FA
:102A0000183023682046CDE904A91B6C04A9984717
:102A100004F5805458B1D4F8A0340133C4F8A0347C
:102A200082E7012F04BFE36BC3F89C50DEE7D4F8C4
:102A3000A4340133C4F8A434012075E72DE9F04132
:102A400005460F4600F58054012639462846FFF713
:102A50004FFF10B184F86364F7E7D4F8B834D4F8C2
:102A600064040133C4F8B83420B10368BDE8F04110
:102A70001B691847BDE8F081F0B5C36B1A6C12F4FE
:102A80007F0F2BD000F580541B6CC4F8BC3441F28E
:102A90007805002347194FF0010C00EB43122A443C
:102AA0005E01117911F0020F15D0490713D4B959FD
:102AB000C66BD6F8C8E00CFA01F111EA0E0F0AD085
:102AC000C6F8D010117941F004011171D4F89C249A
:102AD0000132C4F89C240133202BDED1F0BD00006C
:102AE00010B5254C254B226802B338B31A6D120677
:102AF0000ED580221A6500F063F950EA01020B46F8
:102B000002D0013861F1000302462068FFF780FE21
:102B10001A4A136D1B032AD523684FF4002103F5CD
:102B200080531165012283F8692420E001221A658F
:102B300008221A654FF480621A6510BD196DC80726
:102B400002D4196D890705D50321196510460021A6
:102B5000FFF774FF094B1A6D100702D41A6DD106E6
:102B600005D518221A6520680121FFF767FF206844
:102B7000BDE81040FFF780BF784F002000640040A0
:102B800008B5302383F31188FFF776FF002383F322
:102B9000118808BDC36BD3F8C40080F40010C0F3E3
:102BA0004050704708B5302383F3118800F58050FA
:102BB000406DFFF703F9002383F3118843090CBF2D
:102BC0000120002008BD000000F5805393F869241F
:102BD00062B1C16B8A6922F001028A61D3F8AC2428
:102BE0000132C3F8AC24002283F869247047000046
:102BF0002DE9F743302181F31188002500F5835139
:102C000041F2780E4FF0010800F5805C00EB4514AE
:102C10007444267977071CD4F6061AD5D0F83C9070
:102C20008E69D9F8C87008FA06F63E4211D04F688E
:102C300001970F689742019F9F410AD2C9F8D0605F
:102C4000267946F004062671DCF898440134CCF865
:102C500098440135202D01F12001D7D1002383F3C1
:102C6000118803B0BDE8F083F8B51E460023137049
:102C70000F4605461446FFF795FF80F001003870B7
:102C80001EB12846FFF786FF2070F8BD2DE9F04FF2
:102C900085B09946DDE90EA30D46029313780193A2
:102CA00091F800B08046164600F08AF82B7804466A
:102CB0000F4613B93378002B41D022463B4640469D
:102CC000FFF796FFFFF75CFFFFF77EFF4B463246AC
:102CD0002946FFF7C9FF2B7833B1BBF1000F03D0B2
:102CE000012005B0BDE8F08F337813B1019B002BB4
:102CF000F6D108F580530393029B544577EB030309
:102D00001DD2039BD3F86404C8B10368AAEB040185
:102D10001B6898474B46324629464046FFF7A4FFBA
:102D20002B7813B1BBF1000FDAD1337813B1019BCB
:102D3000002BD5D100F044F804460F46DCE7002014
:102D4000CFE7000008B50020FFF7CAFEBDE8084045
:102D500001F0ACB808B50120FFF7C2FEBDE808409D
:102D600001F0A4B800B59BB0EFF309816822684672
:102D7000FEF7CEFCEFF30583014B9B6BFEE700BF34
:102D800000ED00E008B5FFF7EDFF000000B59BB0D7
:102D9000EFF3098168226846FEF7BAFCEFF305837A
:102DA000014B5B6BFEE700BF00ED00E0FEE70000BB
:102DB0000FB408B5029801F05FFEFEE702F064B9B7
:102DC00002F046B90139C9B202299EBF00EBC10029
:102DD0000023C0E9013370472DE9F8431E461B88E4
:102DE0005B070546884618D4044600F118094C458F
:102DF00013D063686BB12B682846DB6B9847338828
:102E0000A768C1B243F0040360684246B84708347B
:102E1000EDE7A368002BEED1F9E70120BDE8F883C8
:102E200073B56C4684E80600014600224E68D5B2B0
:102E30006EB98E685EB900EBC200021D94E8030013
:102E4000013582E803001D70012002B070BD01321F
:102E5000032A01F10801E9D10020F6E72DE9F04F3E
:102E60002DED028B89B09FED258BBDF85080044677
:102E70008B46054600F11809002708F0040AA94509
:102E800036D06B680BB9AB6863B1BAF1000F0BD1E8
:102E900023682046DB6B98474346C1B25A46D5E9C2
:102EA0000106B0470835EAE7002FFBD18DED008B16
:102EB000ADF808705B4603AA0BF1080C1868596856
:102EC000174603C7083363453A46F7D11868386098
:102ED0009B88BB80FFF774FF0423ADF8083023689C
:102EE000CDE900011B6C6946204698470127D9E7C8
:102EF000012009B0BDEC028BBDE8F08F000000009E
:102F000000000000082817D909280CD00A280CD086
:102F10000B280CD00C280CD00D280CD00E2814BF78
:102F20004020302070470C2070471020704714203C
:102F30007047182070472020704700002DE9F041AD
:102F4000456A15B94162BDE8F0814B6823F06047DE
:102F5000C3F38A464FEAD37EC3F3807816EA23068A
:102F600038BF3E46AC462B465A68BEEBD27F22F0B5
:102F700060440AD0002A18DAA40CB44217D19D424A
:102F80000FD10D60DEE71346EEE7A74207D102F04E
:102F90008044C2F3807242450BD054B1EFE708D2AF
:102FA000EDE7CCF800100B60CDE7B44201D0B4429D
:102FB000E5D81A689C46002AE5D11960C3E70000ED
:102FC0002DE9F047089D01F007044FEAD508224497
:102FD00005F0070500EBD1004FF47F49944201D181
:102FE000BDE8F08704F0070705F0070A57453E469D
:102FF00038BF5646C6F10806111B8E4228BF0E4642
:10300000E10808EBD50E415C13F80EC0B94029FA6F
:1030100006F721FA0AF1FFB28CEA010147FA0AF732
:1030200039408CEA010C03F80EC034443544D5E72E
:1030300080EA0120082341F2210201B24000002968
:1030400080B203F1FF33B8BF504013F0FF03F4D157
:103050007047000038B50C468D18A54200D138BD28
:1030600014F8011BFFF7E4FFF7E7000042684AB1DC
:10307000136843604389818901339BB2994243813C
:1030800038BF83811046704770B588B0202204464F
:103090000D4668460021FEF74DFB20460495FFF7DC
:1030A000E5FF024658B16B46054608AE1C4603CC08
:1030B000B44228606960234605F10805F6D1104640
:1030C00008B070BD082817D909280CD00A280CD0E0
:1030D0000B280CD00C280CD00D280CD00E2814BFB7
:1030E0004020302070470C2070471020704714207B
:1030F000704718207047202070470000082817D913
:103100000C280CD910280CD914280CD918280CD943
:1031100020280CD930288CBF0F200E2070470920A2
:1031200070470A2070470B2070470C2070470D2015
:10313000704700002DE9F843078C072F04461ED97D
:10314000D0E9029800254FF6FF73C5F12006A5F1DE
:10315000200029FA05F108FA06F628FA00F03143B2
:103160000143C9B21846FFF763FF0835402D0346F7
:10317000EBD1E1693A46BDE8F843FFF76BBF4FF684
:10318000FF70BDE8F883000010B54B6823B9CA8A08
:1031900063F30902CA8210BD04691A681C600361E6
:1031A000C38A013BC3824A60EFE700002DE9F84F74
:1031B0001D46CB8A0F46C3F3090105298146924675
:1031C0000B4630D00020AAB207F11A049EB2042E9A
:1031D0001FFA80F80FD8904503F1010306D3FB8A4C
:1031E0000A4462F30903FB8201201AE01AF8006026
:1031F000E6540130EAE79045F1D2A1F1050B1C231A
:103200007C68BBFBF3F203FB12BB1FFA8BF6002CAE
:1032100045D14846FFF72AFF044638B978606FF079
:103220000200BDE8F88F4FF00008E6E700260660D0
:103230007860ADB24FF0000B454510D90AEB08039A
:10324000221D13F8011B9155B1B208F101081B2989
:103250001FFA88F82BD0454506F10106F1D8FB8A04
:10326000C3F30902154465F30903BCE7013292B2C6
:103270001C462368002BF9D16B1F0B441C21B3FBA8
:10328000F1F301339BB29A42D3D2BBF1000FD0D1FC
:103290004846FFF7EBFE20B9C4F800B0BFE70122B3
:1032A000E7E7C0F800B05E4620600446C1E7454548
:1032B000D5D94846FFF7DAFE08B92060AFE7C0F875
:1032C00000B0002620600446B6E700002DE9F04F6C
:1032D0002DED028B1C4683B05B6901920746884640
:1032E000002B00F0A780238C2BB1E269002A00F0AC
:1032F000A180072B35D807F10C00FFF7B7FE054674
:1033000038B96FF00205284603B0BDEC028BBDE86A
:10331000F08F14220021FEF70DFA228CE16905F1ED
:103320000800FEF7F5F9208C013080B2FFF7E6FEC9
:10333000FFF7C8FE013880B2208401302874636929
:10334000228C1B782A4403F01F0363F03F0348F0EC
:1033500000411372384669602946FFF7EFFD0125E9
:10336000D1E702339BB20722C18A0633B3FBF2F3E3
:10337000828A521A9BB292B29342C2D800F10C03D5
:103380004FF0000908EE103A4FF0800A4E464D46C5
:1033900018EE100AFFF76AFE83460028B1D0142207
:1033A0000021FEF7C7F9002E3AD1019BABF8083097
:1033B00002220BF1080E1FFA82FC0CF10100BCF195
:1033C000060F218C80B201D88E422BD3FFF796FED8
:1033D000FFF778FE62691278013802F01F028E4210
:1033E00008BF4FF0400A42EA49121BFA80F14AEA4C
:1033F000020A013048F0004281F808A08BF8100062
:10340000CBF8042059463846FFF798FD238C013548
:10341000B3422DB289F001094FF0000AB8D172E72A
:103420000022C6E7E169895D0EF802100136B6B2E6
:103430000132C0E76FF0010565E70000F8B51546F9
:103440000E463022002104461F46FEF773F9069B04
:103450006360B5F5001F079BA76034BF6A094FF68C
:10346000FF72A36297B2E66104F1100000239A4252
:1034700006D800230360A782E3822383E360F8BDBC
:103480000660013330462036F1E7000003781BB9AF
:103490004BB2002BC8BF0170704700000078704726
:1034A000F8B50C46C969074611B9238C002B37D1F2
:1034B000257E1F2D34D8387828BB228C072A2CD89B
:1034C000268A36F003032BD14FF6FF70FFF7C2FDBB
:1034D00020F001003102400441EA0561400C41EA5C
:1034E00040254FF6FF72234629463846FFF7EEFE89
:1034F000002807DD626913780133DBB21F2B88BF18
:1035000000231370F8BD218A2D0645EA01250543E5
:103510002046FFF70FFE0246E5E76FF00300F1E7F4
:103520006FF00100EEE7000070B58AB00446164661
:103530000021282268461D46FEF7FCF8BDF8383009
:10354000ADF810300F9B05939DF840308DF8183082
:10355000119B07936946BDF84830ADF820302046EE
:10356000CDE90265FFF79CFF0AB070BD2DE9F0417F
:10357000D36905460C4616460BB9138C5BBB377EE8
:103580001F2F28D895F80080B8F1000F26D03046BC
:10359000FFF7D0FD3378210241EAC33141EA080147
:1035A000338A41EA076141EA03410246334641F06A
:1035B00080012846FFF78AFE00280ADD3378012BB8
:1035C00007D1726913780133DBB21F2B88BF002348
:1035D0001370BDE8F0816FF00100FAE76FF00300AF
:1035E000F7E70000F0B58BB004460D461746002102
:1035F000282268461E46FEF79DF89DF84C305A1E5C
:10360000534253418DF800309DF84030ADF81030F2
:10361000119B05939DF848308DF81830149B079343
:103620006A46BDF85430ADF8203029462046CDE931
:103630000276FFF79BFF0BB0F0BD0000406A00B1BF
:1036400004307047436A1A68426202691A60036173
:10365000C38A013BC38270472DE9F041D0F8208036
:10366000194E14461D464146002709B9BDE8F081B0
:10367000D1E90223A21A65EB0303964277EB030319
:103680001ED2036A8B420DD1FFF77EFD036A1B68D1
:10369000036203690B60C38A0161016A013BC38253
:1036A0008846E2E7FFF770FD0B68C8F80030036951
:1036B0000B60C38A0161013BC382D8F80010D4E7D4
:1036C00088460968D1E700BF80841E002DE9F04FCD
:1036D0008BB00D46DDF8509014469B46804600287E
:1036E00000F01981B9F1000F00F01581531E3F2B36
:1036F00000F21181012A03D1BBF1000F40F00B81D0
:103700000023CDE90833B8F81430B5EBC30F4FEA06
:10371000C30703D300200BB0BDE8F08F2B199F42E5
:10372000D8F80C303ABF7F1BFFB227461BB9D8F838
:103730001030002B7AD0272D4ED8C5F12806B7427D
:103740004FF000032CBFF6B23E4600932946D8F84E
:10375000080008AB3246FFF733FCA7EB060A3544F6
:103760005FFA8AFAB8F8143003F10053053BDB0026
:103770000493D8F80C3003932821039B13B1BAF1BA
:10378000000F2CD1D8F8100040B1BAF1000F05D0CD
:10379000009608AB5246691AFFF712FC38B2002FA8
:1037A000B8D066070AD00AAB03EBD401624211F825
:1037B000083C02F00702134101F8083C082C3CD9F0
:1037C000102C40F2B580202C40F2B780BBF1000FE6
:1037D00000F09C80082334E0BA460026C2E7049B30
:1037E000E02B28BFE02306930B44AB42059314D98A
:1037F0005A1B03980096924534BF5246D2B2691ABA
:1038000008AB04300792FFF7DBFB079A1644AAEBDC
:10381000020A1544F6B25FFA8AFA049B069A0599E1
:103820009B1A0493039B1B680393A6E70093D8F8A5
:10383000080008AB3A462946AEE7BBF1000F13D0AB
:103840000123B4EBC30F6CD0082C12D89DF82030A4
:10385000621E23FA02F2D50706D54FF0FF3202FAB4
:1038600004F423438DF820309DF8203089F800308F
:1038700051E7102C12D8BDF82030621E23FA02F254
:10388000D10706D54FF0FF3202FA04F42343ADF816
:103890002030BDF82030A9F800303CE7202C0FD8AC
:1038A0000899631E21FA03F3DA0705D54FF0FF32BA
:1038B00002FA04F40C430894089BC9F800302AE784
:1038C000402C2BD0DDE90865611EC4F12102A4F172
:1038D000210326FA01F105FA02F225FA03F3114356
:1038E0001943CB0712D50122A4F12003C4F1200112
:1038F00002FA03F322FA01F1A240524243EA010321
:1039000063EB430332432B43CDE90823DDE908236E
:10391000C9E90023FFE66FF00100FCE66FF0080044
:10392000F9E6082CA0D9102CB3D9202CEED8C3E787
:10393000BBF1000FADD0022383E7BBF1000FBBD07A
:1039400004237EE730B5012A144638BF0124402CF9
:1039500085B028BF40240025012ACDE9025518D89A
:103960001B788DF8083063070AD004AB03EBD4054D
:10397000624215F8083C02F00702934005F8083C43
:10398000009103462246002102A8FFF719FB05B06B
:1039900030BD082AE4D9102A03D81B88ADF80830B6
:1039A000E1E7202A8DBFD3E900231B680293CDE90C
:1039B0000223D8E710B5CB681BB98B600B618B82F3
:1039C00010BD04691A681C600361C38A013BC3828D
:1039D000CA60F0E703064CBFC0F3C0300220704756
:1039E00008B50246FFF7F6FF022806D15306C2F3D8
:1039F0000F2001D100F0030008BDC2F30740FBE730
:103A00002DE9F04F93B0CDE903230A680446104630
:103A1000FFF7E0FF022814BFC2F306260026002AA3
:103A20000D46824680F2F78112F0C04940F0F381E2
:103A3000097B002900F0EF81022803D02378B342EC
:103A400040F0EC81C2F304630693104602F07F035A
:103A50000593FFF7C5FF059B29444FEA834848EAD1
:103A60000A4848EA4668CE7800230022CDE90823B8
:103A7000F309834648EA0008029367D0059B009348
:103A800002466768534608A92046B847002800F058
:103A9000C881276A4FB9414604F10C00FFF7F4FAD8
:103AA000074690B96FF0020054E03B6998450DD08D
:103AB0003F68002FF9D1414604F10C00FFF7E4FA0A
:103AC00007460028EED0236A3B60276297F817C0AC
:103AD00006F01F08CCF3840CACEB08001FFA80FE44
:103AE0000028B8BF0EF12000A8EB0C031FFA83FEDC
:103AF000D7E90221B8BF00B2002B0793BEBF0EF179
:103B000020031BB2079352EA010338D0039BDFF86E
:103B100024E39A1A049B4FF0000C63EB01019645D5
:103B20007CEB01032BD36B7B97F81AE0734519D11B
:103B3000029B002B78D0012821DC7868F8B9DFF8E7
:103B4000F0C2944570EB010316D337E0276A27B91A
:103B50006FF00C0013B0BDE8F08F3B699845B5D00D
:103B60003F68F4E7B24890427CEB010301D30020A8
:103B7000F0E7029B002BFAD0079B0F2B17DCFA7D96
:103B8000B30002F0030203F07C031343FB753946D4
:103B90002046FFF7F9FA6B7BBB76029B3BB9FB7DB6
:103BA000C3F38402013262F38603FB75D0E76A7BBC
:103BB000BB7E9A42DBD1029B002B35D0B309022B8E
:103BC00032D0039BBB60049BFB60142200210DA834
:103BD000FDF7B0FD039B0A93049B0B932B1D0C93E5
:103BE0002B7BADF83EB0013BDBB2ADF83C30069B21
:103BF0008DF84230059B8DF8433094F82C308DF8C9
:103C000040A083F001038DF844308DF84180A36813
:103C10000AA920469847FB7DC3F38403013303F0D0
:103C20001F039B02FB82A2E7FB7DC6F34012B2EBAF
:103C3000D31F40F0F980C3F38403434540F0FC8078
:103C4000029A2B7BB609002A52D016F0010661D1E8
:103C5000032B40F2F480039BBB60049BFB60FB8A58
:103C600066F30903FB822B7BAE1D033BDBB23246BE
:103C7000394604F10C00FFF799FA00280CDA3946AE
:103C80002046FFF781FAFB7DC3F38403013303F081
:103C90001F039B02FB8205E7DDE90884AB883B83B9
:103CA0004FF6FF73C9F12000A9F1200228FA09F1AB
:103CB00004FA00F0014324FA02F211431846C9B293
:103CC000FFF7B6F909F10809B9F1400F0346E9D148
:103CD000B8822A7B033AD2B23146FFF7BBF9FB7DAB
:103CE000B882DA43C2F3C01262F3C713FB753EE732
:103CF00086B92E1D013BDBB23246394604F10C0079
:103D0000FFF754FA0028BADB2A7BB88A013AD2B20C
:103D10003146E2E7F98AC1F30901013B0429DAB22D
:103D20005BD8281D002307F11B069A4208D910F81A
:103D300001CB06F801C0013101330529DBB2F4D112
:103D400003990A9104990B91934207F11B010C917D
:103D500038BF043379680D9134BF55FA83F30023DB
:103D60000E93FB8AADF83EB0C3F309031A44069BD9
:103D70008DF84230059B8DF8433094F82C30ADF827
:103D80003C2083F001038DF8443000238DF840A0DF
:103D90008DF841807B602A7BB88A013A291DFFF7A4
:103DA00059F93B8BB882834203D1A3680AA9204604
:103DB000984720460AA9FFF7FDFDFB7DBA8AC3F3A9
:103DC0008403013303F01F039B02FB823B8B9A4267
:103DD0000CBF00206FF01000BCE67B68002BAFD05A
:103DE000052001E01C3033461E68002EFAD1091A66
:103DF000081D2E1D184401EB090CBCF11B0F5FFAC6
:103E000089F39DD89A429BD916F8013B00F8013BF3
:103E100009F10109EFE76FF009009BE66FF00A0076
:103E200098E66FF00B0095E66FF00D0092E600BF8C
:103E300040420F0080841E006FF00E008AE66FF093
:103E40000F0087E6EFF3098305494A6B22F0010270
:103E50004A63683383F30988002383F3118870472A
:103E600000EF00E0302080F3118862B60C4B0D4A61
:103E7000D96821F4E0610904090C0A43DA60D3F837
:103E8000FC20094942F08072C3F8FC200A6842F025
:103E900001020A602022DA7783F82200704700BF0F
:103EA00000ED00E00003FA05001000E010B530233B
:103EB00083F311880E4B5B6813F4006314D0F1EEAA
:103EC000103AEFF30984683C4FF08073E361094BCB
:103ED000DB6B236684F3098800F098FD10B1064B74
:103EE000A36110BD054BFBE783F31188F9E700BF21
:103EF00000ED00E000EF00E03F030008420300088F
:103F0000026843681143016003B11847704700001D
:103F1000024A136843F0C003136070470044004036
:103F200013B50F4C204600F0D7FC04F114000D49E6
:103F3000009400234FF4807200F094FB0A490B4B6D
:103F400000944FF4807204F1380000F00DFC084B2F
:103F5000E365002000F0F4F9206602B010BD00BF58
:103F6000844F0020F04F0020F0500020113F000847
:103F70000044004030B5037C214C002918BF0C469A
:103F8000012B0CD11F4B984209D11F4B9A6D42F463
:103F900000329A659A6F42F400329A679B6F2268EA
:103FA000036EC16D846603EB5203B3FBF2F36268E8
:103FB000150442BF23F0070503F0070343EA450356
:103FC000CB60A36843F040034B60E36843F0010318
:103FD0008B6042F4967343F001030B604FF0FF33A4
:103FE0000B62510505D512F0102205D0B2F1805FA9
:103FF00004D080F8643030BD7F23FAE73F23F8E730
:10400000FC550008844F0020001002402DE9F047C5
:10401000C66D3768F46934622107054619D014F07B
:10402000080118BF4FF48071E20748BF41F020013A
:10403000A30748BF41F04001600748BF41F080013D
:10404000302383F31188281DFFF75AFF002383F3E1
:104050001188E2050AD5302383F311884FF480617B
:10406000281DFFF74DFF002383F311884FF030091F
:104070004FF0000A14F0200838D13B0616D54FF057
:10408000300905F1380A200610D589F31188504609
:1040900000F09EFB002836DA0821281DFFF730FFCC
:1040A00027F080033360002383F31188790614D549
:1040B000620612D5302383F31188D5E913239A427F
:1040C00008D12B6C33B11021281D27F04007FFF7D2
:1040D00017FF3760002383F31188E30618D5AA6E13
:1040E0001369ABB1BDE8F0475069184789F31188EF
:1040F000736A95F864102846194000F007FC8AF3AB
:104100001188F469B6E7B06288F31188F469BAE7F8
:10411000BDE8F087434B4FF4007270B51A605A69DE
:1041200012F4C06FFBD1404B9A6802F00C02042AD3
:1041300020D01A6842F480721A601A685205FCD5C1
:1041400001229A609A6802F00C02042AFAD13749D7
:10415000374A0A600A6812F00F02FBD1C3F89820B0
:1041600063221A601A689603FCD42E4A4FF48071B9
:10417000C2F88010C468E50306D51A6842F480329C
:104180001A601A689103FCD5C269D20709D5D3F821
:10419000982042F00102C3F89820D3F8982096079F
:1041A000FBD54269DA6044F480721A6004F08071D1
:1041B00011B11A689501FBD5996802691B4E22F06E
:1041C000030501F003012943996085693560316871
:1041D00069400907FBD1134905680D6046684E60C8
:1041E0008068C1F880006E0417D448698505FCD446
:1041F000996802F0030021F00301014399609200E5
:104200009968514011F00C0FFAD1E2055EBF1A68AF
:1042100022F480721A60002070BD48698005FCD5C8
:10422000E6E700BF0070004000100240002002409E
:104230000006040008B500F091F9BDE8084000F060
:1042400065B9000010B5394C3948A36A4FF0FF3208
:10425000A262A36A0023A362A16AE16A61F07F01FE
:10426000E162E16A01F07F01E162E16A216B2263B0
:10427000216B2363216BA16BA263A16BA363A16B71
:10428000E16BE263E16BE363E16B216C2264226C1E
:104290002364226C226E42F001022266D4F8802050
:1042A00022F00102C4F88020D4F88020A26D42F0F0
:1042B0008052A265A26F22F08052A267A26F1D4AAF
:1042C0004FF400419160D360136253629362D362F2
:1042D000136353639363D363136453649364D3642A
:1042E00013655365116841F480711160D4F8902012
:1042F00012F4407F1EBF4FF48032C4F89020C4F8FF
:1043000090300D4A0023A360C4F88820C4F89C3084
:10431000FFF700FF10B1094800F0AEFBD4F8903071
:1043200023F00323C4F8903010BD00BF00100240FA
:104330001C5600080070004055010051145600083A
:10434000014B53F82000704728230020074A08B586
:10435000536903F00103536123B1054A13680BB19C
:1043600050689847BDE80840FFF7A0BD0004014031
:104370007C540020074A08B5536903F002035361D7
:1043800023B1054A93680BB1D0689847BDE808404F
:10439000FFF78CBD000401407C540020074A08B59B
:1043A000536903F00403536123B1054A13690BB148
:1043B00050699847BDE80840FFF778BD0004014008
:1043C0007C540020074A08B5536903F00803536181
:1043D00023B1054A93690BB1D0699847BDE80840FD
:1043E000FFF764BD000401407C540020074A08B573
:1043F000536903F01003536123B1054A136A0BB1EB
:10440000506A9847BDE80840FFF750BD00040140DE
:104410007C540020164B10B55C6904F478725A6124
:10442000A30604D5134A936A0BB1D06A9847600675
:1044300004D5104A136B0BB1506B9847210604D575
:104440000C4A936B0BB1D06B9847E20504D5094A2F
:10445000136C0BB1506C9847A30504D5054A936CB7
:104460000BB1D06C9847BDE81040FFF71FBD00BFEF
:10447000000401407C540020194B10B55C6904F421
:104480007C425A61620504D5164A136D0BB1506D1A
:104490009847230504D5134A936D0BB1D06D984707
:1044A000E00404D50F4A136E0BB1506E9847A10477
:1044B00004D50C4A936E0BB1D06E9847620404D5B4
:1044C000084A136F0BB1506F9847230404D5054A6F
:1044D000936F0BB1D06F9847BDE81040FFF7E6BC73
:1044E000000401407C54002008B50348FFF78EFD0E
:1044F000BDE80840FFF7DABC844F002008B500F0A3
:10450000E1FEBDE80840FFF7D1BC0000062108B578
:10451000084600F037F80621072000F033F806219E
:10452000082000F02FF80621092000F02BF80621C2
:104530000A2000F027F80621172000F023F80621B2
:10454000282000F01FF807211C2000F01BF8BDE810
:1045500008400C21262000F015B800004FF0E023A1
:10456000002258684FF0FF31930003F1604303F5D8
:10457000614301329042C3F88010C3F88011F3D236
:104580007047000000F1604303F561430901C9B2BF
:1045900083F80013012200F01F039A4043099B0097
:1045A00003F1604303F56143C3F880211A6070474B
:1045B000F8B5154682680669AA420B46816938BF7C
:1045C0008568761AB54204460BD218462A46FDF78E
:1045D0009FF8A3692B44A361A3685B1BA3602846D3
:1045E000F8BD0CD918463246FDF792F8AF1BE168CA
:1045F0003A463044FDF78CF8E3683B44EBE7184655
:104600002A46FDF785F8E368E5E7000083689342F2
:10461000F7B51546044638BF8568D0E90460361AF8
:10462000B5420BD22A46FDF773F863692B446361E8
:10463000A36828465B1BA36003B0F0BD0DD93246CA
:104640000191FDF765F80199E068AF1B3A463144E6
:10465000FDF75EF8E3683B44E9E72A46FDF758F8C2
:10466000E368E4E710B50A440024C361029B846058
:10467000C0E90000C0E90511C1600261036210BD1C
:1046800008B5D0E90532934201D1826882B98268C7
:10469000013282605A1C42611970D0E904329A4298
:1046A00024BFC3684361002100F052FA002008BD16
:1046B0004FF0FF30FBE7000070B5302304460E4694
:1046C00083F31188A568A5B1A368A269013BA36023
:1046D000531CA36115782269934224BFE368A36148
:1046E000E3690BB120469847002383F311882846DD
:1046F00007E03146204600F01BFA0028E2DA85F395
:10470000118870BD2DE9F74F04460E4617469846AE
:10471000D0F81C904FF0300A8AF311884FF0000B4C
:10472000154665B12A4631462046FFF741FF03464C
:1047300060B94146204600F0FBF90028F1D0002383
:1047400083F31188781B03B0BDE8F08FB9F1000F37
:1047500003D001902046C847019B8BF31188ED1AC6
:104760001E448AF31188DCE7C0E90511C160C3610A
:104770001144009B8260C0E9000001610362704740
:10478000F8B504460D461646302383F31188A76812
:10479000A7B1A368013BA36063695A1C62611D70E5
:1047A000D4E904329A4224BFE3686361E3690BB140
:1047B00020469847002080F3118807E031462046C4
:1047C00000F0B6F90028E2DA87F31188F8BD00009E
:1047D000D0E905239A4210B501D182687AB982687E
:1047E000013282605A1C82611C7803699A4224BF9C
:1047F000C3688361002100F0ABF9204610BD4FF083
:10480000FF30FBE72DE9F74F04460E461746984662
:10481000D0F81C904FF0300A8AF311884FF0000B4B
:10482000154665B12A4631462046FFF7EFFE03469E
:1048300060B94146204600F07BF90028F1D0002302
:1048400083F31188781B03B0BDE8F08FB9F1000F36
:1048500003D001902046C847019B8BF31188ED1AC5
:104860001E448AF31188DCE7026843681143016043
:1048700003B11847704700001430FFF743BF000032
:104880004FF0FF331430FFF73DBF00003830FFF723
:10489000B9BF00004FF0FF333830FFF7B3BF00005F
:1048A0001430FFF709BF00004FF0FF311430FFF75D
:1048B00003BF00003830FFF763BF00004FF0FF3246
:1048C0003830FFF75DBF0000012914BF6FF01300FF
:1048D00000207047FFF724BB044B03600023C0E9AE
:1048E0000233436001230374704700BF3C56000845
:1048F00010B53023044683F31188FFF73BFB0223F6
:104900002374002080F3118810BD000038B5C369FE
:1049100004460D461BB904210844FFF7A5FF2946AC
:1049200004F11400FFF7ACFE002806DA201D4FF456
:104930000061BDE83840FFF797BF38BD002303751D
:10494000826803691B6899689142FBD25A680360C8
:1049500042601060586070470023037582680369E5
:104960001B6899689142FBD85A68036042601060E6
:104970005860704708B50846302383F311880B7DD3
:10498000032B05D0042B0DD02BB983F3118808BD60
:104990008B6900221A604FF0FF338361FFF7CEFF6F
:1049A0000023F2E7D1E9003213605A60F3E7000018
:1049B000FFF7C4BF054BD9680875186802681A600C
:1049C000536001220275D860FBF7A4BCF0510020AF
:1049D00030B50C4BDD684B1C87B004460FD02B461E
:1049E000094A684600F046F92046FFF7E3FF009BBE
:1049F00013B1684600F048F9A86907B030BDFFF769
:104A0000D9FFF9E7F051002075490008044B1A68F6
:104A1000DB6890689B68984294BF00200120704733
:104A2000F0510020084B10B51C68D86822681A6045
:104A3000536001222275DC60FFF78EFF014620469D
:104A4000BDE81040FBF766BCF051002038B5074CBC
:104A500007490848012300252370656000F060FCC9
:104A60000223237085F3118838BD00BF58540020FD
:104A700068560008F051002008B572B6044B18655E
:104A800000F0D0FA00F080FB024B03221A70FEE720
:104A9000F05100205854002000F02CB98B60022304
:104AA00008618B82084670478368A3F1840243F84B
:104AB000142C026943F8442C426943F8402C094AFB
:104AC00043F8242CC26843F8182C022203F80C2C5B
:104AD000002203F80B2C044A43F8102CA3F1200009
:104AE000704700BF2D030008F051002008B5FFF704
:104AF000DBFFBDE80840FFF75BBF0000024BDB684F
:104B000098610F20FFF756BFF0510020302383F348
:104B10001188FFF7F3BF000008B50146302383F387
:104B200011880820FFF754FF002383F3118808BD84
:104B3000064BDB6839B1426818605A601360436005
:104B40000420FFF745BF4FF0FF307047F0510020C1
:104B50000368984206D01A6802605060996118464E
:104B6000FFF726BF7047000010B503689C68A2429B
:104B70000CD85C688A600B604C6021605960996851
:104B80008A1A9A604FF0FF33836010BD1B68121BB6
:104B9000ECE700000A2938BF0A2170B504460D462B
:104BA0000A26601900F0B6FB00F0A2FB041BA54228
:104BB00003D8751C2E460446F3E70A2E04D9BDE837
:104BC0007040012000F0ECBB70BD0000F8B5144B44
:104BD0000D46D96103F1100141600A2A196982600A
:104BE00038BF0A22016048601861A818144600F016
:104BF00083FB0A2700F07CFB431BA342064606D337
:104C00007C1C281900F086FB27463546F2E70A2F60
:104C100004D9BDE8F840012000F0C2BBF8BD00BFD8
:104C2000F0510020F8B506460D4600F061FB0F4A32
:104C3000134653F8107F9F4206D12A46014630465C
:104C4000BDE8F840FFF7C2BFD169BB68441A2C1910
:104C500028BF2C46A34202D92946FFF79BFF2246D4
:104C600031460348BDE8F840FFF77EBFF051002011
:104C70000052002010B4C0E9032300235DF8044B68
:104C80004361FFF7CFBF000010B5194C236998426C
:104C90000DD0D0E90032816813605A609A680A44E6
:104CA0009A60002303604FF0FF33A36110BD2346D9
:104CB000026843F8102F53600022026022699A4272
:104CC00003D1BDE8104000F01FBB936881680B441E
:104CD000936000F00DFB2269E1699268441AA242D8
:104CE000E4D91144BDE81040091AFFF753BF00BFD3
:104CF000F05100202DE9F047DFF8BC8008F11007E3
:104D00002C4ED8F8105000F0F3FAD8F81C40AA68DE
:104D1000031B9A423ED81444D5E900324FF00009F3
:104D2000C8F81C4013605A60C5F80090D8F81030DD
:104D3000B34201D100F0E8FA89F31188D5E90331D3
:104D400028469847302383F311886B69002BD8D00D
:104D500000F0CEFA6A69A0EB04094A4582460DD2FA
:104D6000022000F01DFB0022D8F81030B34208D119
:104D700051462846BDE8F047FFF728BF121A2244E3
:104D8000F2E712EB090938BF4A4629463846FFF7D1
:104D9000EBFEB5E7D8F81030B34208D01444211A1E
:104DA000C8F81C00A960BDE8F047FFF7F3BEBDE8F6
:104DB000F08700BF00520020F051002038B500F00D
:104DC00097FA054AD2E90845031B181945F1000175
:104DD000C2E9080138BD00BFF05100200020704733
:104DE000FEE70000704700004FF0FF307047000002
:104DF000BFF34F8F024A1369DB03FCD4704700BF37
:104E00000020024008B5094B1B7873B9FFF7F0FF8B
:104E1000074B5A69002ABFBF064A9A6002F18832DE
:104E20009A601A6822F480621A6008BD70540020EB
:104E3000002002402301674508B50B4B1B7893B94E
:104E4000FFF7D6FF094B5A6942F000425A611A68CF
:104E500042F480521A601A6822F480521A601A686A
:104E600042F480621A6008BD7054002000200240A5
:104E7000FF289ABF00F58030C00200207047000074
:104E80004FF40060704700004FF4807070470000DE
:104E9000FF2808B50BD8FFF7EBFF00F500630268A9
:104EA000013204D104308342F9D1012008BD002031
:104EB000FCE70000FF2838B5044624D8FFF798FF28
:104EC000FFF7A0FF114AF323136102235361C300CC
:104ED0005169C50903F47E7343EAC5230B4353614B
:104EE000536943F480335361FFF782FF4FF400614D
:104EF000FFF7BEFF00F044F9FFF79EFF2046BDE834
:104F00003840FFF7C5BF002038BD00BF0020024079
:104F10002DE9F84340EA020313F00703144606D0D4
:104F2000304B40F282321A600020BDE8F8838518C9
:104F30002D4A95420CD92B4A40F287311160F3E794
:104F4000031D1B684A68934208D1083C08300831A9
:104F5000072C14D902680B689A42F1D0FFF752FF70
:104F6000FFF746FF214E08314FF001084FF00009CE
:104F7000012CA1F1080706D8FFF75EFF01E0002C25
:104F8000ECD10120D1E7C6F81480054651F8083C61
:104F900045F8043B51F8043C4360FFF729FF3369AF
:104FA00043F001033361C6F81490026851F8083CDD
:104FB0009A420CD00B4B40F2AF321A600C4B186087
:104FC0000C4B1C600C4B1F60FFF736FFACE72D68E5
:104FD00051F8043C9D4201F10801EBD1083C083036
:104FE000C6E700BF6C540020000008080020024003
:104FF000605400206854002064540020084908B51B
:105000000B7828B11BB9FFF7FDFE01230B7008BD1B
:10501000002BFCD0BDE808400870FFF70DBF00BFB3
:105020007054002008B50649064800F0ABF8BDE80A
:1050300008404FF400414FF0805000F0A3B800BF8B
:10504000007F010000010020084600F035BA000092
:1050500038B5EFF311859DB9EFF30584C4F3080467
:10506000302334B183F31188FFF7A8FE85F311884C
:1050700038BD83F31188FFF7A1FE84F3118838BD92
:10508000BDE83840FFF79ABE38B5FFF7E1FF114C95
:10509000114AC00840EA4170A0FB025EC908A0FBAB
:1050A000040C1CEB050CA1FB04404FF000035B411A
:1050B000A1FB02121CEB040C43EB000011EB0E01F0
:1050C00042F10002411842F10000090941EA007072
:1050D00038BD00BFCFF753E3A59BC4200244D2B232
:1050E000904200D17047431C800000F1804000F5E1
:1050F0001450006841F8040BD8B2F1E7124B10B518
:10510000D3F89040240409D4D3F89040C3F89040D9
:10511000D3F8904044F40044C3F890400B4C23680B
:10512000024443F480732360D2B2904200D110BD98
:10513000431C800000F1804000F5145051F8044BEE
:105140000460D8B2F1E700BF0010024000700040D8
:1051500007B5012201A90020FFF7C0FF019803B0A5
:105160005DF804FB13B50446FFF7F2FFA04205D03B
:10517000012201A900200194FFF7C0FF02B010BD79
:10518000704700007047000070470000074B45F271
:1051900055521A6003225A6040F2FF729A604CF630
:1051A000CC421A60024B01221A7070470030004056
:1051B00078540020034B1B781BB1034B4AF6AA22FC
:1051C0001A6070477854002000300040054B1A6880
:1051D00032B902F1804202F50432D2F894201A600A
:1051E000704700BF74540020024B4FF40002C3F814
:1051F000942070470010024008B5FFF7E7FF024B0C
:105200001868C0F3407008BD745400207047000057
:10521000FEE700000A4B0B480B4A90420BD30B4BA6
:10522000DA1C121AC11E22F003028B4238BF002280
:105230000021FCF77FBA53F8041B40F8041BECE78D
:10524000FC570008FC540020FC540020FC540020B3
:105250000023054A19460133102BC2E9001102F15F
:105260000802F8D1704700BF7C54002008B5124BEB
:105270009A6D42F001029A659A6F42F001029A67B4
:105280000E4A9B6F936843F0010393600620FFF77B
:1052900057F80B4BB0FBF3F04FF080434FF0FF3269
:1052A00001389862DA6200229A615A63DA605A60C1
:1052B00001225A611A6008BD00100240002004E07B
:1052C00040420F004FF0804208B51169D3680B408F
:1052D000D9B2C9439B07116107D5302383F31188E5
:1052E000FFF7DAFB002383F3118808BDFFF7BEBF89
:1052F0004FF08043586A70474FF080430022586354
:105300001A610222DA6070474FF080430022DA60AF
:10531000704700004FF0804358637047FEE700007D
:1053200070B51B4B01630025044686B0586085624A
:105330000E46FEF797FD04F11003C4E904334FF065
:10534000FF33C4E90635C4E90044A560E562FFF710
:10535000CFFF2B460246C4E9082304F134010D4A6D
:10536000256580232046FFF799FB0123E0600A4A68
:105370000375009272680192B268CDE90223074B6F
:105380006846CDE90435FFF7B1FB06B070BD00BF3C
:105390005854002074560008795600081D53000820
:1053A000024AD36A1843D062704700BFF051002010
:1053B0004B6843608B688360CB68C3600B69436153
:1053C0004B6903628B6943620B680360704700009E
:1053D00008B5204BDA6A42F07F02DA62DA6A22F01C
:1053E0007F02DA62DA6ADA6C42F07F02DA64DA6E3D
:1053F00042F07F02DA66184ADB6E11464FF09040A9
:10540000FFF7D6FF02F11C0100F58060FFF7D0FF27
:1054100002F1380100F58060FFF7CAFF02F1540184
:1054200000F58060FFF7C4FF02F1700100F58060B5
:10543000FFF7BEFF02F18C0100F58060FFF7B8FFB7
:1054400002F1A80100F58060FFF7B2FFBDE8084057
:10545000FEF7F8BE001002408056000808B500F0C4
:1054600009F8FFF7F3FABDE80840FFF7AFBE000008
:105470007047000008B5FEF7DDFEFFF7E9FEFFF715
:1054800029FAFFF7F5FFBDE80840FFF72FBF00003E
:105490000B460146184600F001B8000010B5054C57
:1054A00013462CB10A4601460220AFF3008010BD1E
:1054B0002046FCE700000000024B01461868FFF799
:1054C000C3BD00BF5023002010B5013902449042F3
:1054D00001D1002005E0037811F8014FA34201D06B
:1054E000181B10BD0130F2E72DE9F041A3B1C91A34
:1054F00017780144044603F1FF3C8C42204601D951
:10550000002009E00578BD4204F10104F5D10CEB5F
:105510000405D618A54201D1BDE8F08115F8018D2A
:1055200016F801EDF045F5D0E7E70000034611F865
:10553000012B03F8012B002AF9D170476F72672EF7
:105540006172647570696C6F742E486F6C796272E9
:105550006F47345F436F6D706173730053544D3305
:105560003247343F3F00000040A2E4F164689106F6
:105570000041A3E5F26569920700000042616420E2
:1055800043414E496661636520696E6465782E000B
:10559000000000000000000075250008052000083C
:1055A0008D2C00087520000881200008CD220008FD
:1055B000252200083D20000841200008192000088D
:1055C000012000088922000825200008212E00085B
:1055D000C52D0008312000085D22000801040E05D9
:1055E000054B02020E05054B04010E05054B050196
:1055F0000B04044B0801060303460000009600005C
:10560000000000000000000000000000000000009A
:1056100000000000636C6B73776300000003000000
:105620000000000000010000000001010300000074
:1056300013283101040704000100000000000000ED
:105640009548000881480008BD480008A94800089E
:10565000B5480008A14800088D48000879480008AE
:10566000C948000863300000645600084852002012
:10567000585400206D61696E0069646C650000001B
:10568000A000802A00000000AAAAAAAA50000024B4
:10569000FFFF0000007700000090090000010040BB
:1056A00000000000AAA9AAAA00000000EFFF000065
:1056B00000000000000000000010101400000000B6
:1056C000AAAAAAA600000010FFDF00000000000048
:1056D000000000000000000000000000AAAAAAAA22
:1056E00000000000FFFF00000000000000000000BC
:1056F0000000000000000000AAAAAAAA0000000002
:10570000FFFF00000000000000000000000000009B
:1057100000000000AAAAAAAA00000000FFFF0000E3
:105720000000000000000000000000000000000079
:10573000AAAAAAAA00000000FFFF000000000000C3
:105740000000000000000000400400000000000015
:105750000070070000000000FE2A0100D2040000D3
:10576000FF000000844F0020000000005C5500088E
:10577000006889096D8BB90200B4C4040068890906
:105780000068890900688909006889090068890931
:105790000068890900000000542300200000000078
:1057A00000000000000000000000000000000000F9
:1057B00000000000000000000000000000000000E9
:1057C00000000000000000000000000000000000D9
:1057D00000000000000000000000000000000000C9
:1057E00000000000000000000000000000000000B9
:1057F000000000000000000000000000FFFFFFFFAD
:10580000FFFFFFFFFFFFFFFFFFFFFFFFFFFFFFFFA8
:10581000FFFFFFFFFFFFFFFFFFFFFFFFFFFFFFFF98
:10582000FFFFFFFFFFFFFFFFFFFFFFFFFFFFFFFF88
:10583000FFFFFFFFFFFFFFFFFFFFFFFFFFFFFFFF78
:1090000000070020D19F0008F9190108551901082F
:10901000C1190108551901088D190108D39F0008CD
:10902000D39F0008D39F0008D39F0008496D010813
:10903000D39F0008D39F0008D39F0008D39F000848
:10904000D39F0008D39F0008D39F0008D39F000838
:10905000D39F0008D39F0008497F0108717F010852
:10906000997F0108C17F0108E97F0108CD740108DB
:10907000E1740108F5740108097501081D750108FE
:109080003175010845750108D39F0008D39F00087A
:10909000D39F0008790E0108890E0108118001088C
:1090A000D39F0008D39F0008D39F0008D39F0008D8
:1090B000F9800108D39F0008D39F0008D39F0008C0
:1090C000D39F0008D39F0008D39F0008D39F0008B8
:1090D000D39F0008D39F0008E5800108D39F0008B4
:1090E00075800108D39F0008D39F0008D39F000814
:1090F000D39F0008D39F0008D39F0008D39F000888
:10910000D39F0008D39F0008D39F0008D39F000877
:10911000D39F0008D39F0008D39F0008D39F000867
:109120006D7501088175010895750108A97501081B
:10913000BD750108D39F0008D39F0008D39F000886
:10914000D39F0008D39F0008D39F0008D39F000837
:10915000D39F0008D39F0008D39F0008D39F000827
:10916000D39F0008D39F0008D39F0008D39F000817
:10917000D39F0008D39F0008D39F0008D39F000807
:10918000D39F0008D39F0008D39F0008D39F0008F7
:10919000D39F0008D39F0008D39F0008D39F0008E7
:1091A000D39F0008D39F0008D39F0008D39F0008D7
:1091B000D39F0008D39F0008D39F0008D39F0008C7
:1091C00059750108D1750108E5750108F97501089F
:1091D000D39F0008D39F0008D39F0008D39F0008A7
:1091E00029A500088DF10008A9130108491B0108F1
:1091F0005531010855550108395B0108B95B010873
:1092000040A2E4F1646891069DF56F618D4AA989D9
:1092100084C6010003BEC59300004004FFFFFFFFAA
:10922000FFFFFFFF81F0004102E000BF83F0004339
:1092300030B54FEA41044FEA430594EA050F08BFF1
:1092400090EA020F1FBF54EA000C55EA020C7FEAB5
:10925000645C7FEA655C00F0E2804FEA5454D4EB32
:109260005555B8BF6D420CDD2C4480EA020281EAFC
:10927000030382EA000083EA010180EA020281EA34
:109280000303362D88BF30BD11F0004F4FEA013186
:109290004FF4801C4CEA113102D0404261EB410195
:1092A00013F0004F4FEA03334CEA133302D052421B
:1092B00063EB430394EA050F00F0A780A4F10104D7
:1092C000D5F1200E0DDB02FA0EFC22FA05F2801811
:1092D00041F1000103FA0EF2801843FA05F35941F7
:1092E0000EE0A5F120050EF1200E012A03FA0EFC76
:1092F00028BF4CF0020C43FA05F3C01851EBE371A0
:1093000001F0004507D54FF0000EDCF1000C7EEBBC
:1093100000006EEB0101B1F5801F1BD3B1F5001FFA
:109320000CD349085FEA30004FEA3C0C04F1010419
:109330004FEA445212F5800F80F09A80BCF1004F42
:1093400008BF5FEA500C50F1000041EB045141EAC4
:10935000050130BD5FEA4C0C404141EB0101013C8D
:1093600028BFB1F5801FE9D291F0000F04BF01467C
:109370000020B1FA81F308BF2033A3F10B03B3F14E
:1093800020020CDA0C3208DD02F1140CC2F10C02DE
:1093900001FA0CF021FA02F10CE002F11402D8BF3C
:1093A000C2F1200C01FA02F120FA0CFCDCBF41EA08
:1093B0000C019040E41AA2BF01EB0451294330BDD7
:1093C0006FEA04041F3C1CDA0C340EDC04F11404B4
:1093D000C4F1200220FA04F001FA02F340EA03008B
:1093E00021FA04F345EA030130BDC4F10C04C4F1D1
:1093F000200220FA02F001FA04F340EA03002946B1
:1094000030BD21FA04F0294630BD94F0000F83F4FA
:10941000801306BF81F480110134013D4EE77FEADD
:10942000645C18BF7FEA655C29D094EA050F08BF29
:1094300090EA020F05D054EA000C04BF194610460A
:1094400030BD91EA030F1EBF0021002030BD5FEA4E
:10945000545C05D14000494128BF41F0004130BD76
:1094600014F580043CBF01F5801130BD01F00045CA
:1094700045F0FE4141F470014FF0000030BD7FEA3D
:10948000645C1ABF194610467FEA655C1CBF0B4638
:10949000024650EA013406BF52EA033591EA030F4F
:1094A00041F4002130BD00BF90F0000F04BF002147
:1094B000704730B54FF4806404F132044FF000057A
:1094C0004FF0000150E700BF90F0000F04BF0021F3
:1094D000704730B54FF4806404F1320410F0004559
:1094E00048BF40424FF000013EE700BF42004FEA54
:1094F000E2014FEA31014FEA02701FBF12F07F43D1
:1095000093F07F4F81F06051704732F07F4208BF87
:10951000704793F07F4F04BF41F40021704730B58E
:109520004FF4607401F0004521F000411CE700BFDA
:1095300050EA010208BF704730B54FF000050AE05D
:1095400050EA010208BF704730B511F0004502D55E
:10955000404261EB41014FF4806404F132045FEA60
:10956000915C3FF4D8AE4FF003025FEADC0C18BF09
:1095700003325FEADC0C18BF033202EBDC02C2F1FB
:10958000200300FA03FC20FA02F001FA03FE40EA8D
:109590000E0021FA02F11444BDE600BF70B54FF091
:1095A000FF0C4CF4E06C1CEA11541DBF1CEA13556F
:1095B00094EA0C0F95EA0C0F00F0DEF82C4481EAD7
:1095C000030621EA4C5123EA4C5350EA013518BFF7
:1095D00052EA033541F4801143F4801338D0A0FBE4
:1095E00002CE4FF00005E1FB02E506F00042E0FB91
:1095F00003E54FF00006E1FB03569CF0000F18BF97
:109600004EF0010EA4F1FF04B6F5007F64F540743E
:1096100004D25FEA4E0E6D4146EB060642EAC621D1
:1096200041EA55514FEAC52040EA5E504FEACE2E3E
:10963000B4F1FD0C88BFBCF5E06F1ED8BEF1004F41
:1096400008BF5FEA500E50F1000041EB045170BDBD
:1096500006F0004646EA010140EA020081EA030101
:10966000B4EB5C04C2BFD4EB0C0541EA045170BDFD
:1096700041F480114FF0000E013C00F3AB8014F177
:10968000360FDEBF002001F0004170BDC4F10004C0
:10969000203C35DA0C341BDC04F11404C4F1200541
:1096A00000FA05F320FA04F001FA05F240EA02009C
:1096B00001F0004221F0004110EBD37021FA04F6D2
:1096C00042EB06015EEA430E08BF20EAD37070BD8C
:1096D000C4F10C04C4F1200500FA04F320FA05F0EB
:1096E00001FA04F240EA020001F0004110EBD370ED
:1096F00041F100015EEA430E08BF20EAD37070BD5D
:10970000C4F1200500FA05F24EEA020E20FA04F335
:1097100001FA05F243EA020321FA04F001F00041E4
:1097200021FA04F220EA020000EBD3705EEA430E55
:1097300008BF20EAD37070BD94F0000F0FD101F084
:109740000046400041EB010111F4801F08BF013CBD
:10975000F7D041EA060195F0000F18BF704703F0FB
:109760000046520043EB030313F4801F08BF013D82
:10977000F7D043EA0603704794EA0C0F0CEA13553E
:1097800018BF95EA0C0F0CD050EA410618BF52EAF8
:109790004306D1D181EA030101F000414FF00000FE
:1097A00070BD50EA410606BF1046194652EA43060C
:1097B00019D094EA0C0F02D150EA013613D195EA80
:1097C0000C0F05D152EA03361CBF104619460AD1C8
:1097D00081EA030101F0004141F0FE4141F47001D2
:1097E0004FF0000070BD41F0FE4141F4780170BDC2
:1097F00070B54FF0FF0C4CF4E06C1CEA11541DBF27
:109800001CEA135594EA0C0F95EA0C0F00F0A7F828
:10981000A4EB050481EA030E52EA03354FEA013155
:1098200000F088804FEA03334FF0805545EA131368
:1098300043EA12634FEA022245EA111545EA106530
:109840004FEA00260EF000419D4208BF964244F1C7
:10985000FD0404F5407402D25B084FEA3202B61AE6
:1098600065EB03055B084FEA32024FF480104FF4BA
:10987000002CB6EB020E75EB030E22BFB61A75462E
:1098800040EA0C005B084FEA3202B6EB020E75EBC1
:10989000030E22BFB61A754640EA5C005B084FEA29
:1098A0003202B6EB020E75EB030E22BFB61A7546F6
:1098B00040EA9C005B084FEA3202B6EB020E75EB01
:1098C000030E22BFB61A754640EADC0055EA060EC2
:1098D00018D04FEA051545EA16754FEA06164FEA05
:1098E000C30343EA52734FEAC2025FEA1C1CC0D1B1
:1098F00011F4801F0BD141EA00014FF000004FF03E
:10990000004CB6E711F4801F04BF01430020B4F1FE
:10991000FD0C88BFBCF5E06F3FF6AFAEB5EB030CB6
:1099200004BFB6EB020C5FEA500C50F1000041EBB3
:10993000045170BD0EF0004E4EEA113114EB5C0480
:10994000C2BFD4EB0C0541EA045170BD41F4801153
:109950004FF0000E013C90E645EA060E8DE60CEA5B
:10996000135594EA0C0F08BF95EA0C0F3FF43BAF78
:1099700094EA0C0F0AD150EA01347FF434AF95EA2F
:109980000C0F7FF425AF104619462CE795EA0C0F13
:1099900006D152EA03353FF4FDAE1046194622E7E0
:1099A00050EA410618BF52EA43067FF4C5AE50EABA
:1099B00041047FF40DAF52EA43057FF4EBAE12E7AA
:1099C0004FF0FF3C06E000BF4FF0010C02E000BF8B
:1099D0004FF0010C4DF804CD4FEA410C7FEA6C5C6E
:1099E0004FEA430C18BF7FEA6C5C1BD001B050EA11
:1099F000410C0CBF52EA430C91EA030F02BF90EAFC
:109A0000020F0020704710F1000F91EA030F58BFBA
:109A1000994208BF90422CBFD8176FEAE37040F01C
:109A2000010070474FEA410C7FEA6C5C02D150EABA
:109A3000013C07D14FEA430C7FEA6C5CD6D152EA75
:109A4000033CD3D05DF8040B704700BF844610463A
:109A500062468C461946634600E000BF01B5FFF739
:109A6000B7FF002848BF10F1000F01BD4DF808ED09
:109A7000FFF7F4FF0CBF012000205DF808FB00BFDA
:109A80004DF808EDFFF7EAFF34BF012000205DF834
:109A900008FB00BF4DF808EDFFF7E0FF94BF012081
:109AA00000205DF808FB00BF4DF808EDFFF7CEFF82
:109AB00094BF012000205DF808FB00BF4DF808EDC1
:109AC000FFF7C4FF34BF012000205DF808FB00BF92
:109AD0004FEA410C7FEA6C5C02D150EA013C0AD1AA
:109AE0004FEA430C7FEA6C5C02D152EA033C02D19C
:109AF0004FF0000070474FF0010070474FEA4102FD
:109B000012F5001215D211D56FF47873B3EB6252CF
:109B100012D94FEAC12343F0004343EA505311F0F6
:109B2000004F23FA02F018BF404270474FF0000088
:109B3000704750EA013005D111F0004008BF6FF0C6
:109B4000004070474FF00000704700BF4A0011D23C
:109B500012F5001211D20DD56FF47873B3EB625287
:109B60000ED44FEAC12343F0004343EA505323FA93
:109B700002F070474FF00000704750EA013002D108
:109B80004FF0FF3070474FF0000070474FEA41023E
:109B9000B2F1E04324BFB3F5001CDCF1FE5C0DD94B
:109BA00001F0004C4FEAC0024CEA5070B2F1004F95
:109BB00040EB830008BF20F00100704711F0804F98
:109BC00021D113F13872BCBF01F00040704741F45D
:109BD00080114FEA5252C2F11802C2F1200C10FA61
:109BE0000CF320FA02F018BF40F001004FEAC12345
:109BF0004FEAD32303FA0CFC40EA0C0023FA02F3E9
:109C00004FEA4303CCE77FEA625307D150EA0133BE
:109C10001EBF4FF0FE4040F44000704701F000408E
:109C200040F0FE4040F40000704700BF7BB972B9BD
:109C30000029BEBF00204FF0004106E008BF002809
:109C40001CBF6FF000414FF0FF3000F0BFB9ADF125
:109C5000080C6DE904CE002909DB002B1ADB00F0AB
:109C60004DF8DDF804E0DDE9022304B0704740421E
:109C700061EB4101002B1BDB00F040F8DDF804E054
:109C8000DDE9022304B0404261EB4101524263EB43
:109C900043037047524263EB430300F02FF8DDF8B3
:109CA00004E0DDE9022304B0404261EB410170476A
:109CB000524263EB430300F021F8DDF804E0DDE9F4
:109CC000022304B0524263EB4303704753B94AB9CD
:109CD000002908BF00281CBF4FF0FF314FF0FF30B4
:109CE00000F074B9ADF1080C6DE904CE00F006F88F
:109CF000DDF804E0DDE9022304B070472DE9F04708
:109D0000089D04468E46002B4DD18A42944669D95F
:109D1000B2FA82F252B101FA02F3C2F1200120FA42
:109D200001F10CFA02FC41EA030E94404FEA1C4890
:109D3000210CBEFBF8F61FFA8CF708FB16E341EA8C
:109D4000034306FB07F199420AD91CEB030306F112
:109D5000FF3080F01F81994240F21C81023E634433
:109D60005B1AA4B2B3FBF8F008FB103344EA0344D7
:109D700000FB07F7A7420AD91CEB040400F1FF33EC
:109D800080F00A81A74240F207816444023840EA29
:109D90000640E41B00261DB1D4400023C5E9004362
:109DA0003146BDE8F0878B4209D9002D00F0EF80E5
:109DB0000026C5E9000130463146BDE8F087B3FA18
:109DC00083F6002E4AD18B4202D3824200F2F98000
:109DD000841A61EB030301209E46002DE0D0C5E903
:109DE000004EDDE702B9FFDEB2FA82F2002A40F04F
:109DF0009280A1EB0C014FEA1C471FFA8CFE012652
:109E0000200CB1FBF7F307FB131140EA01410EFBF5
:109E100003F0884208D91CEB010103F1FF3802D29C
:109E2000884200F2CB804346091AA4B2B1FBF7F096
:109E300007FB101144EA01440EFB00FEA64508D9B9
:109E40001CEB040400F1FF3102D2A64500F2BB80F6
:109E50000846A4EB0E0440EA03409CE7C6F1200745
:109E6000B34022FA07FC4CEA030C20FA07F401FA8B
:109E700006F31C43F9404FEA1C4900FA06F3B1FB14
:109E8000F9F8200C1FFA8CFE09FB181140EA014179
:109E900008FB0EF0884202FA06F20BD91CEB010116
:109EA00008F1FF3A80F08880884240F28580A8F16E
:109EB00002086144091AA4B2B1FBF9F009FB1011C0
:109EC00044EA014100FB0EFE8E4508D91CEB01015E
:109ED00000F1FF346CD28E456AD90238614440EA01
:109EE0000840A0FB0294A1EB0E01A142C846A64681
:109EF00056D353D05DB1B3EB080261EB0E0101FA0A
:109F000007F722FA06F3F1401F43C5E90071002666
:109F10003146BDE8F087C2F12003D8400CFA02FCBC
:109F200021FA03F3914001434FEA1C471FFA8CFECC
:109F3000B3FBF7F007FB10360B0C43EA064300FBBC
:109F40000EF69E4204FA02F408D91CEB030300F15A
:109F5000FF382FD29E422DD9023863449B1B89B211
:109F6000B3FBF7F607FB163341EA034106FB0EF39A
:109F70008B4208D91CEB010106F1FF3816D28B4247
:109F800014D9023E6144C91A46EA004638E72E4613
:109F9000284605E70646E3E61846F8E64B45A9D20B
:109FA000B9EB020864EB0C0E0138A3E74646EAE77A
:109FB000204694E74046D1E7D0467BE7023B614428
:109FC00032E7304609E76444023842E7704700BF91
:109FD00002E000F000F8FEE772B6374880F3088828
:109FE000364880F3098836483649086040F2000058
:109FF000CCF200004EF63471CEF200010860BFF3DF
:10A000004F8FBFF36F8F40F20000C0F2F0004EF6AA
:10A010008851CEF200010860BFF34F8FBFF36F8FFE
:10A020004FF00000E1EE100A4EF63C71CEF2000156
:10A030000860062080F31488BFF36F8F0FF0A8FD2F
:10A040000FF0DAFE4FF055301F491B4A91423CBFDA
:10A0500041F8040BFAE71D49184A91423CBF41F808
:10A06000040BFAE71A491B4A1B4B9A423EBF51F8B0
:10A07000040B42F8040BF8E700201849184A9142F3
:10A080003CBF41F8040BFAE70FF086FD0FF0FAFE33
:10A09000144C154DAC4203DA54F8041B8847F9E719
:10A0A00000F032FA114C124DAC4203DA54F8041BA2
:10A0B0008847F9E70FF06EBD00070020002300205D
:10A0C0000090000808ED00E00001002000070020DB
:10A0D00070540208002300201425002018250020B9
:10A0E00050650020E09100080092000800920008EE
:10A0F000009200082DE9F04F2DED108AC1F80CD028
:10A10000C3689D46BDEC108ABDE8F08F002383F341
:10A1100011882846A04700200EF038FFFEE70EF019
:10A12000C7FD00DFFEE7000010F8012B11F8013B2E
:10A13000012A28BF9A42F7D0D01A7047034613F875
:10A14000012B002AFBD1181A0138704701F0FF01DA
:10A15000102A2BDB10F0070F08D010F8013B013A52
:10A160008B422DD010F0070F42B3F6D1F0B441EA84
:10A17000012141EA014122F007047FF0000700239A
:10A18000F0E80256083C85EA010586EA010685FAF0
:10A1900047F5A3FA87F586FA47F6A5FA87F68EB94A
:10A1A000EED1F0BC01F0FF0102F0070232B110F86D
:10A1B000013B013A83EA010313B1F8D10020704753
:10A1C00001387047002D06BF35460338073815F0B3
:10A1D000010F07D1013015F4807F02BF013015F463
:10A1E000C03F0130F0BC0138704700BF38B50022D5
:10A1F000002304460D46FFF743FC28B920462946B4
:10A20000BDE8384000F00AB8204605F1004100F0F2
:10A2100005F8404261EB410138BD00BFD0B50C4BA1
:10A22000002206460F46FFF7B9F9FFF78FFC0446F8
:10A23000FFF73AF9074B0022FFF7B0F902460B4649
:10A2400030463946FEF7F2FFFFF780FC2146D0BDCD
:10A250000000F03D0000F0417047000070B504467A
:10A26000183005F0C7F804F13C0005F03BFA154B37
:10A270001549196004F5A270002314269DB206FB4F
:10A2800005120133127C002AF8D1104B1D80104BAF
:10A290001A6812B10F4807F0B3FB186004F5805339
:10A2A000012104F58950C3F82C2183F82A111030BC
:10A2B00006F034FE084B1A680AB10848EBE71C6048
:10A2C000204670BD20370020C0DF01081E37002067
:10A2D000E0360020CCDE010818250020E7DE01086A
:10A2E00038B51C4D04460FF007FC0FF019FC286828
:10A2F00020231A46006C4FF4E13102F013F928686C
:10A300004FF4807380224FF4E131C06C02F00AF9FF
:10A31000204600F02DF90FF003FC204600F0E4FF8A
:10A3200004F1180005F022F90FF0FAFB05F04EFEDB
:10A330002B68D86A03685B68984710B1064806F036
:10A3400063FE04F13C0005F0B3FABDE8384007F0C5
:10A3500081BB00BF3825002008DF01080148FFF756
:10A36000BFBF00BF3C2500202DE9F341144C154E22
:10A37000DFF86080144F20460FF026FB134A014699
:10A38000121B134801F068F80EF0B6FB0446A4B1A6
:10A39000206AE1690191B04214BF251AA8EB0605B5
:10A3A0000FF012FB019902462B46384601F054F893
:10A3B00020460EF0B1FB0446E9E702B0BDE8F081AB
:10A3C000000100200007002032DF01080007002004
:10A3D00028DF01080023002010B50F4C03F0C2FF56
:10A3E0002368986A03680522DB690021984723687F
:10A3F000986A036864211B6998472368986A036810
:10A4000028215B6898472368986A0368BDE8104074
:10A410001B690021184700BF3825002038B50546C4
:10A4200007F018FB2A4A1368C31AB3F57A7F04466B
:10A4300008D9284B10601B7823B9274A536983F445
:10A440008063536105F0A4FD244A136841F288310A
:10A45000E31A8B4206D9016821B1146002892048B1
:10A4600000F0FAFF6B7ADA070AD51E4A136841F248
:10A470008831E31A8B4203D928461460FFF774FF32
:10A480006B7A9B0709D4184A1368E31A132B1DD85B
:10A490002846BDE8384001F063B807F0DBFA43F620
:10A4A00098239842EFD91148FFF796FF10480FF014
:10A4B0001DFABFF34F8F0F490F4BCA6802F4E062D9
:10A4C0001343CB60BFF34F8F00BFFDE71460DFE79E
:10A4D0001C2500200023002000080048242500201F
:10A4E00044DF010820250020282500203C250020ED
:10A4F000010007B000ED00E00400FA050148FFF795
:10A500008DBF00BF3C25002038B5054B1C68236873
:10A510000A461D68034B01462046A847002038BD67
:10A52000382500202C25002010B50A4C2046FFF7C6
:10A5300095FE094A094920460FF0C4FC06F02CFF9D
:10A54000074B084A1860BDE810400749074801F06A
:10A5500009BF00BF3C250020843F002059A200080D
:10A5600038250020FDA400085DA300082C2500204C
:10A5700013B5044604F060FC03F012FC204604F01E
:10A58000DBFB18B1B4F90030022B0BD004F0D8FE7D
:10A5900003F0D8F802230DF106012046ADF806308D
:10A5A00004F07AFE02230DF106012046ADF80630D4
:10A5B00004F068FE02B0BDE8104004F0FBBA0000F1
:10A5C000BFF34F8F0549064BCA6802F4E06213439C
:10A5D000CB60BFF34F8F00BFFDE700BF00ED00E091
:10A5E0000400FA0513B51022002104468DF8072057
:10A5F0000FF0A0FC054B1B68D86A03680DF1070239
:10A600001B6B2146984702B010BD00BF38250020C3
:10A61000F0B58BB0174604460E4607F01BFA054608
:10A6200002F020FD03464FF4C87005F5167504F5D9
:10A630008054B3FBF0F202FB103315FA83F3C4F835
:10A640002431FD7E35B91F4806F0DEFC84F8285120
:10A650000BB0F0BD384605A901F0D2FA0746002834
:10A66000F6D101A8FFF7BEFF9DF8165001A92A46B2
:10A670000DF117000FF040FC28B1134806F0C4FCA0
:10A6800084F82871E4E70F2D0CD8D4F8243184F82D
:10A690002851A3F51673C4F8243129460B4806F057
:10A6A000B3FCD5E79DF814100029D1D030460BF04B
:10A6B0005DFE9DF8142094F82A11054806F0A4FCCC
:10A6C000C6E700BF88E00108B3E00108D4E0010854
:10A6D000F6E0010807B5104601A901F03FF958B9A5
:10A6E000074B9DF804101B68D86AA1F1FF020368AC
:10A6F00051421B685141984703B05DF804FB00BF0D
:10A700003825002038B5084615461C460BF036FEA5
:10A7100060B99DF81030022B07D1012C05D11BA385
:10A72000D3E90023C5E90023012038BD0B2C0BD849
:10A7300084B1601E0A280DD8DFE800F00E0C0C0C66
:10A74000160C0C0C0C1E1A00282C09D040F24C439D
:10A750009C4215D00020E8E70EA3D3E90023E1E7EF
:10A760000EA3D3E90023DDE70EA3D3E90023D9E745
:10A770000EA3D3E90023D5E70EA3D3E90023D1E745
:10A780000EA3D3E90023CDE7AFF30080401DA12045
:10A7900026812A0B9E6AC421818A46EE2641727266
:10A7A000DF25D7B7F017304A39059E56D5A4D139E1
:10A7B000F922B6A7CDD269EBC51A133B03806A55BF
:10A7C00075F3008713B59DF81040CDE900341346AA
:10A7D0000A460146806AFFF795FF02B010BD0000EF
:10A7E00070B500F580560D46D6F820417CB90C2195
:10A7F00001200EF057FFC6F8200108B9002070BDF7
:10A80000056084600430FAE72646A46824B1236812
:10A81000AB42F9D1201DF2E70C2101200EF042FFDE
:10A82000B0600028EAD00560B3689C60B068E9E7D2
:10A830002DE9F04190B000F58951BDF858700446FB
:10A840001646103140F2434201A8984601F0C8FD77
:10A85000012F0ED146EA07412046FFF7C1FF05460A
:10A8600070B9002401A801F0D7FD204610B0BDE862
:10A87000F08104F5A8700BF081FD0028EAD1F0E723
:10A880003822002102A80FF055FB02238DF8083072
:10A890009DF85C308DF82030189B0993BDF864302A
:10A8A000ADF82830CDE90468ADF81870079507F0C9
:10A8B000D3F80D4BC01841F10001CDE90C0104F5AE
:10A8C000A87002A90BF05CFD084B0028D5BF9A8840
:10A8D0001A6801321218D4BF9A801A600028D4BFB7
:10A8E00000240124BEE700BF40420F009036002044
:10A8F00030B58FB014460D463822002168460FF05F
:10A9000019FBDDE91223CDE90223BDF85030ADF883
:10A91000103004F119030593A37E8DF81830159BB0
:10A920000793BDF85830ADF8203007F095F80D4B7F
:10A93000C31841F100016A46CDE90A312846E17E9B
:10A940000BF062FD084B0028D5BF9A881A680132C7
:10A950001218D4BF9A801A600028D4BF00200120AA
:10A960000FB030BD40420F0090360020F0B591B0DE
:10A9700004460E46104608A9154601F009FA60BBC8
:10A980009DF82030012B0CD104F0DAFC02F0DAFE45
:10A9900004F010F904F050FA144904F13C0004F0FA
:10A9A0007FF91022002106AF0CA80FF0C3FA012294
:10A9B00039460CA88DF8382001F00EFA0A230293CC
:10A9C00008A3D3E9002380B2CDE90370CDE90023C9
:10A9D00031462A462046FFF78BFF11B0F0BD00BF7D
:10A9E000AFF30080CDD269EBC51A133BF4E5010843
:10A9F0002DE9F041ADF5487D66AC05460E4617469B
:10AA000000214FF4C47220460FF094FA07F022F8A8
:10AA10002F4B4FF47A72B0FBF2F0186093E8070006
:10AA200084E8070001F06AFB037C237401F066FBF5
:10AA3000437C63740323A374264B5A6962610DF54A
:10AA4000DD709A68DB68A261E361FFF7CBFD44F239
:10AA50000403EA682384204B002A18681F4B29DD71
:10AA6000CDE900320DF2CB211D4BC06A502201F01E
:10AA7000F5FD50210DF2CB200FF032FF0DF11C0837
:10AA800084F8320141460122204600F081FF012373
:10AA900002930DA3D3E9002380B2CDE90380CDE971
:10AAA000002331463A462846FFF722FF0DF5487D40
:10AAB000BDE8F081009350220A4BC06A0DF2CB2111
:10AAC00001F0CCFDD5E700BF9E6AC421818A46EE25
:10AAD0008436002000920008382500201BE1010880
:10AAE00014E101085C4C02082DE9F0411546ADF572
:10AAF000866D06460F460FF013F808A9284601F0A8
:10AB000081F90446002840F09F8001464FF4D0723E
:10AB1000A4A80FF00FFA9DF8B880B8F1100F7ED8F6
:10AB200008F1FF330F2B2BD842460DF1B9010DF27E
:10AB3000D1300FF0F1F9424651490DF1B9000FF053
:10AB4000A7FE0246B0B94F480DF11F0103F016FBF6
:10AB50000446002C63D09DF8B83073B39DF82830BC
:10AB60005BB39DF81F20013A032A6DD8DFE802F09D
:10AB70001C2E384122460DF11F010DF2D130E5E7C0
:10AB8000BDF82000479447AA0DF11F0103F03AFEDB
:10AB90000446002843D0012300930DF2D132112343
:10ABA00047A903F027FAD4E7012B4DD10C9B8DF870
:10ABB0001C3147A9204604F051FB9DF81F30013B92
:10ABC000032B41D8DFE803F01C444A4F012B3BD153
:10ABD0000C9BADF81C3147A9204604F077FBECE74D
:10ABE000012B31D10C9B479347A9204604F098FBD9
:10ABF000E3E7022B28D10CA9204604F0F7FADCE7A2
:10AC000001238DF8903294F90030DA17CDE9A6329D
:10AC10005C210DF2D1300FF063FE8DF8D00347AC0C
:10AC200001222146A4A801F015FA0B23029312A3D6
:10AC3000D3E9002380B2CDE90340CDE900233946B2
:10AC40002A463046FFF754FE0DF5866DBDE8F081CB
:10AC500001238DF89032B4F90030D6E701238DF846
:10AC600090322368D1E702238DF890322368A693AF
:10AC7000CEE700BFAFF30080D5A4D139F922B6A743
:10AC80003CE1010845E101082DE9F04FDFF8D8A0CB
:10AC90008BB0804608F5A87948460BF0F1FB0546D5
:10ACA000002858D00024007E0694CDE90744ADF872
:10ACB000244001F01BFB2A7E8DF8240005F11001D1
:10ACC00007A80FF029F92B6843F00043069306F01C
:10ACD000C3FE224B0390C218DAF804000E4641F17D
:10ACE000000308F5805760B30168009409690D46B8
:10ACF00006A9A847A04224DCDAF8040003689B6A8E
:10AD00009847D0E90A23CDE9042306F0A5FEDDE942
:10AD10000423801A61EB0301114B834274EB01039E
:10AD20000FD397F82931072B12D90E4A87F82941FA
:10AD30009388013393804846039A33460BF0AEFB69
:10AD400009E048460BF0A0FB002387F82931A1E772
:10AD5000013387F829310BB0BDE8F08F40420F0076
:10AD60007F841E0090360020B03600202DE9F0418F
:10AD70004FF00053DFF8E0801B684345FCB0054608
:10AD80000C46164604D03148DC2200210FF0D2F8E0
:10AD90004FF0005749A9C7F80080304600F07CFF0B
:10ADA000002849D19DF824313B750BB9F37E3B75E2
:10ADB0009DF8252126480DF593710FF0ADF820463A
:10ADC0000BF0DCFA4FF0005307AF587581220021D9
:10ADD00028A80FF0AFF83946012228A800F0A2FFFA
:10ADE0002823029317A3D3E9002380B2CDE903708F
:10ADF000CDE90023214632462846FFF779FD154F5D
:10AE00003326013E16F0FF06284608D0FFF73CFF28
:10AE10003B68986A036801215B689847F1E7FFF790
:10AE2000DBFA20460BF0AAFA40F0304040F4002054
:10AE30000EF05CFDFFF7C4FB7CB0BDE8F08100BF05
:10AE4000AFF3008026417272DF25D7B704000020DF
:10AE500016000020382500209AAD44C5F0B5044600
:10AE600089B008460E4615460BF088FA68B92B7E65
:10AE7000022B1FD1EB8A012B1CD12A4631462046DA
:10AE800009B0BDE8F040FFF7C3BBEB8A0B2B0BD832
:10AE900083B1013B0A2B0DD8DFE803F00E0C0C0C3C
:10AEA0001E0C0C0C0C473F00282B0DD040F24C42DE
:10AEB000934242D009B0F0BD2A463146204609B03F
:10AEC000BDE8F040FFF794BD2A463146204609B060
:10AED000BDE8F040FFF74ABF07AF1E4806F094F800
:10AEE0000122394606A88DF8182000F02BFE052314
:10AEF000029316A3D3E9002380B2CDE90023CDE964
:10AF000003702A4631462046FFF7F2FC06F0A2FD08
:10AF100004F58054C4F82C01CCE72A46314620467B
:10AF200009B0BDE8F040FFF7DFBD2A4631462046B4
:10AF300009B0BDE8F040FFF719BD2A46314620466A
:10AF400009B0BDE8F040FFF7C5BB00BFF017304ABD
:10AF500039059E5650E101080A460146806AFFF70E
:10AF60007DBF000049421B4B112912D8DFE801F0D8
:10AF70000911110D1111111111111519151D21258D
:10AF8000292D9A6801329A6070479A8901329A8114
:10AF90007047DA890132DA8170475A8B01325A835D
:10AFA00070471A8B01321A8370471A8A01321A824B
:10AFB00070475A8A01325A8270479A8B01329A83BB
:10AFC00070479A8A01329A827047DA8A0132DA82AD
:10AFD000704700BF903600202DE9F04F374E97B0F4
:10AFE0000023CDE90B330A93ADF83430736804467F
:10AFF000002B5FD0324D01274FF0000A4FF0000BBD
:10B0000070688DF814704FF000088DF81580036893
:10B01000CDE900AB0DF11502D3F8089005A9434620
:10B02000C8479DF81430002B44D0414620220EA87A
:10B030000EF080FF7068036806AAD3F814800AA98E
:10B040000DF11603C047002834DD9DF8340001F0EF
:10B0500069F90BA902468DF8500012A80EF05CFFAA
:10B0600004F5A8780A9B0E930EA9DDE90623404655
:10B070000BF042FC10F10D0F014603D02046FFF704
:10B0800071FFBDE70E980BF027FC03900E980BF0B4
:10B090001DFC039BCDE9000708AA41462046FFF7A7
:10B0A00031FB18B12B8A01332B82A9E76B8B01335B
:10B0B0006B83A5E717B0BDE8F08F00BFB036002066
:10B0C0009036002007B500F5A87168460BF0C8FB64
:10B0D000BDF8040064235843BDF80030B0FBF3F022
:10B0E00080B203B05DF804FBF0B597B0044606F0FB
:10B0F000B1FC4FF47A73B0FBF3F0434B434D1B6844
:10B100002860D86A03685B6D98474FF6FF739842D2
:10B1100028BF184628810EA90122284600F0EAFC23
:10B120000EAB80B20293182240F255130025CDE9F0
:10B13000003203902EA3D3E9002304952046FFF7A5
:10B1400077FB637A59074ED501220EA93048314F5B
:10B1500000F05EFB0EAB80B202931F264FF4AB7380
:10B16000CDE90036039024A3D3E9002304952046BB
:10B17000FFF75EFB786803689B6A9847002832D027
:10B180003A788DF8382002680F924268ADF8402076
:10B190008268ADF84220C268ADF844200269ADF87B
:10B1A00046204269ADF8482082691392C269ADF821
:10B1B0005020026AADF8522007AF436AADF8543010
:10B1C000012239460EA800F0CDFA40F2571380B2A2
:10B1D000CDE902700093049509A3D3E900230196F9
:10B1E0002046FFF725FB17B0F0BD00BFAFF300808E
:10B1F000F1C6A7C1D068080FD1F886A9B8E33A769E
:10B20000753CA33CAE0C08CE3825002084360020C7
:10B2100090360020B0360020F0B506468DB000F51F
:10B22000A8700BF0ABF82E4D20B100232B7001203D
:10B230000DB0F0BD06F00EFC2B7804463BB1304655
:10B24000FFF740FF01210246264805F0DDFE01F030
:10B2500009FF4FF4C87306F58057B0FBF3F202FB09
:10B26000130304F5167010FA83F000238DF81830DC
:10B2700097F82831C7F8240123B901228DF8182046
:10B2800087F82A3108A8FFF7ADF997F82811C1F11E
:10B290001004E4B2062C28BF062408AB2246194449
:10B2A0000DF119000EF038FE013406AB00250293B3
:10B2B00018220123E4B2CDE90032049506A3D3E9B4
:10B2C000002303943046FFF7B3FA87F82851284645
:10B2D000AEE700BFAFF30080401DA12026812A0BFE
:10B2E0000023002060E1010870B52B4D2B4E4FF478
:10B2F000807386B0AB80044606F0ACFB4FF47A73E3
:10B30000B0FBF3F028606288B4F902307F2A98BF5E
:10B3100033700DF11701002304F108008DF8173088
:10B3200003F09CFF94F91430002B13BF012300237A
:10B33000012200221B0143EA0253194A41F2E8406C
:10B34000936100F0DFFE054608B105F0F1F8154BFA
:10B350001D60154B00225D601A702DB12B6861686D
:10B360005B68012228469847104B009304F5A870AB
:10B3700004F5C0710E4B01944FF47A6203900AF009
:10B38000C9FF3178039821B106B0BDE870400AF0DA
:10B39000EDBF06B070BD00BF84360020C53600206A
:10B3A00000040048B8360020B0360020C5A70008C9
:10B3B00059AF000830B50628134698BF1D4AC7B0DC
:10B3C00098BF155C07930C464FF07C024FF00001CC
:10B3D00027A888BF00250EF0ADFD079B22465A2105
:10B3E0000DF1BE0005F0C6FD5A2828BF5A2008AC52
:10B3F0008DF8BD002146012227A88DF89C5000F051
:10B40000ABFB0023049380B243F6FF731822CDE90F
:10B410000240CDE90032084804A3D3E90023FFF736
:10B4200007FA47B030BD00BFAFF30080759D040C34
:10B430008EA454D61CE201083C2500200EB403B5AE
:10B4400003AA52F8041B0192FFF7B4FF02B05DF8A3
:10B4500004EB03B0704700000FB407B504AA07203F
:10B4600052F8041B0192FFF7A5FF03B05DF804EB4F
:10B4700004B0704737B5044600F5A8700BF00EF81D
:10B480002046FFF71FFE462802D92B4805F0BCFDD9
:10B490002046FFF729FE94F90850002D38D00023EC
:10B4A00004F10800EDB201A98DF8043003F0D6FED6
:10B4B0002A2D224C0AD1224D2846FFF7CDFF2368C2
:10B4C000986A036864215B689847F5E72B2D04D1DF
:10B4D0001C48FFF7C1FF1C4B98474FF4FA6101A8C5
:10B4E00000F064FF2468A06A03684FF47A715B6817
:10B4F0009847E06A03689B6A984718B1012816D0FC
:10B50000124800E01248FFF7A7FF01A800F05AFF19
:10B51000104B00225A7106F09DFA47F230539842C0
:10B5200007D90D4803B0BDE830400EF0DFB90B4835
:10B53000E9E703B030BD00BF98E1010838250020DD
:10B54000B6E10108C7E1010838ED00E002E20108B8
:10B55000D7E1010884360020263A09B0ECE1010861
:10B560002DE9F341044606F075FA3B490B68C31A0E
:10B57000322B05461BD9394B1B78C3B138480278AA
:10B580000123934023F4AA4323F055031B041B0C0F
:10B59000002B0EBF012600264FF4806343EA86632A
:10B5A0000132304E02F01F02B36102700D6004F5EB
:10B5B000805606F04FFAD6F82431984202D9204638
:10B5C000FFF72AFE284A1368EB1AB3F57A7F07D3F0
:10B5D000156006F041FA02460B462046FFF74AFF87
:10B5E000204600F051F806F031FA04F58955DFF8ED
:10B5F0007C800746103506F029FAC01BB0F57A7F2B
:10B6000017D2D8F80030986A03684FF480619B68BD
:10B61000984740F2D772294601A800F0E1FE204683
:10B62000FFF732FB2046FFF7D7FC01A800F0F4FE3D
:10B63000E1E7D6F82C3163B106F00CFAD6F82C31DC
:10B64000C01AB0F57A7F04D92046FEF7C5FEFEF792
:10B65000B7FF02B0BDE8F081C03600200023002013
:10B66000C436002000080048BC36002038250020E1
:10B6700010B590F80511044604F06CF86423C0B2CC
:10B6800003FB0044A06E10BD70B52DED048B90F946
:10B6900041309EB00446002B57D090F83F31002B2C
:10B6A00053D006F0D7F9D4F84831C01A27284CD91E
:10B6B00004F13C05284604F063F82846D4F84861B4
:10B6C000FFF7D6FF864240D094F84111284604F097
:10B6D00051F8002839D02846FFF7CAFF94F84111E5
:10B6E000C4F84801284604F035F86423C0B203FBCF
:10B6F00000409FED1B0A983001F0CCFC0AAD2822D7
:10B70000002114A8B0EE409AF0EE608AB0EE418AB3
:10B710000EF010FC0122294611A88DED119ACDEDF5
:10B72000128A8DED138A00F0CFF8002380B2182220
:10B73000049340F2E933CDE90250CDE900322046CE
:10B7400005A3D3E90023FFF773F81EB0BDEC048B0B
:10B7500070BD00BFAFF30080F2C20B46A9D4A7E2D0
:10B760006F12833A70B50C46192605463246002101
:10B7700020460EF0DFFB2B462046082200210BF06E
:10B7800027F82B1D2046202208210BF021F805F177
:10B7900008032046102228210BF01AF805F10A03AD
:10B7A0002046102238210BF013F805F10C03204637
:10B7B000102248210BF00CF805F10E032046102250
:10B7C00058210BF005F805F11003204610226821DE
:10B7D0000AF0FEFF05F114032046202278210AF02A
:10B7E000F7FF05F118032046102298210AF0F0FF18
:10B7F00005F11A0320461022A8210AF0E9FF20468D
:10B8000005F11C031022B8210AF0E2FF304670BD9A
:10B8100070B50C461C2605463246002120460EF027
:10B8200089FB2B462046202200210AF0D1FF2B1D48
:10B830002046102220210AF0CBFF05F10803204604
:10B84000202230210AF0C4FF05F10C03204610220B
:10B8500050210AF0BDFF05F10E03204610226021A1
:10B860000AF0B6FF05F110032046102270210AF0FD
:10B87000AFFF05F112032046102280210AF0A8FF35
:10B8800005F114032046102290210AF0A1FF05F1D2
:10B89000160320461022A0210AF09AFF05F1180392
:10B8A00020461022B0210AF093FF05F11A0320462A
:10B8B0001022C0210AF08CFF2046AB191022D021A3
:10B8C0000AF086FF304670BD2DE9F3410E4604466E
:10B8D00017460021192230460EF02CFBA046002509
:10B8E000B8EC010A0AF0C4FF2946ADF806000DF1D4
:10B8F00006031022304610350AF06AFF302DEFD1D2
:10B90000237B092B28BF09238DF805303FB9294631
:10B910000DF10503042230460AF05AFF3425103495
:10B920004FF000089DF80530984505EB081704D343
:10B93000F81DC00802B0BDE8F081B4EC010A0AF0BD
:10B9400097FF0DF10603ADF8060010223946304688
:10B950000AF03EFF08F10108E4E7000013B50446D1
:10B96000007F10B1A38A012B0CD80023009108227C
:10B97000194620460AF0EEFD237FA08A23B9B0FACB
:10B9800080F0400902B010BD013818BF0120F9E76E
:10B990002DE9F3470D46044600219046284640F223
:10B9A00079120EF0C7FA23462022002128460AF019
:10B9B0000FFF231D0222202128460AF009FF631DE4
:10B9C0000322222128460AF003FFA31D032225217A
:10B9D00028460AF0FDFE04F108031022282128461B
:10B9E0000AF0F6FE04F110030822382128460AF076
:10B9F000EFFE04F111030822402128460AF0E8FE78
:10BA000004F112030822482128460AF0E1FE04F15D
:10BA100014032022502128460AF0DAFE04F118030C
:10BA20004022702128460AF0D3FE04F120030822A8
:10BA3000B02128460AF0CCFE04F121030822B821E7
:10BA400028460AF0C5FE04F12207C0263B463146CF
:10BA50000822284608360AF0BBFEB6F5A07F07F19B
:10BA60000107F3D194F832308DF8073031460DF1EB
:10BA70000703082228460AF0ABFE002604F1330A29
:10BA80009DF807304FEAC6099E4209F5A47720D3F6
:10BA900094F83231502B28BF50238DF80730B8F17D
:10BAA000000F08D139460DF10703072228460AF096
:10BAB0008FFE09F24F17002604F233149DF8073069
:10BAC0009E4207EBC6010DD30731C80802B0BDE89E
:10BAD000F0870AEB06030822394628460AF078FE6A
:10BAE0000136CDE7A319082228460AF071FE013677
:10BAF000E4E7000013B50446084600210160234630
:10BB0000C0F80310202201900AF062FE0198231D64
:10BB1000022220210AF05CFE0198631D03222221EB
:10BB20000AF056FE0198A31D032225210AF050FEBB
:10BB3000019804F10803102228210AF049FE072089
:10BB400002B010BD08B5034608460021017001226D
:10BB50000AF03EFE012008BD2DE9F3410D460446E2
:10BB60000021164628467B220EF0E4F923460322E4
:10BB7000002128460AF02CFE63781F2B28BF1F23C4
:10BB80008DF8063005220DF10603032128460AF040
:10BB90001FFE01239DF80620DF0003F10108013B91
:10BBA0009A421CD894F821305A2B28BF5A238DF87A
:10BBB00007303EB939460DF10703072228460AF03F
:10BBC00007FE0737002622349DF807309E4207EB18
:10BBD000C6010DD30731C80802B0BDE8F08104EBFF
:10BBE00008030822394628460AF0F2FD4346D1E709
:10BBF000A319082228460AF0EBFD0136E4E700000D
:10BC0000F7B5047F05460E462CB1838A122B02D964
:10BC1000012003B0F0BD00231946072200962846F4
:10BC20000AF098FC731C0093012200230721284688
:10BC30000AF090FCD4B9B31C0093052223460821D6
:10BC400028460AF087FC0D24B378102BE0D837463D
:10BC5000B278BB1B934210D32B7FA88A0734E40829
:10BC6000B3B9844294BF00200120D2E7AB8ADB0045
:10BC7000083BDB08B3700824E6E7FB1C0093214671
:10BC80000023082228460AF065FC08340137DFE764
:10BC9000201A18BF0120BCE7F7B5047F05460E4601
:10BCA0002CB1838ACA2B02D9012003B0F0BD002336
:10BCB00019460096082228460AF04CFC731CD4B999
:10BCC000082200931146234628460AF043FC10241C
:10BCD0007378C82BE8D8012372785F1C013B93422C
:10BCE00010D32B7FA88A0734E408B3B9844294BFE9
:10BCF00000200120D9E7AB8ADB00083BDB0873702A
:10BD00000824E5E7F319009321460023082228467A
:10BD10000AF020FC08343B46DEE7201A18BF012059
:10BD2000C3E70000F7B50D46044600211646284635
:10BD300081220EF0FFF823460822002128460AF04F
:10BD400047FD94F901206378002AB8BF7F238DF85E
:10BD500007309EB90DF107030722082128460AF093
:10BD600037FD0F27002602349DF807309E4207EB6F
:10BD7000C60105D30731C80803B0F0BD0827F1E7B5
:10BD8000A319082228460AF023FD0136ECE700003B
:10BD900037B50446007F0D4610B1A38A072B15D88E
:10BDA0000023194600950822204608350AF0D2FBE8
:10BDB000012300953022082120460AF0CBFB237F87
:10BDC000A08A2BB906288CBF0020012003B030BD0B
:10BDD000073818BF0120F9E738B50C46002121606B
:10BDE0000546C4F803100346302220460AF0F0FC52
:10BDF000204605F10803012230210AF0E9FC072062
:10BE000038BD00002DE9F04390F81C8085B006464F
:10BE10000D46B8F1000F06D0838AE02B03D901202C
:10BE200005B0BDE8F083002319460D220095304689
:10BE30000AF090FB0DF10F030093032200230D2164
:10BE400030460AF087FB9DF80F30042BE7D82B72A1
:10BE5000013B032B03D8DFE803F025303B461024D9
:10BE6000B8F1000F5FD105F19803009321464346D6
:10BE7000072230460AF06EFB073495F898305C2BA9
:10BE8000CDD82F4695F898207B1B934252D3337F11
:10BE9000B08A0734E408002B58D1844294BF0020B4
:10BEA0000120BDE705F1100300934022012310217A
:10BEB00030460AF04FFB5024D2E705F110030093FF
:10BEC00020220123102130460AF044FB3024C7E72A
:10BED00005F11003009308220023102130460AF0D8
:10BEE00039FB1824BCE705F1100300930822002356
:10BEF000102130460AF02EFB2B7C802B8FD8002798
:10BF000005F111092B7CFC009F4204F11804A7D213
:10BF100009EB0703009308220023214630460AF06C
:10BF200019FB0137EEE7B38AC4EBC303DB0885F8DE
:10BF30009830A2E707F199030093214600230822D5
:10BF400030460AF007FB083401379BE7201A18BF78
:10BF5000012065E7F7B50C46137809688DF80630BF
:10BF600015460DF10603032206460AF031FC21684E
:10BF7000033121602B78013B032B0CD8DFE803F061
:10BF8000020D161F05F10803402230460AF020FC7E
:10BF900023684033236003B0F0BD05F1080320227D
:10BFA00030460AF015FC23682033F3E705F1080357
:10BFB000082230460AF00CFC23680833EAE72B7AA3
:10BFC000802B28BF80238DF8073008220DF107034E
:10BFD00030460AF0FDFB236808332360002709354B
:10BFE0009DF807309F42D6D2EB19216808223046CF
:10BFF0000AF0EEFB2368083323600137F0E7000006
:10C0000073B50C46137809688DF8073015460DF1A5
:10C010000703022206460AF0DBFB21680231216099
:10C020002B78012B03D0022B0BD002B070BD05F191
:10C030000803402230460AF0CBFB236840332360DC
:10C04000F3E705F10803202230460AF0C1FB23681C
:10C050002033F4E773B50D46044600211646284602
:10C0600040F273120DF066FF0523224601A928460F
:10C070000193FFF76FFF019B04F19002053301A9C3
:10C0800028460193FFF766FF019B04F59072063383
:10C0900001A928460193FFF7B3FF019B04F59872AD
:10C0A000063301A928460193FFF7AAFF94F840310F
:10C0B0005C2B28BF5C238DF803304EB90DF10303D0
:10C0C0000199072228460AF083FB019B073301935D
:10C0D000002604F241149DF8033001999E4203D3D7
:10C0E0000731C80802B070BDA319082228460AF01B
:10C0F0006FFB019B083301930136ECE70048704762
:10C100006CE201080121884238BF08460DF0CABA26
:10C11000FFF7F8BF08B10DF0C9BA7047FFF7FABFD3
:10C1200010B4026854681A4623465DF8044B184759
:10C1300000207047012070470020704700207047A2
:10C1400000207047704700000020704700207047B3
:10C15000704700007047000037B505460C46832243
:10C16000011D01A800F03CF9611EC9B202299EBF61
:10C1700005EBC1010023C1E9073301A800F04CF928
:10C1800003B030BD2DE9F7431E461B885B0705460B
:10C19000884620D4011D422201A800F021F92C4636
:10C1A00005F118094C4513D0E3696BB12B6828469B
:10C1B0005B6C98473388276AC1B243F00403E06997
:10C1C0004246B8470834EDE7236A002BEED1F9E781
:10C1D00001A800F021F9012003B0BDE8F0830000C0
:10C1E0007FB56D4685E806000446011D712203A84F
:10C1F0001E4600F0F5F821460022C869D3B288B97E
:10C20000086A78B995E8030004EBC2021C320133D6
:10C2100082E803000124337003A800F0FDF82046F3
:10C2200004B070BD0132032A01F10801E5D10024F8
:10C23000F2E700002DE9F04F2DED028B8BB00446A4
:10C240008B465322011D01A8BDF858809FED258B18
:10C2500000F0C6F8254604F11809002708F0040A82
:10C26000A94536D0EB690BB92B6A63B1BAF1000F5F
:10C270000BD1236820465B6C98474346C1B25A46AF
:10C28000D5E90706B0470835EAE7002FFBD18DED69
:10C29000028BADF810705B4605AA0BF1080C18680C
:10C2A0005968174603C7083363453A46F7D11868FB
:10C2B00038609B88BB8005F0CFFB0423ADF81030BD
:10C2C0002368CDE902019B6C02A92046984701270B
:10C2D000D9E701A800F0A0F801200BB0BDEC028B5B
:10C2E000BDE8F08F0000000000000000082817D90A
:10C2F0000C280CD910280CD914280CD918280CD9C2
:10C3000020280CD930288CBF0F200E207047092020
:10C3100070470A2070470B2070470C2070470D2093
:10C3200070470000082817D909280CD00A280CD01B
:10C330000B280CD00C280CD00D280CD00E2814BFC4
:10C340004020302070470C20704710207047142088
:10C350007047182070472020704700004368184736
:10C360008368184710B5024C8260C0E9004110BDD7
:10C3700004E30108007B00F00100704770470000F3
:10C380008160828070470000826838B504465AB1E7
:10C39000037B13F0010507D143F0010303739047BA
:10C3A000237B65F30003237338BD000010B5044BF5
:10C3B0001B680446986A03681B699847204610BDAD
:10C3C0003825002010B5054B1B680446986A0368A1
:10C3D00000211B699847204610BD00BF382500206A
:10C3E000F8B50C4B01601E680446B06A03681B6C0C
:10C3F00017469847054610B1F36AA3F842702068C3
:10C4000003689B6898471DB1F36A0022A3F8422095
:10C410002046F8BD3825002010B5044600680368A2
:10C42000DB689847204610BDC181B1FA81F0400910
:10C4300070470000C08970477047000000207047B7
:10C4400070470000704700000020704700207047D0
:10C45000704700004FF4B450704700000020704750
:10C460000020704700207047002070470020704770
:10C47000007B70477047000007B503688DF8071010
:10C48000DB6801220DF10701984703B05DF804FB5A
:10C4900008B5036801225B6A98470028D4BF0020D2
:10C4A000012008BD07B503680DF10701DB69984756
:10C4B00020B19DF8070003B05DF804FB4FF0FF309A
:10C4C000F9E7000013B5044608460191FDF736FE72
:10C4D00023680199DB680246204602B0BDE810409F
:10C4E0001847000005F0B8BA10B444682CB90368C6
:10C4F0005DF8044BD3F88030184700205DF8044BFA
:10C500007047000082681AB90368D3F89030184762
:10C510000020704782681AB90368D3F8943018472E
:10C520000020704730B4456825B90468E46FA4461C
:10C5300030BC604730BC704700231A46FFF7F2BF9B
:10C5400010B484680CB19C4206D103685DF8044BBA
:10C55000D3F8843092B2184700205DF8044B70473E
:10C560000023FFF7EDBF0000013901298CBF002037
:10C57000012070470020704700207047002070475E
:10C580007047000000230B707047000070470000E8
:10C59000704700000020704700207047002070475F
:10C5A000704700004368C26893423CBF8268D15420
:10C5B000436801334360012070470000F8B5054629
:10C5C0000C468F180026BC4207D02B6814F8011BBC
:10C5D0009B68284698470644F5E73046F8BD0000BA
:10C5E00000207047002070470020704700207047EF
:10C5F00038B590F89C308B4204460D460CD080F83C
:10C600009C1005F027FA2368C4F8A0005B68204658
:10C61000984708B984F84D5038BD00007FB50D46E5
:10C620001446194600267AB1531E0B4A6846CDE9D6
:10C630000026089ACDE9025300F08EF80198844252
:10C6400004D92E5404B070BD1346EEE7002CF9D087
:10C650002C4404F8016CF5E728E3010808B410B590
:10C6600085B007AC54F8043B00940394FFF7D6FF61
:10C6700005B0BDE8104001B07047000070B5044639
:10C6800003F086FC5E224FF4000103F06DFC0D4EBA
:10C690000D4B1D6833783BB9E86A042221464830C7
:10C6A00005F0DCF901233370EB6A2A2283F8462077
:10C6B000EB6A93F89C301BB90448214605F0A0F9B9
:10C6C00070BD00BFC6360020382500200CE30108ED
:10C6D00007B503680DF10701DB69984720B19DF8A4
:10C6E000070003B05DF804FB4FF0FF30F9E70000EE
:10C6F000F8B506460F4614460025AC420AD033680A
:10C7000030469B699847431C01D12846F8BD7855AF
:10C710000135F2E72046F9E70EB403B503AA036832
:10C7200052F8041B5B680192984702B05DF804EB75
:10C7300003B0704700F010B813B5044608460191E5
:10C74000FDF7FCFC23680199DB680246204602B035
:10C75000BDE81040184700002DE9F04F2DED028B89
:10C7600006468DB0904691F80090B9F1000F00F0A8
:10C77000DE82B9F1250F08D04B1C0393336849467C
:10C780009B68304698470399EDE791F801908B1C20
:10C79000B9F1250F0393F1D00025AA462C461F2C92
:10C7A0003BD8B9F12B0F2DD01CD8B9F1200F2BD0CD
:10C7B000B9F1230F2ED0A9F13003DBB2092B36D803
:10C7C00060064BBF05EB85050AEB8A0A03EB4505BE
:10C7D00003EB4A0A4EBF05F0FF050AF0FF0A44F0DA
:10C7E000200407E0B9F12D0F11D0B9F1300FE2D1DB
:10C7F00044F00104039B13F8019B0393B9F1000F6C
:10C80000CDD126E044F0020444F00404F2E744F001
:10C810000804EFE744F01004ECE77F2CCBD92306A3
:10C8200017D5B9F16C0F14D144F48074E2E7B9F173
:10C830002E0F05D1620600F17A8244F04004D9E758
:10C84000B9F16C0F02D144F08004D3E7B9F1680F5D
:10C85000D0D0A9F14503022B61D809F1200944F099
:10C8600010045FFA89F908F1070828F00708F8E8CA
:10C870000201FDF78BF914F0400F08BF062524F0E4
:10C88000C004B9F1650F08EE100AA4B250D144F00B
:10C89000400427060DD59FED977AF0EEC87AF4EEA6
:10C8A000C77AF1EE10FAC2BF4FF63F73234043F050
:10C8B000400414F0800346D03B2DA94628BF4FF01A
:10C8C0003B0909F101095FFA89F9072717220021BD
:10C8D00006A802930DF02EFB4A46394606A8B0EE94
:10C8E000480A05F0ADFB9DF81830019303F00902EA
:10C8F000012A029B83462FD0A0072FD414F0040FE7
:10C900000CBF00222022019911F00C0758D0002AF8
:10C9100040F0AB82BAF1030F50D8174637E0A9F1C7
:10C920006503022B00F25B8124F01004A4B29AE7A5
:10C93000B9F1660F02D144F08004AAE7002DA8D017
:10C94000013DEDB2A5E70A2D83BF0A2599462F4682
:10C950002F4698BF9946B9E72D22D4E72B22D2E77C
:10C960000427AAEB07072107FFB20AD43368029213
:10C970009B6820213046013F984717F0FF07029A35
:10C98000F4D122B1336811469B6830469847019B29
:10C99000594D13F0080F594B08BF1D46013D04F0D7
:10C9A000100415F8011F002900F0B5800CB12039E2
:10C9B000C9B2336830469B689847F2E70327D0E74F
:10C9C000CDF808B0002B36D0019BD944DB065FFAC6
:10C9D00089F907D59DF81930312B04BF09F1FF39CA
:10C9E0005FFA89F94FFA89F3002B44DDB9F1080F9A
:10C9F00028BF4FF0080914F0800304931ABF2BEAF4
:10CA0000EB730133052302B101330DB1691C0B44F3
:10CA10009A45C4BFAAEB0303DFB214F0090F2FD16C
:10CA200077B3336805929B6820213046013F9847D1
:10CA3000FFB2059AF4E76006DDD45D4504DB1BF127
:10CA4000040FA8BF44F080046B1C06A90B4435B149
:10CA500013F80119302902D1013DEDB2F7E72106A3
:10CA6000C9D505F101095D455FFA89F906DDA5EB38
:10CA70000B05EDB2BFE74FF00109BCE70025BAE7AF
:10CA800022B1336811469B6830469847220708D484
:10CA90003FB1336830219B683046013F9847FFB271
:10CAA000F6E7049B002B47D02BEAEB74ABEB040AB0
:10CAB00006AB9A44ABEB09096D42A34517DBA145D0
:10CAC00015DA9AF80110013CA54219DC002900F0A2
:10CAD000D281336830469B689847631C04D1336821
:10CAE0002E219B68304698470AF1010AE5E730217C
:10CAF000E9E700BF7F96184B58E3010854E30108AB
:10CB0000A34507D19DF81930352B0FD802D1019BD1
:10CB1000DD060BD559B9002F3FF435AE336820211F
:10CB20009B683046013F9847FFB2F4E731213368F4
:10CB30009B6830469847EEE79DF8191031291EBFD3
:10CB4000019B03F0EF030193336830469B689847DD
:10CB5000E5B9336814F0100F14BF452165219B68B7
:10CB600030469847BBF1000F29DACBF1000302935E
:10CB70002D21336830469B6898473021029B092B52
:10CB800023DD01310A3BC9B20293F7E733682E2156
:10CB90009B68304698470235EDB24FF002094B468C
:10CBA0000CAA1A44336812F8181C9B6809F1010991
:10CBB0005FFA89F930469847A945F0D1C9E702D113
:10CBC000019BDC06D1D42B21D3E7336830469B6828
:10CBD00098470299336830319B68C9B2A9E7B9F127
:10CBE000630F37D0B9F1730F4FD0B9F1640F63D130
:10CBF00024F0900714F4807FBFB20DF118097BD0A8
:10CC000008F1070222F007029046516858F8080B15
:10CC1000002904DA404261EB410147F080070A2312
:10CC20004A4600F07BF9A0EB0900C4B27B0640F154
:10CC30009F8027F00109AC421FFA89F980F0D28069
:10CC400007F01403102B03D127F011071FFA87F9FF
:10CC5000AB468FE058F8043B8DF8183001250DF1F4
:10CC60001809200701D4AA451CD84D445746A945A8
:10CC70003FF451AF336819F8011B9B683046984761
:10CC8000002FF4D0013FFFB2F1E758F8049B14F0F5
:10CC9000400F14BF29464FF0FF3148460DF020FEEB
:10CCA0000546DEE7336820219B6830460AF1FF3AEB
:10CCB00098475FFA8AFAD6E7B9F1690F98D0B9F1C7
:10CCC000750F27D124F01004A7B20A2317F4807F30
:10CCD000DBB20DF1180944D008F1070828F0070865
:10CCE000F8E802014A4600F019F9A0EB090027F024
:10CCF0008007C4B2BFB299E758F8040B0028B8BF48
:10CD000040424FF00A024946B8BF47F0800700F0A2
:10CD1000B7F888E724F00607B9F1700FBFB214D056
:10CD20000AD8B9F1580F13D0B9F16F0F17D00DB061
:10CD3000BDEC028BBDE8F08FB9F1780FF7D1F906A1
:10CD400001D547F004071023C0E747F01007F6E7C6
:10CD5000E20601D547F006074FF40473B6E708234F
:10CD6000B4E758F8040B1A46494600F089F8BCE7C6
:10CD7000A346B94619F0100F41D00CAB234413F869
:10CD8000193C302B30D129F016091FFA89F919F016
:10CD9000080744D119F0010F35D0DA4545D904EB25
:10CDA0000A05A5EB0B05EDB2336819F0100F9B686F
:10CDB0003FD030213046984719F0040F08D033682F
:10CDC00019F0020F9B6814BF58217821304698470C
:10CDD0003368AC429B6839D230213046013D9847D8
:10CDE000EDB2F5E7A346C5E719F0040F02D10BF148
:10CDF000010B01E00BF1020B5FFA8BFBC7E719F0A7
:10CE0000860FC4D0F3E73368DA459B680FD9202139
:10CE100030460BF1010B98475FFA8BFBF3E7DA45DD
:10CE200005D9AAEB0B07FFB2BEE72546BCE70027F2
:10CE3000BAE719F0860FCBD019F0020F14BF2B21DF
:10CE4000202119F0800F18BF2D21BFE7651E06AB0A
:10CE500053FA85F5336815F801199B68013CE4B273
:10CE600030469847002CF5D155E6BAF1040F3FF64D
:10CE700077AD002786E5A3457FF44DAE42E600BFBF
:10CE8000082A30B505D10346C008FCD130330B70F9
:10CE90000DE0102A0DD100F00F0202F13003392B02
:10CEA00088BF02F13703000901F8013BF3D10846BE
:10CEB00030BD03460022DCB223F00103023342F10D
:10CEC0000002580840EAC270C31842EB5202180927
:10CED00040EA0270C01842EB1212030A43EA0263EE
:10CEE000181842EB1222030C43EA02431B1842EBD0
:10CEF0001242D31842F100001B0943EA0073C3EB4E
:10CF00004315C3EB85053034020904EB450453EAAD
:10CF1000101001F8014BCED1C9E70000082B30B545
:10CF20000AD10346C00840EA4170C90850EA01042A
:10CF3000F7D13033137013E0102B13D100F00F042E
:10CF400004F13003392B4FEA101088BF04F1370386
:10CF500040EA0170090902F8013B50EA0103EDD1F2
:10CF6000104630BD20F00104023441F10003610895
:10CF700041EAC3710C1943EB5303210941EA0371E0
:10CF80000C1943EB1313210A41EA03610C1943EB1B
:10CF90001323210C41EA0341091943EB13435918A8
:10CFA00043F10003C5B2080940EA0370C0EB401426
:10CFB000C0EB84043035190905EB440550EA13131E
:10CFC00002F8015BCED1CBE770EE600ADFED057AA7
:10CFD000F0EEE00AF4EEE70AF1EE10FA4CBF0120A1
:10CFE000002070470000003410B5B4EE400AF1EEA6
:10CFF00010FA2DED028B0446B0EE608AF0EE418A05
:10D000000FD702F0C5FFA2B24FF4806102F0ACFF6F
:10D0100038EE288AB6EE000A28EE000ABDEC028B34
:10D0200010BDB4EEE00AF1EE10FA07D4B4EE410AF6
:10D03000F1EE10FAC8BFB0EE410AEFE7B0EE600AB9
:10D04000ECE70000884203D39042014628BF114616
:10D0500008467047884203DB90420146A8BF11464C
:10D0600008467047094A136849F2690099B21B0CD7
:10D0700000FB01331360064B186844F2506182B222
:10D08000000C01FB0200186080B2704708230020EA
:10D0900004230020D0ED010A90ED021AD0ED007AB1
:10D0A00060EE200A20EE011A27EE800A88B008B050
:10D0B000704700BF91ED005AD1ED015A91ED026A1F
:10D0C000D0ED006A90ED017AD0ED027A76EE856AB5
:10D0D00037EE257A77EE867AC0ED006A80ED017A28
:10D0E000C0ED027A704700BFD0ED006A90ED017A82
:10D0F000D0ED027A66EE806A27EE007A27EE800A8B
:10D10000C0ED006A80ED017A80ED020A704700BF31
:10D1100090ED007AD0ED017A90ED026AC7EE006AD8
:10D1200087EE807AC6EE007AC0ED006A80ED017A63
:10D13000C0ED027A704700BFD0ED007AF4EE677A56
:10D14000F1EE10FA10D6D0ED017AF4EE677AF1EE36
:10D1500010FA09D6D0ED027AF4EE677AF1EE10FA01
:10D160006CBF01200020704701207047D0ED007A8D
:10D170009FED0F7AF0EEE77AF4EE477AF1EE10FACF
:10D1800014DCD0ED017AF0EEE77AF4EE477AF1EEB6
:10D1900010FA0BDCD0ED027AF0EEE77AF4EE477A83
:10D1A000F1EE10FACCBF012000207047012070473B
:10D1B000FFFF7F7F08B52B2900F28282DFE811F0A4
:10D1C00044004602400233022A021B026801570152
:10D1D0004E016E0158003F01790184014500D400E1
:10D1E0000401EF003901290120010B0191010A021C
:10D1F000E501DF0145005800D101C401B901AA01D0
:10D200009F01C700BE00B700AA009B00700061002C
:10D210002C006D0262025102D0ED016AD0ED007A5D
:10D220009FEDDD6A36EEA77A77EEE67AD0ED026AF8
:10D2300027EE067A67EE867AF1EE666AC0ED016A3D
:10D2400080ED027AC0ED007A08BD90ED007AD0ED55
:10D25000016AD0ED027AF1EE666AB1EE477AF1EE3C
:10D26000677AC0ED006A80ED017AC0ED027A08BDF0
:10D27000D0ED027A036842680260F1EE677A43609B
:10D28000F3E7D0ED007A90ED026ADFEDC36A37EE86
:10D29000867A77EEC67A27EE267A67EEA67ACFE709
:10D2A000D0ED017ADFEDBD5ADFEDBD6A9FEDBD7AAD
:10D2B00090ED006ADFEDBC4A9FEDBC5A67EEA66AAE
:10D2C00027EE877A67EEA57ADFEDB95AE6EE246A93
:10D2D000A6EE057AE6EE257ADFEDB64A90ED026A13
:10D2E0009FEDB55ADFEDB55AE6EE246AA6EE057A53
:10D2F000E6EE257AB5E790ED027AD0ED007A436844
:10D300008360B1EE477AF1EE677A80ED007AC0ED86
:10D31000017A08BD90ED017AD0ED007A8368B1EE14
:10D32000477AF1EE677A80ED027A0360EFE7816871
:10D330000268436841608260036008BDD0ED017AF5
:10D3400083680268F1EE677AC0ED017AF3E790ED49
:10D35000027AD0ED017A0368B1EE477AF1EE677A8E
:10D3600080ED017A83606DE7D0ED007A90ED017A6F
:10D37000DFED935A9FED886A77EE876A77EEC77A7A
:10D3800090ED027A66EEA56A67EE867AB1EE477A8C
:10D39000C0ED016AC0ED007A80ED027A08BD90ED23
:10D3A000026AD0ED007ADFED7C6A436837EE867A58
:10D3B00077EEC67A67EEA67A27EE267A8360C0ED0E
:10D3C000017A80ED007A08BDD0ED027A436883606F
:10D3D000F1EE677A9BE7D0ED026AD0ED007A9FED1F
:10D3E0006E6A37EEE67A77EEA67AD0ED016A67EEDE
:10D3F000867AF1EE666A27EE067AC0ED026ADEE70B
:10D40000D0ED017A8368F1EE677AC0ED027A43606D
:10D4100008BDD0ED026AD0ED007A9FED5F6A4368E7
:10D4200037EEE67A77EEA67ADFED656A67EE867A02
:10D43000C2E782684168036881600260E7E7D0ED77
:10D44000017A90ED007A9FED546A77EE876A77EE65
:10D45000C77A90ED027A66EE866A95E790ED017ADA
:10D46000D0ED027AB1EE477AF1EE677AFBE6D0EDC5
:10D47000007A90ED016ADFED486A36EE677A77EE62
:10D48000867A27EE267A67EEA67A80ED017AD9E6CB
:10D49000D0ED007A4368F1EE677A46E7D0ED007A86
:10D4A00090ED017A9FED3C6A77EEC76A77EE877A56
:10D4B000CFE790ED007AD0ED027AB1EE477AF1EE47
:10D4C000677A80ED007AD0E6D0ED007A90ED017AAF
:10D4D000DFED315A9FED3A6A77EE676A77EE877A29
:10D4E0004EE790ED017AD0ED027A0368B1EE477A0B
:10D4F000F1EE677A80ED027AC0ED007A87E7D0ED31
:10D50000007A436882684260F1EE677AC0ED007A83
:10D51000836008BDD0ED026AD0ED017A90ED007A0B
:10D52000F1EE666AB1EE477AF1EE677AC0ED016A14
:10D53000C7E7D0ED017A90ED007A83684360F1EEA1
:10D54000677AB1EE477A7BE6D0ED016AD0ED027AD8
:10D5500090ED007AF1EE666AF1EE677AB1EE477A05
:10D560006CE690ED027AD0ED007A4368B1EE477A2E
:10D57000F1EE677A80ED017AC0ED027ADCE6D0ED5B
:10D58000027A0368F1EE677AECE6D0ED007A836800
:10D59000F1EE677AF0E700BFF304353FDB26B93ED2
:10D5A00046D0BC3EC9355BBFCF78123E4F0DAABEF8
:10D5B000C6AC6EBF4D1F6BBFF184CABEF63BCC2319
:10D5C000F30435BFF304353F81177E3FA296F93D42
:10D5D000A296F9BDD0ED026AD0ED007A5FED075A50
:10D5E0001FED096A37EEA67A77EEE67AD0ED016A8A
:10D5F00067EEA57AFDE6D0ED006AD0ED017A1FED69
:10D60000106A37EEA67A77EEE67A5FED126A27EEB9
:10D61000067A38E790ED007AD0ED017AB1EE477ADC
:10D62000F1EE677A71E6D0ED016AD0ED007A1FED78
:10D630001B6A37EEE67A77EEA67A5FED1F6AE6E7B9
:10D64000D0ED017A0368F1EE677A55E7D0ED007A04
:10D6500090ED016A5FED256A37EE867A77EEC67A3D
:10D660000FE7D0ED017A90ED026A5FED2A6A36EE9F
:10D67000677A77EE867A27EE267A67EEA67A80EDCD
:10D68000027A44E6D0ED017A90ED026A5FED336AEA
:10D6900037EE867A77EEC67AEDE7D0ED027A1FEDA7
:10D6A000366A1FED367AD0ED006A5FED375A27EE05
:10D6B000877A67EE867AA6EE867AE6EEA57A00E7A6
:10D6C00002F066FCBDE8084040F211124FF4800100
:10D6D00002F04ABC90ED020A90ED017AD0ED007A9A
:10D6E00020EE000AA7EE070AA7EEA70AB1EEC00ACD
:10D6F000704700BF7047000038B5056804462DB17B
:10D70000284604F02FFB2846FEF704FD204638BDCE
:10D7100013460246014801F04DBE00BF1A370020F3
:10D7200013B50422054B0193044601460DEB02009C
:10D73000FFF7EEFF024B1C8002B010BDFFFF3F0061
:10D740000C37002007B5502304228DF80430412304
:10D7500000210DEB02008DF8053006238DF8063010
:10D760008DF80710FFF7D4FF0420FFF7D9FF03B0AF
:10D770005DF804FB00EB0212907B20B91BB192898B
:10D78000120758BF3F20984008447047430608D40A
:10D79000000A08D0054B1B88184214BF0120002046
:10D7A0007047002070470120704700BF10370020ED
:10D7B00010B50B4B1A880B4B01301B6880B2142438
:10D7C00004FB0033824207D9DC898C4203F1140345
:10D7D00004D0013080B2F5E7002010BD0120FCE745
:10D7E0001E3700202037002082898368D20648BF78
:10D7F0001B6818467047000082898368D20648BFBC
:10D800001B6818467047000007B5042300220DEB83
:10D8100003010B48019201F0ADFD9DF80430502B3F
:10D8200007D19DF80530412B03D19DF80630062B1A
:10D8300001D0FFF787FF012003B05DF804FB00BFB4
:10D840001A37002082894368920705D51B68181E85
:10D8500018BF01200B6070470120FBE737B58B89AB
:10D860001446DA070D4605D523684A681344236039
:10D87000012012E09B07FBD50A4B1B68142201A96B
:10D8800002FB0030FFF7DEFF48B1019922686B68A8
:10D890000A44D3581BB15B1A236003B030BD00208B
:10D8A000FBE700BF203700202DE9F04F8BB01F466B
:10D8B0009DF85480069114235343059308F1060301
:10D8C000DBB2054616464FF0000B07935FFA8BFA62
:10D8D00007EB0A1999F80F40002C4CD0062C28D1E0
:10D8E000B8F10B0F21D84846FFF77EFF0446C8B1B8
:10D8F000169B099309AA49463046FFF7AFFF88B146
:10D900001499434652463846FFF734FF099B029369
:10D91000079B0699CDE90003324623462846FFF7C8
:10D92000C3FF18B90BF1010BD0E700200BB0BDE825
:10D93000F08F1499434652463846FFF71BFFB0EB71
:10D94000953FEFD1C5F30423A342EBD10B4C059BCC
:10D95000206809A91844FFF775FF0028E2D0D9F81C
:10D960000430099A1344169A1344069A13602068E7
:10D97000059B1844DAE72046D8E700BF203700208F
:10D980002DE9F04F1F4B5FFA80F8B3F800A0C0F309
:10D99000403348EA03281C4B1E680F4687B00546F3
:10D9A000C0F3042B00211FFA81F9CA4527D9F38956
:10D9B0004345344620D1337C062B0FD13046FFF748
:10D9C0001BFFC8B10023CDE9013300934A4603464B
:10D9D00039462846FFF768FF044609E09B450BD10E
:10D9E00005A93046FFF72EFF0028F5D0059B3B60C8
:10D9F000204607B0BDE8F08F01311436D3E700248C
:10DA0000F6E700BF1E370020203700202DE9F04F39
:10DA100098468DB0142353430693484B9DF8589075
:10DA2000DDF868B004461868069B0E4618440AA93B
:10DA30001746FFF707FF00287DD00023079309F161
:10DA40000603DBB209939DF81CA006EB0A15EB7BDD
:10DA5000002B70D0062B3BD12846FFF7C5FE08905F
:10DA6000002831D0B9F10B0F65D8179B0B930BAA87
:10DA700029463846FFF7F2FE30B39BF80030012B01
:10DA800059D85A1C0BEB83038BF8002041465D608C
:10DA900052464B463046FFF76DFE1B9A0899CDE97A
:10DAA00004B2199A0392189A02920B9A0192099A57
:10DAB000009203463A462046FFF7A8FF00BB9BF8BA
:10DAC0000030013B8BF80030079B01330793BAE726
:10DAD000179A686810440A9A1044A04213D14B4622
:10DAE000524641463046FFF745FE189B1B9A186088
:10DAF000199B1D6000231370104B1868069B184477
:10DB00000DB0BDE8F08F052BDED1031D9C4203D084
:10DB100000F108039C42D7D11B9B201A8008187083
:10DB200052464B4641463046FFF724FE189B18608C
:10DB3000199B1D60E0E70020E2E700BF20370020CE
:10DB40002DE9F04F8BB00025DFF8A4A0079306461F
:10DB50000F4690461560254B1B881FFA85FB5B45D9
:10DB600041D9DAF80000142303FB0B0409A920466D
:10DB700094F81090FFF766FE98B3B9F1060F17D12D
:10DB80002046FFF739FE014658B3149B0593079BC7
:10DB90000297CDE903830023CDE900335A4630468E
:10DBA000FFF734FF0446E0B120460BB0BDE8F08F2C
:10DBB0000998B04204D1149A00233B601370F3E734
:10DBC000B9F1050F0DD1031D9E4203D000F10803EA
:10DBD0009E4206D1149B301A8008187000233B60C7
:10DBE000E2E70135B7E70024DEE700BF1E3700207B
:10DBF000203700202DE9F04798460D88234B044636
:10DC0000C5F30809186809EB890588B000EB85059C
:10DC100007A92846119E95F810A01746FFF712FE97
:10DC200020B90025284608B0BDE8F0870021BAF1E8
:10DC3000060FC8F8001013D12846FFF7DDFD0028B5
:10DC4000EFD0109B0091CDE90383CDE901170B467E
:10DC5000059601464A462046FFF7D8FE0546E1E70D
:10DC60000798A04202D139603170DBE7BAF1050FA5
:10DC7000D7D1031D9C4203D000F108039C42D0D1B0
:10DC8000241AA408002334703B60CBE7203700201F
:10DC90000138C0B204289ABF014B185C00207047BD
:10DCA000BCE301082DE9F04F2DED028B83B0002479
:10DCB0000093931DDBB208EE103A05460E46174658
:10DCC000A246A0464FF0010BE0B2010105EB0010A7
:10DCD00090F80F90B9F1000F5AD0837B3F2B02D9F7
:10DCE0002E4803F08DFE17B1002B08BF3F23C3F170
:10DCF000200EA3F1200C2AFA03F208FA0EFE28FAED
:10DD00000CFC42EA0E0242EA0C0212F0010FC3F1CF
:10DD1000200CA3F12002E3D10BFA02F22BFA0CFC47
:10DD200042EA0C020BFA03F3B9F1060F43EA0A0ABE
:10DD300042EA080813D10B2FD2D8FFF755FD8146D0
:10DD400058B16858FCF7FAF9009B1844C3B218EEB2
:10DD5000102A31464846FFF7A5FF0134B4E748468C
:10DD6000FFF796FF01900028BAD06858FCF7E6F953
:10DD7000009B1844C0B2B9F1050F04BF0230C0B215
:10DD80001028019BACD83088043003443380E4E78A
:10DD900003B0BDEC028BBDE8F08F00BF5CE301086F
:10DDA0002DE9F04F85B00423DFF89890ADF80E30E0
:10DDB00000244FF0140A214B1B881FFA84F84345B6
:10DDC00039D9D9F800300AFB08F15D182F7CB5F875
:10DDD0000EB0062F23D1B8F1000F02D1184803F07E
:10DDE0000FFE28460193FFF707FD0646A8B1019BE9
:10DDF0005858FCF7A3F90022C3B20DF10E013046CA
:10DE0000FFF750FF59464046FFF7D2FC0028E5D106
:10DE1000062F02D0AB899B07E0D40134CBE738460C
:10DE2000FFF736FF0028D9D0BDF80E300433184470
:10DE3000ADF80E00E6E705B0BDE8F08F1E37002014
:10DE40005CE3010820370020437803F01F021F2AFB
:10DE50000FD00278C3F3401342EA032340F2FF12CB
:10DE6000934206D000680138C31C94BF00200120F3
:10DE700070470120704700002DE9F341224FDFF881
:10DE8000908006460D4604247B88A34237D904239C
:10DE90000DEB03012246384601F06CFA9DF805109F
:10DEA000737881EA0302D20618D196F800C09DF873
:10DEB0000400C3F34013C1F340124CEA032340EAC9
:10DEC000022293420AD13268019B534013EA080FA1
:10DED00004D12C80012002B0BDE8F08101A8FFF739
:10DEE000B3FF20B1094B2C801C800020F3E701F028
:10DEF0001F00FFF7CDFE031D1C44A4B2C4E74FF67C
:10DF0000FF732B80F1E700BF1A3700200C37002089
:10DF100000C0FFFF70B50C462046114615461E4650
:10DF20000CF0DEFC831CAB420AD85F22225422187C
:10DF30000330A84206F1580656709CBF0022E254F6
:10DF400070BD00002DE9F74FDDE90D5407468A4604
:10DF5000164609689DF830809B4622469DF83C3065
:10DF6000009328460CF0A8FC4FF000099BF8001025
:10DF70005FFA89F29142019212D9214628460CF0AB
:10DF8000AFFCC0B28442019A07D90BEB8202516800
:10DF9000221A096828440CF08FFC09F10109E5E711
:10DFA000E6B1214628460CF09BFCC3B29C4204D942
:10DFB0003168E21AE8180CF07FFC009B13B9B8F145
:10DFC000000F13D0F37B052B10D143462246294680
:10DFD000384603B0BDE8F04FFFF79CBF009B13B974
:10DFE000B8F1000F02D09AF81030ECE703B0BDE8AA
:10DFF000F08F0000F0B58BB007AC1F460023C4E9DA
:10E00000013307930DF11303CDE90043154606AB29
:10E0100005AA0646FFF7EEFD014610B928700BB0C1
:10E02000F0BD9DF84030069A0195CDE902739DF848
:10E030001330009330462346FFF784FFEFE70000DC
:10E040002DE9F04F984689B014234B43DFF828A1FF
:10E05000039204460E4604934FF000095FFA89F5D7
:10E060002B0108EB0515059395F80FB0BBF1000FD8
:10E070007FD0BBF1060F58F803702AD13846FCF761
:10E080005DF83946024620460CF0E0FB002869D1D5
:10E090002846FFF7A9FB0746002863D0039B079398
:10E0A00007AA29463046FFF7D9FB00285AD0059B1E
:10E0B00058F80300FCF742F8129B0093079A3B467E
:10E0C00031462044FFF7BCFF00284BD009B0BDE823
:10E0D000F08F394620460CF09FFB88B9DAF8000033
:10E0E000049B07A91844FFF7ADFB00283AD0129B08
:10E0F00083F800B06868079B1844039B1844E5E761
:10E10000BBF1050F2ED1102138460CF0E9FB5FFA68
:10E1100080FB5A46394620460CF0BAFB10BB14F976
:10E120000B305F2B1ED10BF1010B14F80B30583B59
:10E13000022B17D8DAF80000049B07A91844FFF750
:10E1400081FB78B16868079B129A1844039B1844B6
:10E150000423137014F90B30592B06D05A2B06D018
:10E16000582BB3D009F1010978E70430AEE7083045
:10E17000ACE75846AAE700BF203700202DE9F04F52
:10E180008BB0DFF8C8B002910446174600252E4B2D
:10E190001B881FFA85FA534552D91422534653431C
:10E1A000DBF8002002EB0309D35899F81080B8F18E
:10E1B000060F33D11021184603930CF091FB039BFB
:10E1C0005FFA80F84246194620460CF061FB06468D
:10E1D000002833D14846FFF70FFB034670B3029A7D
:10E1E000009204EB080032465146FFF729FF8046B3
:10E1F00020B37FB10DF11303009306AA07AB05A965
:10E20000CDE9076605960996FFF79AFC069B0BB1C8
:10E210009B893B8040460BB0BDE8F08F19462046F5
:10E220000CF0FAFA50B9029B07A983F8008048461F
:10E23000FFF708FB20B1DDF81C80EBE70135A6E70E
:10E240004FF00008E6E700BF1E370020203700200F
:10E2500010B590B00023CDE9083306930A930DF171
:10E260001703009306A908AB07AA0446FFF768FC4A
:10E27000014668B111230122CDE902320BAB0193B3
:10E280009DF817300093079A08AB2046FFF75AFE17
:10E2900010B010BDF0B5304D87B040F2A51202901D
:10E2A0008DF80C1006460C4601A8291DFEF798F8BB
:10E2B000052204A9286803F09BFE074601A8FEF783
:10E2C000ABF8052F06D1049BB34203D19DF814305F
:10E2D000A3423ED0214E224F4FF4B072314601A8E6
:10E2E000FEF77EF8286803F0A7FD042821D92868E6
:10E2F000052202A903F016FE431F5C425C4101A8FF
:10E30000FEF78AF82CBB3C68E36A93F89C3093B91B
:10E31000A06A036801211B699847A06A03684FF44B
:10E32000FA719B689847A06A036800211B699847A7
:10E33000D2E70024E3E7A06A03681B6C9847002833
:10E34000E6D001F025FE40F2FA424FF4801101F0D0
:10E350000BFE07B0F0BD00BFE4360020E836002019
:10E36000382500202DE9F341154E164FC92406F13A
:10E370000408013CA4B2FCB140F24B12414601A892
:10E38000FEF72EF8306803F03DFD054601A8FEF7C4
:10E3900043F8042D10D93D68A86A03680A211B6957
:10E3A0009847A86A03680A215B689847A86A0368C7
:10E3B00000211B699847DCE702B0BDE8F08100BF8F
:10E3C000E43600203825002000B58BB00023CDE9CD
:10E3D0000733049309930DF10D03009305AA07ABCE
:10E3E00004A9FFF7ADFB10B3059B23B3DB7BC28908
:10E3F0008DF8182003F01F03C2F300221B0243EA2A
:10E400004233049A43EA82339DF818200DF10E013D
:10E41000134306A80693FFF72FFD40B19DF819306E
:10E4200003F01F03052B03D09DF80D3003B100202E
:10E430000BB05DF804FB037CD9E70000F0B5144F86
:10E440003B8889B006460D46FBB10DF10B03002455
:10E45000009304AA05AB03A9CDE9054403940794EE
:10E46000FFF76EFB88B10B4B38881B68A2B2904255
:10E470000BD91A46013411688E4203F10C03F5D111
:10E48000137A2B70012009B0F0BD0020FBE700BF1C
:10E49000143700200837002013B50DF1070104469A
:10E4A000FFF7CCFF10B92046FFF78EFF02B010BD7A
:10E4B0000138032816D8DFE800F002080E13FDEE3D
:10E4C000C07A17EE903A0B707047BDEEC00A10EE9E
:10E4D000103A0B807047BDEEC00A81ED000A70470C
:10E4E00081ED000A7047000037B5036803F0004370
:10E4F00003600A4B1B880C4613B9002003B030BDE3
:10E50000074D01A92868FFF79DF90028F5D014B13F
:10E510002B681B7C23700198F0E700BF1E3700209A
:10E52000203700202DE9F04F8FB09B469DF87030CA
:10E530000B93142343439DF860901A9D0A9307465A
:10E5400088460892002307939DF81CA008EB0A1642
:10E55000F47B002C00F0BC80B089FFF717F900288D
:10E5600000F0B380062C2FD13046FFF73DF904466A
:10E57000002800F0AA80199B0D930DAA3146384659
:10E58000FFF76CF9002800F0A0804B465246594630
:10E590004046FFF7EFF81D9A05920B9A04921B9ADA
:10E5A000CDE902520D9A019209F10602D2B2034658
:10E5B00000922146089A3846FFF7B4FF002800F081
:10E5C00084800FB0BDE8F08F089B1B780993002B67
:10E5D0003CD02B8867F308032B8052464B465946A4
:10E5E0004046FFF7C7F83B4B03EA40302B6823F067
:10E5F000FF4323F4FF0323F4FC4318431B9B2860D1
:10E6000003B11C70344B18680A9B0DA91844FFF71E
:10E6100019F9002859D00D9A73681344199A98185B
:10E620000B9A002ACDD02D4A1278002AC9D0F27B4D
:10E63000012AC6D1B2895207C3D5199A9B56002B1D
:10E64000BFD1EB7843F08003EB70BAE74B465246FC
:10E6500059464046FFF78EF82B68C3F35133984272
:10E6600033D1089A0123137095F90330002B06DA91
:10E67000EB78099A62F3C713EB701046A1E7052CFB
:10E6800023D16B78C3F34302022A1ED8013262F30E
:10E6900044036B701B9B13B11B9A042313700E4B26
:10E6A00018680A9B0DA91844FFF7CCF868B1706888
:10E6B0000D9C95F801B0199B2044CBF3430B1844F3
:10E6C0000BF1FF3B00EB8B007BE7079B01333AE745
:10E6D000204676E700E0FF7F203700200C23002053
:10E6E0002DE9F04F8BB0DFF8EC9004880792002200
:10E6F0008DF82720B9F800201F46C4F308039A427A
:10E7000005460E461C4662D9DFF8CC801BB2D8F80D
:10E71000001003EB83039A0001EB83031B7C052BA2
:10E7200018D14378C3F34301022915D8013161F3AD
:10E73000440343700EB104233370D8F80010687896
:10E740000A44C0F34300431E506800EB83000BB043
:10E75000BDE8F08F062B04D001340123A4B28DF85C
:10E7600027304FF0140B4FF0000AB9F80030A342E5
:10E770002DD9D8F800200BFB04229089FFF706F86A
:10E78000B8B1117C062917D11046FFF735F80146BC
:10E7900078B1079B0597CDE90363CDE901A5CDF8D5
:10E7A00000A000230DF127022046FFF7BBFE002842
:10E7B000CDD10134A4B2D8E72B68C4F3080403F028
:10E7C000004323432B6006B131705068BFE700203F
:10E7D000BDE700BF1E3700202037002073B5054677
:10E7E0000C461646334601220DF107012846FFF775
:10E7F00077FF28B19DF80730042BF3D804B12370BC
:10E8000002B070BDF8B514460746002220460E46F9
:10E81000FFF76AFE002540B1BD4206D00022314616
:10E820002046FFF7DBFF0135F5E7F8BD0139032985
:10E830000BD8DFE801F00204060800F01BBD00F071
:10E8400051BD00F077BD00F0E1BC9FED010A7047BB
:10E850000000C07FB4EE400AF1EE10FA10B5044695
:10E860000CD69FED327AF0EEC07AF4EE477AF1EEF4
:10E8700010FA03DC042902D180ED000A10BD03293F
:10E8800019D1B5EEC00A9FED2A7ADFED2A7A9FED05
:10E890002A1ADFED2A0AF1EE10FA58BFF0EE477A95
:10E8A00030EE270A40F6C900FEF79EFBBDEEC00A17
:10E8B00084ED000AE2E702291AD1B5EEC00A9FED05
:10E8C0001C7ADFED1C7A9FED1E1ADFED1E0AF1EEB9
:10E8D00010FA58BFF0EE477A30EE270A40F6CE0025
:10E8E000FEF782FBBDEEC00A10EE103A2380C5E7AA
:10E8F0000129C3D1B5EEC00A9FED0D7ADFED0D7A87
:10E900009FED111ADFED110AF1EE10FA58BFF0EE8B
:10E91000477A30EE270A40F6D300FEF765FBFDEE9E
:10E92000C07A17EE903A2370A8E700BFFFFF7F7F01
:10E930000AD7233C0AD723BC0000004F000000CFB9
:10E9400000FEFF46000000C70000FE42000000C3BA
:10E950002DE9F3411D4690F90030232B0F469046D8
:10E960004FF000042CD01749019401AA0CF06AFE64
:10E97000064618B9002002B0BDE8F081FBF7DEFBC7
:10E980001028F7D80F4901AA20460CF05BFE00289A
:10E99000F0D021460CF0D2FD0A4988ED000A01AA08
:10E9A0003E6020460CF04EFE30B10749FBF7BCFB41
:10E9B00010B901202870DEE700232B700120DAE770
:10E9C0002046D8E770E3010877E301082DE9F0431A
:10E9D0004FF000089DB005460E461746A2F800808D
:10E9E000002E35DDB2B200239CB2A24203F1010930
:10E9F00002D9EB5C0A2B29D1632C28BF6324224661
:10EA0000294603A80BF088FA1CAB1C44A6EB0906A8
:10EA100004F8648C9DF90C30232B4D44E0D0002B7E
:10EA2000DED00DF1020302AA01A903A8FFF790FFAF
:10EA30000028D5D0019800220DF10301FFF79EFBBD
:10EA40000028CDD03B8801333B80C9E74B46CBE75C
:10EA500001201DB0BDE8F0832DE9F04FDFF82881DB
:10EA60000546D8F800009FB00E4608B1FDF756FBEA
:10EA7000434FDFF818A1DFF8189100240DF10A02C6
:10EA800031462846C8F800403C80AAF80040A9F862
:10EA90000040ADF80A40FFF799FF00286DD0BDF89F
:10EAA0000A300C205843FDF733FBC8F8000010B9BA
:10EAB000344802F0A5FFBDF80A303B80A346BDF8FC
:10EAC0000A30A34257D9002E55DDB1B2002297B2C9
:10EAD000B94202F1010302D9AA5C0A2A49D1632F83
:10EAE00028BF63273A46294605A801930BF014FA7C
:10EAF0001EAB1F44019B07F864BCF61A1D449DF928
:10EB00001430232BDBD0002BD9D002AB04AA03A9ED
:10EB100005A8FFF71DFF0028D1D0039800220DF1B2
:10EB20000901FFF72BFB07460028C8D00C2303FB85
:10EB300004F2D8F800309850D8F800301344049A02
:10EB40005A609DF808201A7222B1B9F800300133DA
:10EB5000A9F8003001343846A4B2FFF735FC00288C
:10EB6000ADD19DF809109DED040A3846FFF772FEFD
:10EB7000A5E71A46ABE7AAF800301FB0BDE8F08F52
:10EB80001637002084E301080837002014370020DE
:10EB90000437002002460248418A1430FFF75CBF68
:10EBA000C4E30108024B5B8A0BB1FFF7F3BF704768
:10EBB000C4E3010830B5002085B0FFF7F3FF214B17
:10EBC0001A7872B901221A701F4B204A1B680292F0
:10EBD000986A1F4A0368039204AA12E906009B6A16
:10EBE00098471C4D04246B88A34229D9042322464C
:10EBF0006946284600F0BEFB6846FFF725F918B1C4
:10EC0000154B1C8005B030BD009801A9FEF7B8FE79
:10EC100060B19DF8010000F01F00FFF739F8221DD8
:10EC20000346019992B2284600F0A4FB9DF801002A
:10EC300000F01F00FFF72CF804300444A4B2D2E720
:10EC40000020DFE71837002038250020C7360020D5
:10EC50007DF100081A3700200C37002070B50E4BEC
:10EC60001E880E4B1B68002294B2A64209D91C468E
:10EC700001322568854203F10C03F5D194ED010AB8
:10EC800070BD8B891B0649BF8B6891ED020AC01AC3
:10EC900090ED000AF4E700BF143700200837002089
:10ECA0002DE9F04105460F464FF000085FFA88F362
:10ECB00007EB0311CC7BDCB1042C0BD84E682E443F
:10ECC0003046FFF7CBFF31462046FFF7F1FB08F156
:10ECD0000108EBE7052CFAD14C682C442046FFF7DD
:10ECE000BDFF84ED000A84ED010A84ED020AEEE71F
:10ECF000BDE8F08170B50E4B1E880E4B1B680022DC
:10ED000094B2A64209D91C4601322568854203F116
:10ED10000C03F5D194ED010A70BD8B891B0649BF28
:10ED20008B6891ED020AC01A90ED000AF4E700BF6B
:10ED300014370020083700202DE9F0418AB0002365
:10ED4000CDE90733039309930DF10903009304AA56
:10ED500007AB03A90446FEF7F3FE054620B90026DB
:10ED600030460AB0BDE8F081049B002B3AD0DB7B33
:10ED7000EA898DF8142003F01F03C2F300221B025E
:10ED800043EA4233039A43EA82339DF814200DF19B
:10ED90000A01134305A80593FFF76EF8064658BB12
:10EDA00006A92846FEF74EFD0028D9D09DF815701B
:10EDB0000499DDF8188007F01F07B9B19DF81C30E1
:10EDC00093B1089A012B556802D0099B5B681D44DA
:10EDD0002046FFF743FF4968414429443846FFF77E
:10EDE00067FBBDE7037CC3E73546F1E729462046CC
:10EDF000FFF780FF4146F1E79DF815009DF80930C7
:10EE000000F01F02052A0FD0002BA8D100F01F0030
:10EE1000FEF73EFFBDF80A200432034692B22146B7
:10EE2000044800F0A7FA9BE7002BEFD0A4EB830483
:10EE3000ECE700BF1A3700202DE9F04385B0FEF75C
:10EE4000E3FC134E134F00254FF014083288ABB289
:10EE50009A4219D91C463B6808FB043494F8109078
:10EE6000B9F1040F0ED803A92046FEF7EBFC48B118
:10EE7000039801902146FFF73DFF0198014648465F
:10EE8000FFF716FB0135E1E705B0BDE8F08300BFF1
:10EE90001E370020203700202DE9F347DFF88C9043
:10EEA0001F4940F678226846FDF79AFAB9F80070D3
:10EEB0002FB11C4B1A881C4B1B889A4228D0194E24
:10EEC000194D05244FF00008B9F800701FB13288C1
:10EED0002B889A421CD0013C14F0FF0418D0002269
:10EEE000114601A83788CDF80480FFF7FDFA4FF0EE
:10EEF000000A1FFA8AF30AF1010A28B1002211461A
:10EF000001A8FFF76BFCF4E7A9F800302F80DBE7DE
:10EF10006846FDF781FA384602B0BDE8F08700BFC9
:10EF2000C836002002370020123700200E3700209C
:10EF3000024A138801331380704700BF0237002054
:10EF40002DE9F0412DED028B90B00023CDE908337F
:10EF500005930A930DF1110300930E4608AB06AA20
:10EF600005A90446FEF7ECFD0546D8B10699F1B1B6
:10EF7000CA7BEB898DF81C3002F01F02C3F300201E
:10EF80001302059A9DF8117043EA403343EA823335
:10EF90009DF81C201A43C3F30423052B079200F0AD
:10EFA000868037B110B0BDEC028BBDE8F081027CE9
:10EFB000DFE7012B05D121B18B895B0701D5FFF775
:10EFC000B7FF274677E0BDF812204FF6FF739A424D
:10EFD0000AD14C4B83F800804B4B4C491B68986915
:10EFE00003681B689847DDE79DF81D1001F01F01BD
:10EFF000042925D99DF81D00BDF81220444900F0D0
:10F000001F00FEF745FE4988131808338B424AD289
:10F010000432104480B2FEF783FB9DF81D0000F01F
:10F020001F00FEF735FEBDF812100431024689B20A
:10F030003846FEF76DFBBDF81210042207A85EE00B
:10F040002046FFF7F3FB0699F0EE408A71B12046A7
:10F05000FFF704FEB0EE408AF0EE400AB0EE680A18
:10F06000FDF7B2FF38B1002EC4D19BE729462046F8
:10F07000FFF740FEEEE7002EBCD19DF81D3003F0F7
:10F080001F03032BB6D09FED230A38EEC88AF0EE9B
:10F09000E88A68EE808AB0EEC88AB4EEE88AF1EEBB
:10F0A00010FAA7D57EE7174B01221A7094E7002FBC
:10F0B00087D0A4EB870711234FF00108CDE9023870
:10F0C0000BAB01939DF81130009329462046069A18
:10F0D00008ABFEF737FF0DF1120107A8FEF7CCFED3
:10F0E00000283FF470AF9DF81D0000F01F00FEF7F0
:10F0F000CFFDBDF812100431024689B23846FEF742
:10F1000007FB4FE70037002038250020ACE301085B
:10F110001A37002017B7D1387FB5164D2E1D40F293
:10F120007F12314601A8FDF75BF9286802F06AFEFC
:10F13000042812D92868052202A902F075FF431F8E
:10F140005C425C4101A8FDF767F944B19DF80C10E1
:10F1500002980122FFF7F4FEE1E70024F2E7064BF4
:10F160001B68986A03685B6B984708B1FFF794FEC9
:10F1700004B070BDE436002038250020FFF7CCBF76
:10F1800010B50446FCF7C6FF204610BD38B511483F
:10F19000114D01F0C3FE114A11490E480AF092FECA
:10F1A0002846002340F8043B01F0B8FE1420FCF789
:10F1B000A9FF044610B19B2102F0C2FD0949074A8C
:10F1C00005482C600AF07EFEBDE838400648002164
:10F1D00000F0C8B8C8360020E4360020843F002084
:10F1E000F5D60008F9D600081A370020D1ED007ACC
:10F1F00090ED007AF4EE477AF1EE10FA04D0C0ED0B
:10F20000007A0121FFF746B87047000090ED000A30
:10F210007047000091F9002090F90010914202D04F
:10F220000270FFF715B8704791F9001090F900309F
:10F230009FED097A01705B1A07EE903AF8EEE77AD3
:10F24000F0EEE77AF4EEC77AF1EE10FA4CBF012146
:10F250000021FFF71FB800BF0000003491F9002023
:10F2600090F90010914203D002700121FFF712B80B
:10F270007047000090F9003000EE103AB8EEC00A76
:10F280007047000038B504460D46FFF705F910B980
:10F29000B5F90030238038BDB1F90010B0F9003065
:10F2A0009FED097A01805B1A07EE903AF8EEE77A53
:10F2B000F0EEE77AF4EEC77AF1EE10FA4CBF0121D6
:10F2C0000021FEF7E7BF00BF00000034B1F90020C5
:10F2D000B0F90010914203D002800121FEF7DABF9D
:10F2E00070470000B0F9003000EE103AB8EEC00AE6
:10F2F0007047000038B504460D46FFF7CDF808B951
:10F300002B68236038BD00000B6803607047000065
:10F310000A6801688A4202D00260FEF799BF70470E
:10F320000A6801688A4203D002600121FEF7B2BF79
:10F330007047000090ED000AB8EEC00A7047000068
:10F3400008B5064B1B68586903685B68984720B985
:10F35000BDE80840024801F057BE08BD382500202E
:10F36000D8E40108017011B10023438070474FF4C5
:10F370004873FAE770B51C460378A3B9B2F5487F25
:10F3800011D212FA84F3B3F5487F094B1B68586910
:10F39000C8BFC2F548750368D4BFA5B2ADB29E68B8
:10F3A0002B46B047641BB4FA84F0400970BD00BF1F
:10F3B0003825002070B51C460378A3B9B1F5487F05
:10F3C00011D211FA84F3B3F5487F094B1B685869D1
:10F3D000C8BFC1F548750368D4BFA5B2ADB2DE6839
:10F3E0002B46B047641BB4FA84F0400970BD00BFDF
:10F3F0003825002010B5044B044918600446FFF777
:10F400004FFC204610BD00BF243700204CE501080A
:10F4100090F8233063B9012380F823300548006851
:10F420004FF40073006C80224FF4E131FDF77AB89D
:10F43000704700BF38250020002850DD6F2846D0D7
:10F440001BDC132845D00EDC431E082B11D8082BDB
:10F4500033D8DFE803F04105323632323232390038
:10F460004FF416607047392839D064283AD02628DE
:10F470003AD04FF47A7358437047B0F5FA7F36D0DC
:10F4800010DCB0F5807F34D006DC732834D0E62859
:10F49000EFD14FF461307047B0F5E67FE9D14FF41A
:10F4A000E120704740F2DC53984228D0B0F5FA6F63
:10F4B00027D040F29933984225D0B0F5FA6FD8DDC5
:10F4C00070474FF4965070474FF4165070470F48EE
:10F4D00070474FF4964070474FF4966070474FF472
:10F4E000614070470A4870474FF41640704709481A
:10F4F00070474FF47A3070474FF4E1307047064858
:10F500007047064870474FF46120D9E7FCB101000D
:10F51000A086010020A1070060E3160080841E0081
:10F520000068FFF789BF00000E4B70B51D68CBB2B5
:10F53000092B0C4612D8103355F8232000EBC103D9
:10F54000116810464E6B9988B04750B9A8690649B2
:10F55000036822461B68BDE87040184700231B68FB
:10F56000FFDE70BD38250020F8E401082DE9FF41D9
:10F57000FF23804603A921308DF80C30FFF76EFE83
:10F580004046FFF745FF564B1B68019308F10804FE
:10F5900001267327019A06F1100352F82350E671F1
:10F5A0007DB3B1B24046FFF7BFFF94F90630013397
:10F5B000332B00F28C80DFE803F0241A1A1A2C3364
:10F5C00035353D478A338A528A8A245A8A8A698A1B
:10F5D0008A4C8A7D8A8A8A8A8A248A8A8A8A8A8A3C
:10F5E0008A8A8A8A8A8A1A8A8A8A8A8A8A242046FF
:10F5F000FFF796FF4FF48073014680222846FCF700
:10F6000091FF0136042E04F10804C3D104B0BDE813
:10F61000F081092303A920460393FFF775FEF0E765
:10F620003923F7E72046FFF77BFF102301464FF40D
:10F630008072E3E703A920460397FFF765FE802366
:10F640001A464FF4E131D9E703A920460397FFF7A3
:10F650005BFE2046FFF764FF80230146CDE70923C8
:10F6600003A9A01D8DF80C30FFF7DEFDC9E703A943
:10F6700020460397FFF748FE2046FFF751FF1E2361
:10F6800001461A462846FCF74DFF0DE02046FFF7DD
:10F6900047FF802301461A462846FCF743FF2B68A4
:10F6A0000121DB6C284698472B680021DB6B28463C
:10F6B0009847A6E703A920460397FFF71BFE2046BD
:10F6C000FFF72EFF102301464FF40072DAE72046C1
:10F6D000FFF726FF01462846FCF72EFF91E700BF03
:10F6E000382500204FF0FF33002110B50022436180
:10F6F0000446417200F12003E830D9709A60DA6064
:10F700001A615A629A62DA621A635A639A63DA6316
:10F710001A645A645A659A65DA6564338342ECD197
:10F72000044B1A6822B904491C602046FFF7B8FA56
:10F73000204610BD28370020F4E5010890F822107B
:10F7400029B9012343841170837118467047002042
:10F75000704700004FF000007047000041B103798E
:10F76000012B05D05A1C027140F82310012070476C
:10F770000020704711B990F82100704700207047B1
:10F7800038B590F90530044633B390F803311BB314
:10F7900000252279EBB29A4206D954F82300036877
:10F7A0009B6898470135F4E702F054F9A36EC01A3C
:10F7B000B0F5FA7F94F9E8302CBF0020012084F8DE
:10F7C000210013B1002384F8053194F80511204677
:10F7D000BDE83840FFF7CEBF002038BD024690F9A3
:10F7E0000500B0B192F8030198B1D2ED0D7A9FED0A
:10F7F000097AF4EEC77AF1EE10FA09D4B7EE087A76
:10F80000F4EEC77AF1EE10FAD4BF01200020704761
:10F8100000207047ABAA2A3F014B1868704700BF11
:10F820002837002010B50446006810B103685B68F3
:10F830009847204610BD000037B5D0F8F42012F4E8
:10F840008034054617D10D4B0D491B689868036835
:10F850001B6898472246CDE900042146684600F01F
:10F8600043FB01462846FFF779FF6846FFF7DAFFBA
:10F8700001A8FFF7D7FF03B030BD00BF3825002037
:10F88000ACE5010810B50446FFF7D6FF23790BB1AC
:10F89000A37943B9044B05491B6898690368BDE81F
:10F8A00010401B68184710BD38250020B4E501083A
:10F8B00010B590F9053004461BB3012380F80431DC
:10F8C000836B13B1002280F804212364A37923B948
:10F8D0002046FFF7D7FFA3794BB10A4B1B68986A04
:10F8E000036864215B6898472046FFF749FF94F856
:10F8F000223003B9A363012384F80331002384F881
:10F90000043110BD38250020064B10B503600446B5
:10F91000FFF782FF606004F1080001F0FFFA204663
:10F9200010BD00BF4CE60108F7B5054664276C68BA
:10F93000164607FB024306FB0744084693F870107F
:10F940000190FDF737FC94F92030019833B96B68CA
:10F95000597A03B0BDE8F040FDF72CBC94F82410B0
:10F96000F7E700002DE9F04146684FF064080746CC
:10F970000D4608FB0261144628312846FDF79AFB24
:10F9800078682146FFF72AFF40B108FB046494ED34
:10F990000D0A2846BDE8F041FDF7A6BBBDE8F081A1
:10F9A00010B54368642404FB023407C904F15C0306
:10F9B00083E8070002F04EF8A06602F047F8E06620
:10F9C00010BD0000F0B5074685B00D46164600F1A3
:10F9D0000801A72203A8FCF703FD7C68642303FB4E
:10F9E0000543D3F8802022B903A8FCF715FD05B024
:10F9F000F0BDBEB196ED007AD3ED1D7A67EE877A41
:10FA0000C3ED1D7A96ED017AD3ED1E7A67EE877A03
:10FA1000C3ED1E7A96ED027AD3ED1F7A67EE877AF0
:10FA2000C3ED1F7A642607EE902A06FB0541743168
:10FA3000B8EE670A08460191FDF76AFB01992A466C
:10FA40003846FFF7ADFF06FB05410023CB678B6708
:10FA50004B670023C1F88030C6E700004068FFF71D
:10FA60006DBE0000F7B5064640680192642707FBAB
:10FA700001000D46383001A91446FFF749FC7168B2
:10FA800007FB0515EC6303B0F0BD000013B5436838
:10FA900064200C4600FB013191F92010022908D0A6
:10FAA00020330DF1070104FB00308DF80720FFF72C
:10FAB000B1FB02B010BD00004368642000FB0131BF
:10FAC00081F8702070470000F8B5054608460F46DB
:10FAD000FDF74CFB10B100242046F8BD3846FDF779
:10FAE0002BFB04460028F6D16B6893F9F8607EB1D1
:10FAF0003846FDF7EFFD95ED087ADFED1F7AF0EE61
:10FB0000C76AF4EEE76AF1EE10FA03D585ED080A4C
:10FB10000124E1E777EE407A30EE076AF0EEE77A0B
:10FB2000C7EE866AF6B207EE906A9FED146AF8EEA9
:10FB3000677A26EE866AF4EEC67AF1EE10FA48BFCE
:10FB4000B2EE046ADFED0E7A45BF6B6A66EE866A36
:10FB5000B0EE676A87EEA66A46BF01336B62012486
:10FB6000F7EE007A77EEC67A20EE060AA7EE270AAD
:10FB700085ED080AB0E700BF0000003400004843EC
:10FB8000CDCCCC3D2DE9F74304460E4615461F4625
:10FB9000FFF7CAFE314620462A46FFF7E3FE31460C
:10FBA0002046FFF791FF28B3992204F1080101A82C
:10FBB000FCF716FC64684FF0640909FB054808F17E
:10FBC000740831464046FDF775FA09FB0542D2F844
:10FBD00080100131C2F880104FB1B94207D34908F3
:10FBE000C2F88010B0EE000A4046FDF791FA01A875
:10FBF000FCF712FC03B0BDE8F083000090F82C1075
:10FC00000022FFF7DFBE0000F8B504460D46174698
:10FC10001E46FFF779FE074B23602B68A362002284
:10FC20004FF07E532A6084F82D7084F82E60236391
:10FC30002046F8BD90E601087FB50446806A036857
:10FC40009B6A984703689B689847A06A037A03F009
:10FC50000703022B02D1802102F070F8A06A03682A
:10FC60000A21DB6C9847A06A01230DF103020421ED
:10FC700001F0EAFF50B9A06A03689B6A98470368DD
:10FC8000DB6898470025284604B070BDA06A0123B0
:10FC90000DF10202052101F0D7FF0028EBD0A06A88
:10FCA00001230DF10502062101F0CEFF0028E2D06C
:10FCB000A06A012301AA072101F0C6FF0028DAD0BB
:10FCC000A06A01230DF10702082101F0BDFF002801
:10FCD000D1D0A06A01230DF10602092101F0B4FF81
:10FCE0000028C8D09DF80230C82BC4D19DF804303C
:10FCF000C82BC0D19DF805209DF8033013439DF813
:10FD000007201343B7D19DF80630C82BB3D10A2280
:10FD10000821A06A01F01EFF012394220B21A06A92
:10FD200001F06EFF012319467122A06A01F068FFFD
:10FD3000012300220421A06A01F062FF0123C822EE
:10FD40000521A06A01F05CFF012300220621A06AC0
:10FD500001F056FF0123C8220721A06A01F050FFDD
:10FD6000012300220821A06A01F04AFFC8220123D2
:10FD70000921A06A01F044FFA06A254B23630368B0
:10FD80000321DB6C9847A06A03689B6A9847036865
:10FD9000DB689847A06A112101F0F4FEA36A04F120
:10FDA0002C0299682046FFF759FE054600283FF4CB
:10FDB0006AAFA36A94F82C109A682046FFF752FEA7
:10FDC000144BA26A1B68527A9869134903681E682B
:10FDD00094F82C30B04794F82E2094F82C1020463C
:10FDE000FFF76AFE94F82D302BB194F82C10012205
:10FDF0002046FFF74BFEA06A02940368DE6A074BB9
:10FE0000039304AB13E90C0043F2D401B0473AE783
:10FE10008988083E3825002058E60108E5FE0008DC
:10FE200010B588B004460123806A0DF10702342121
:10FE300001F00AFF002850D09DF90730002B4CDA62
:10FE4000A06A092302AA242101F0FEFE002844D062
:10FE50009DF809109DF808309DF80C209DF80E00C3
:10FE6000D4ED0C6A090441EA03619DF80A3041EAC5
:10FE700003219DF80B30120442EA03629DF80D3015
:10FE8000091242EA03229DF80F3007EE101A1B04F4
:10FE900043EA0063B8EEC77A9DF8100027EE267A91
:10FEA00043EA002312121B1207EE903A8DED057AF9
:10FEB00007EE102AF8EEE77AB8EEC77A67EEA67A70
:10FEC00027EE267A94F82C208DED067A0A2305A9D0
:10FED0002046CDED077AFFF755FEA06A01F0D8FE67
:10FEE00008B010BDFFF79CBF30B51346026885B05F
:10FEF0000D461AB90024204605B030BD002101602E
:10FF0000342001930392FCF7FDF8044620B1019BD5
:10FF10002A4603A9FFF778FE03A8FFF783FC002C0D
:10FF2000E8D02046FFF788FE05460028E3D1236885
:10FF300020465B6898472C46DDE7000010B5044B6F
:10FF4000044640F8283BFFF76DFC204610BD00BF7B
:10FF500090E6010810B50446FFF7F0FF2046FCF7D5
:10FF6000D9F8204610BD000010B50368028119437E
:10FF70004368016001334360044B1B68DC6AA16283
:10FF8000D96A40688885DB6ADA8510BD382500208B
:10FF9000004870472C37002008B50449FAF7C4F828
:10FFA0000028034818BF002008BD00BF9CE60108D8
:10FFB000AC3E020810B50C46FFF7EEFF10B18368A7
:10FFC0002360006910BD00007047000010B4064BAC
:10FFD000064A1B680649986903681C68537E127EAE
:10FFE000A4465DF8044B60473825002000920008C5
:10FFF000C03E020810B41346026814680022A446EA
:020000040801F1
:100000005DF8044B6047000000F5805090F88104D3
:100010007047000000F5805090F87A0470470000A7
:1000200000F5A5507047000000F5805090F980045D
:100030007047000050207047302383F3118800F58B
:100040008052D2F8C434D2F8C0041844D2F8BC3478
:100050001844D2F8A4341844D2F8B4341844D2F86E
:10006000B0341844002383F31188704700F58050A2
:10007000C0F87C14012070472DE9FF47054600F5C4
:1000800080500C4690F87A14BDF830A099B1D0F8A1
:10009000A0140131C0F8A01421688E0006D4217B81
:1000A00008290BD9667B0EB10F2907D9D0F8A434E3
:1000B0000133C0F8A4344FF0FF30A4E0302181F3C5
:1000C0001188696DD1F8C46016F4001813D0D0F807
:1000D000A8140131C0F8A814D0F8AC14002940F0DD
:1000E0009580CDF800A021462846FCF7A3F8002310
:1000F00083F3118887E0D1F8C4702668E96CC7F3F0
:1001000001474FF04809002E19FB0719B4BF46F00C
:100110008046B604C9F800602168490044BF46F033
:100120000056C9F80060267B390641EA0641C9F845
:10013000041094F80DC07E01BCF1000F27D041F4EB
:100140004011C9F80410D0F8D8140131C0F8D814FF
:10015000A91901F58451087D40F020000875207B25
:10016000CDE90223FCF7DEF8DDE90223033080103D
:100170005FFA88F1814208F101080FDA04EB810C83
:1001800009EB8101DCF804C0C1F808C0F0E7A91947
:1001900001F58451087D6CF34510DFE7696D01209E
:1001A000B840C1F8CC00A91901F58351C1E9062373
:1001B000A7F17C01C9B2204605EB411104F10C0CFA
:1001C00050F804EB41F804EB6045F9D10088088051
:1001D0002E4441F29001775006F580560AF0030153
:1001E00096F8940041F0100120F01F00014386F8BA
:1001F0009410002181F31188CDF800A021462846F3
:10020000FCF718F8012004B0BDE8F08700206EE785
:1002100038B5426D936923F001039361044601F000
:1002200019FC0546636D9B69DB0706D501F012FCDE
:10023000431BFA2BF6D9002004E004F5805401207A
:1002400084F87A0438BD000030B52DED028B0446E9
:10025000A1B00D46302383F3118804F580540220A9
:1002600007F06CFED4F8DC341C93D4F8D8341B931C
:10027000D4F8E0341A93D4F8D4341993D4F8D034A1
:100280001893D4F8C4341793D4F8C0341693D4F820
:10029000BC341593D4F8B8341493D4F8B43413930D
:1002A000D4F8B0341293D4F8AC341193D4F8A83401
:1002B0001093D4F8A4340F93D4F8A0340E93B4F868
:1002C0008A349FED248A244AB0FBF2F207EE903A7A
:1002D000F8EEE77A1F9267EE887A17EE900AF9F740
:1002E00005F9CDE90C0194F890340A9394F88F3411
:1002F000099394F88E340893B4F88C340793D4F8A7
:1003000098340693B4F8823407EE903AF8EEE77A20
:1003100067EE887A17EE900AF9F7E8F8CDE904015C
:1003200094F88834039394F88734029394F88634CD
:100330000193B4F884340093D4F894341F9A074995
:10034000284601F0C9FB002383F3118821B0BDECDE
:10035000028B30BDCDCCCC3D40420F00D03E0208D8
:1003600013B500F580540191E06E01F065FD1F2882
:100370000AD90199E06E202201F0D4FDA0F12003FA
:100380005842584102B010BD0020FBE708B53023A9
:1003900083F3118800F58050C06E01F021FD002329
:1003A00083F3118808BD0000002202608281426050
:1003B0008260704710B500220023C0E900230023AB
:1003C000044603810C30FFF7EFFF204610BD00000C
:1003D0002DE9F0479A4688B0074688469146302373
:1003E00083F3118807F580546846FFF7E3FFE06E5A
:1003F00001F008FD1F282DD9E06E2022694601F08A
:1004000013FE202826D194F87A341BB303AD44465A
:1004100005AB2E4603CE9E4220606160354604F156
:100420000804F6D130682060B388A380DDE900239A
:10043000C9E90023BDF80830AAF80030002383F38F
:10044000118853464A464146384608B0BDE8F04751
:10045000FBF798BE002080F3118808B0BDE8F08754
:100460002DE9F84F2E4B054640F8043B88462E46B2
:1004700000F054FD1822002105F11C0009F05AFD7E
:10048000284B46F8583B05F5825437461834384611
:100490002037FFF78FFFA742F9D105F580544FF4BD
:1004A0008053A6650026C4E91736E766012305F5E3
:1004B000845705F5A459666684F8683084F870306E
:1004C000183709F118094FF0000A4FF0000B47E9FF
:1004D00008ABA7F11800FFF767FF203747F8286C33
:1004E0004F45F4D184F88084A4F88264A4F884642D
:1004F000A4F8866484F88864A4F88A64A4F88C64F8
:10050000A4F88E6484F89064B8F1000F02D0064815
:1005100001F076FA054B6B652846BDE8F88F00BF01
:10052000B0E2010804410208E8400208006400400B
:1005300010B5044B197804464A1C1A70FFF790FF57
:10054000204610BD3D3700202DE9F84315460C46E6
:1005500000295CD0022007F0F1FC2E49B0FBF4F733
:100560008C428CBF0A2111214B1EB7FBF1F601FB17
:100570001671DAB221B1022B1946F5D8002032E00B
:10058000731EB3F5806FF9D2C2EBC20808F1030104
:100590004FEAE10EC1F3C701A2EB010C0EF1010914
:1005A0004FF47A735FFA8CF70EFB033E59FA8CFC1A
:1005B000BEFBFCFCBCF5617F17DC1FFA8CF34A1C08
:1005C00057FA82F27243B0FBF2F08442D6D14A1E4F
:1005D0000F2AD3D87A1E072AD0D801202B806E800C
:1005E00028716971AF71BDE8F88308F1FF314FEAF6
:1005F000E10CC1F3C701521A0CF1010ED7B20CFB8A
:1006000003335EFA82F2B3FBF2F39BB2D7E70846FC
:10061000E9E700BF3F420F0030B50D4B0D4D0520FF
:100620001C786C438C420ED1597851809978517165
:10063000D9789171197911715B7903EB83035B00B0
:100640001380012030BD013803F10603E8D1F9E73A
:100650005041020840420F000B4B10B54FF454724A
:1006600004460021184609F065FC084B236440331A
:100670006364D833A364F033E364636DE063002202
:10068000C3F8C02010BD00BF00A4004070A400400B
:100690002DE9F04F00F580551F4695F88034012B69
:1006A00089B004468946904604D90026304609B0F0
:1006B000BDE8F08F9E4A52F8231041B942F823005A
:1006C00000F06EFE95F8803400EB8300C463994817
:1006D000C4F83490017884F8387099B9302383F3E2
:1006E0001188954B9A6D42F000729A659A6B42F0B0
:1006F00000729A639A6B22F000729A63012303706E
:1007000081F3118895F879647EB9302383F31188D9
:100710000321152007F034FD0321162007F030FDDA
:10072000012385F8793486F31188302383F3118807
:10073000626D936923F01003936101F08BF9824697
:10074000636D9E6916F0080609D001F083F9A0EBED
:100750000A03FA2BF4D9002686F31188A6E79A69D2
:1007600042F001029A6101F075F98246636D9A695F
:10077000D00706D401F06EF9A0EB0A03FA2BF5D9E5
:10078000E9E79A6942F002029A61636D4FF0000A4C
:10079000C3F854A08AF31188E86E01F021FB04F538
:1007A000835B0BF1180B20220021684609F0C2FB85
:1007B00002A8FFF7F9FDCDF818A06A460BEB060377
:1007C0000DF1180E9446BCE80300F445186059601A
:1007D000624603F10803F5D1DCF80000186020360A
:1007E0009CF804201A71B6F5806FDCD1002304F563
:1007F000A45285F8783485F87B3402324946204685
:10080000FFF7A2FE064690B9626D936923F00103DB
:10081000936101F01FF90546636D9B69D9077FF568
:1008200044AF01F017F9431BFA2BF5D93DE795F8D2
:100830008634C5F89494591E95F88734626D013B4F
:100840001B0243EA416395F8881401390B43B5F85C
:100850008414013943EA0143D361B8F1000F36D063
:1008600004F5A4520A3241462046FFF7D5FE90B95E
:10087000626D936923F00103936101F0EBF8054683
:10088000636D9B69DA077FF510AF01F0E3F8431B56
:10089000FA2BF5D909E795F88F24C5F89884511EED
:1008A00095F89024636D013A120142EA012295F80D
:1008B0008E1401390A43B5F88C14013942EA014219
:1008C00042F40002DA60636D4FF420629A642046BD
:1008D000FFF7C2FE002385F88134636D6FF040425C
:1008E0001A65636D154A5A65636D44229A65636D96
:1008F0000722C3F8DC20636D03229742DA653FF4D8
:10090000D5AE626D936923F00103936101F0A2F803
:100910000746636D9B69DB0705D501F09BF8C31B98
:10092000FA2BF6D9C1E6012385F87A34BEE600BF7A
:10093000383700203C370020001002409B000800A0
:100940002DE9F04F00F5A6578BB004469046994626
:100950004FF0000B41F2900A1037636DD3F8D4309A
:1009600023FA0BF3DD0752D504EB4B1151444FEA48
:100970004B120B7918074AD404F58056D6F8AC34DC
:100980000133C6F8AC3447E902890B79990648BFB0
:10099000D6F8DC3404EB020148BF0133514448BFB0
:1009A000C6F8DC340B7943F008030B71DB0723D561
:1009B00096F87B3403B302A80192FFF7FBFC019A7F
:1009C00004F58455154405AB05F1080C28686968E1
:1009D0001A4603C2083565451346F7D128681060EA
:1009E000AA889A800123ADF810302368CDE90289E6
:1009F0009B6C02A920469847D6F8D034D6F87C04E0
:100A00000133C6F8D03410B103681B6998470BF165
:100A1000010BBBF1200FA0D10BB0BDE8F08F00009F
:100A20002DE9F04F8DB004460F4601F015F88246CF
:100A30008946002F56D1636DD3F89020920141BFB3
:100A400004F58051D1F8C0240132C1F8C024D3F894
:100A50009020160703D100200DB0BDE8F08FD3F829
:100A60009050666CC5F30125482303FB0566E846F4
:100A70004046FFF799FC326851004ABF22F06043BC
:100A8000C2F38A4343F00043920048BF43F08043DF
:100A90000093736813F400131FBF04F58052012301
:100AA0008DF80D30D2F8E0340EBF8DF80D300133E3
:100AB000C2F8E034F38803F00F038DF80C304FF0E8
:100AC000000B9DF80C00FBF72DFC5FFA8BF39842AE
:100AD00020D9F2180CA90B44127A03F82C2C0BF134
:100AE000010BEEE7012FB6D1636DD3F89820950185
:100AF00041BF04F58051D1F8C0240132C1F8C024AF
:100B0000D3F898201007A6D0D3F89850A66CC5F358
:100B10000125A9E7EFB9636DC3F8945004A8FFF766
:100B200049FC98E80F0007AD07C52B800023ADF8FE
:100B3000183023682046CDE904A99B6C04A9984786
:100B400004F5805458B1D4F8B8340133C4F8B8343B
:100B500082E7012F04BF636DC3F89C50DEE7D4F831
:100B6000BC340133C4F8BC34012075E72DE9F041F1
:100B700005460F4600F58054012639462846FFF702
:100B80004FFF10B184F87B64F7E7D4F8D034D4F881
:100B90007C040133C4F8D03420B10368BDE8F041CF
:100BA0001B691847BDE8F081F0B5436D1A6C12F46B
:100BB0007F0F2BD000F580541B6CC4F8D43441F265
:100BC0009005002347194FF0010C00EB43122A4413
:100BD0005E01117911F0020F15D0490713D4B959EC
:100BE000466DD6F8C8E00CFA01F111EA0E0F0AD0F2
:100BF000C6F8D010117941F004011171D4F8B42471
:100C00000132C4F8B4240133202BDED1F0BD000042
:100C100010B5254C254B226802B338B31A6D120665
:100C20000ED580221A6500F017FF50EA01020B462C
:100C300002D0013861F1000302462068FFF780FE10
:100C40001A4A136D1B032AD523684FF4002103F5BC
:100C500080531165012283F8812420E001221A6566
:100C600008221A654FF480621A6510BD196DC80715
:100C700002D4196D890705D5032119651046002195
:100C8000FFF774FF094B1A6D100702D41A6DD106D5
:100C900005D518221A6520680121FFF767FF206833
:100CA000BDE81040FFF780BF3837002000640040E7
:100CB00008B5302383F31188FFF776FF002383F311
:100CC000118808BD436DD3F8C40080F40010C0F350
:100CD0004050704708B5302383F3118800F58050E9
:100CE000C06E01F08FF8002383F3118843090CBF15
:100CF0000120002008BD000000F5805393F88124F6
:100D000062B1416D8A6922F001028A61D3F8C4247C
:100D10000132C3F8C424002283F881247047000004
:100D20002DE9F743302181F3118800F58351183103
:100D3000002541F2900E4FF0010800F5805C00EBB9
:100D400045147444267977071CD4F6061AD5D0F8D2
:100D500054908E69D9F8C87008FA06F63E4211D050
:100D60004F6801970F689742019F9F410AD2C9F8C7
:100D7000D060267946F004062671DCF8B0440134D0
:100D8000CCF8B0440135202D01F12001D7D100234A
:100D900083F3118803B0BDE8F0830000F8B51E4668
:100DA000002313700F4605461446FFF793FF80F0AB
:100DB000010038701EB12846FFF784FF2070F8BD8F
:100DC0002DE9F04F85B09946DDE90EA30D4602935B
:100DD0001378019391F800B08046164600F03CFE6F
:100DE0002B7804460F4613B93378002B41D02246A6
:100DF0003B464046FFF794FFFFF75AFFFFF77CFFA3
:100E00004B4632462946FFF7C9FF2B7833B1BBF179
:100E1000000F03D0012005B0BDE8F08F337813B187
:100E2000019B002BF6D108F580530393029B544598
:100E300077EB03031DD2039BD3F87C04C8B103688E
:100E4000AAEB04011B6898474B46324629464046A8
:100E5000FFF7A4FF2B7813B1BBF1000FDAD1337881
:100E600013B1019B002BD5D100F0F6FD04460F46CF
:100E7000DCE70020CFE7000008B50020FFF7C8FE40
:100E8000BDE8084005F094BF08B50120FFF7C0FE9B
:100E9000BDE8084005F08CBF036800211B681847B7
:100EA00008B5043007F0F2FD012008BD043007F05A
:100EB000E3BD00002DE9F84306460D4621B9043094
:100EC00007F0B8FD012424E003685B689847002818
:100ED000F8D100F0C1FD104B8846D3F800904FF4D4
:100EE0007A7107464D43D9F828000368C8219B68EA
:100EF0009847336830465B68984704460028E1D13C
:100F000000F0AAFDC01B61EB0801A84271F10003CB
:100F1000E9D32046BDE8F8833825002010B5044BFE
:100F2000044640F8043B07F043FD204610BD00BFD7
:100F300078410208034BC068DB68C31A5842584125
:100F4000704700BF186200200CB430B585B008AC03
:100F50000A46074954F8043B0D6800940146E86AC4
:100F60000394FBF75BFB05B0BDE8304002B070476F
:100F70003825002013B5054C0093246813460A4613
:100F80000146E06AFBF74AFB02B010BD382500209D
:100F90002DE9F341134601920E460A460021074609
:100FA0000846FFF7E7FF041E019B05DC4FF0FF3406
:100FB000204602B0BDE8F08104F10108012140465D
:100FC000019308F06FFB05460028EFD0019B3246E5
:100FD0004146FFF7CFFF3D60EAE700000EB403B5DE
:100FE00003AA52F8041B0192FFF7D2FF02B05DF88A
:100FF00004EB03B0704700000A460146014805F0C3
:1010000025BF00BF905F00200FB407B5054B04A9B2
:101010001B6851F8040B0191984703B05DF804EB8D
:1010200004B07047102300200F2070470F20704736
:101030000120704700207047704700000020704773
:1010400070470000704700007047000070470000C4
:1010500070470000084608F0DDB90000084608F0B7
:10106000A9BA000073B51E460C461546011D102294
:1010700001A8FBF7B5F932462946204608F01AFACE
:10108000044601A8FBF7C8F9204602B070BD000075
:1010900013B50D220C46011D01A8FBF7A1F920464E
:1010A00008F0CAF9044601A8FBF7B6F9204602B0D9
:1010B00010BD000008F0AAB9084608F0A3B9000066
:1010C000084608F097B9000010B5064B044640F8F2
:1010D000843B00F047FE04F1700000F043FE204620
:1010E00010BD00BF9C48020810B4BDF80440019434
:1010F0005DF8044B00F096BB10B4BDF804400194B9
:101100005DF8044B00F03CBB00F052BB00F080BB2C
:1011100030B51C4B03600021102591B004460171CD
:101120002A4600F54A7008F005FF04F54E70FFF7F7
:10113000F5FE284608F066F9134B0A94CDE90B3406
:10114000124BCDE90D34124B0F9310A9024611E951
:10115000030005AB83E80300DDE90C0103AB83E882
:101160000300DDE90A0101AB83E80300094B0093AA
:1011700004F10801234604F5597001F00FF92046E7
:1011800011B030BDA4420208F9100108091101088C
:101190000D110108E91001081B4A1C491C4B10B530
:1011A00002611C4A42611C4A826102641B4A426419
:1011B0001B4A82641B4AC161C2641B491B4A01620B
:1011C00002651B491B4A416242651B491B4A036079
:1011D000816282651A4B1B491B4A4360C162C2652A
:1011E0001A4B1B491B4A8360016300231A4902669C
:1011F0001A4AC360044641634266C36300F0FEFBC3
:10120000174B2360204610BD803F00204037002050
:10121000A4410208F83A002000390020683A002072
:10122000783A0020883A002048370020983A002079
:101230002C380020A83A0020A03E0020B83A002018
:10124000943E002058380020C83A0020983E0020E4
:1012500014230020D83A0020A4370020E83A0020C8
:101260000442020808B5302383F31188074B1B683A
:101270009A68996B8A4201D0824200D29860986342
:1012800007F034FD002383F3118808BDA037002048
:101290007FB51422002101A81C46334E334D08F0BF
:1012A00049FE69464FF461433148009307F04AF91B
:1012B000304BF2681A60B4202C6007F06DFE03F02A
:1012C000B7FF08F021FB2C4B1C684FF4E131206C78
:1012D000FBF732F9206903681B689847A06A036826
:1012E0001B6898470A20FFF7BDFF08F03BFC40B1A0
:1012F0002248132108F046FC20494C22881808F0A7
:101300000BFE1F4B286801229A7303681B689847DD
:101310001C4B1B6813B11B6ADB0701D508F0ECFB03
:10132000E06A03685B68984738B1FEF731FE4FF416
:1013300097724FF40061FEF717FE114802F0C2F9F0
:10134000A06A0F4C03681B6B9847F3680E4ADA617A
:10135000B42007F021FE286803685B6898472046A0
:1013600002F0B0F9F7E700BF18620020C037002094
:10137000905F0020A0370020382500205C38002036
:10138000A03E0020983F002090410208014B1868C1
:10139000704700BFA037002000487047C4370020C6
:1013A00000487047C437002038B53A4D3A4C002108
:1013B000284602F05BFD39492246284608F082FDA6
:1013C0003748384D00F0E4FF374800F0E1FF374878
:1013D00000F0DEFF364800F0DBFF364800F0D8FFB3
:1013E000354800F0D5FF354800F0D2FF344800F012
:1013F000CFFF344800F0CCFF334B344A1A60344BF3
:10140000344A1A60344800F029FF2846FFF780FE6E
:10141000224632492846324D08F054FD314804F046
:10142000ABFA2846304B40F8043B2422002108F058
:1014300081FD05F13400FFF771FD4FF0FF332B49BB
:10144000EB642246284608F03DFD294B29482A4DE9
:1014500030221A714FF47A72DA804FF4FA621A81EC
:10146000264A1A6002F0D2F8254B002283F89C200D
:101470002846244A1A60244B40F8043BFFF74EFDEF
:1014800022462846214908F01DFDBDE83840204885
:10149000FFF782BE00390020843F0020C9100108F8
:1014A000683A0020F83A0020783A0020883A002074
:1014B000983A0020A83A0020B83A0020C83A002004
:1014C000D83A0020E83A0020943E0020B0410208BB
:1014D000983E002020460208803F00204910010865
:1014E0004837002040370020644502084D100108AD
:1014F0002C380020A03E0020A4370020E44302083E
:1015000058380020C04A0208E04102085110010882
:10151000C437002070470000037933B108304FF41E
:101520004873086013600120704718467047000038
:1015300000F5597001F04AB910B50446007948B178
:1015400000F088FAD4F86033C01AB0F5FA6F2CBFF7
:101550000020012010BD000008B5FEF719FDA222F1
:101560004FF40031FEF700FD002008BDF8B5064637
:10157000EAB1CC0801390A44C2F3CC050127A542DF
:1015800015D3632C0ED8630906EB830304F01F0206
:1015900007FA02F1D3F828230A43C3F828230134B9
:1015A000A4B2ECE7FFF7D8FF0028ECD1F7E7F8BDCD
:1015B000102110B511220446A0F858130548FFF772
:1015C00023FD04F5597001F049F910B9024800F003
:1015D00017FA10BD084202082E42020810B5017920
:1015E000044671B9102200F54A7008F0A3FC2046A9
:1015F000FFF7DEFF022121710248BDE81040FFF72E
:1016000003BD10BD4C420208B3F5487FF8B507464C
:101610000E4614461D460DD8C3F548739A4209D8A4
:101620000834FFF7DBFF2A4639193046BDE8F84099
:1016300008F072BCF8BD0000B3F5487F2DE9F34116
:1016400005460E4690461C4622D8C3F5487399427B
:101650001ED801F10807074422463946404608F0E3
:101660004BFCA8B12846FFF7B9FFF12205F54E71F2
:1016700001A8FAF7B5FE22464146384608F04CFC70
:101680002846A2B23146FFF771FF01A8FAF7C4FE5F
:1016900002B0BDE8F081000037B505460C4601A850
:1016A0000121FAF783FEE10089B2082205F559709D
:1016B00000F0CEFF044601A8FAF784FE204603B0EE
:1016C00030BD00002DE9F74F0379044603B300F560
:1016D0004A7300F54E7853F8042B32B94345FAD1DA
:1016E00000F0B8F9C4F8600312E000250123C5F347
:1016F0004A1604EB860605F01F07D6F8282303FADE
:1017000007F717421FFA85FA05D10135642DEED18E
:1017100003B0BDE8F08FED0008354FF48872414604
:1017200001A8FAF75DFE04EB050B6359C4F85033CA
:10173000DBF80430C4F8543301A8FAF76DFE2379BE
:10174000022B04F55479E3D151462046FFF7A4FF5C
:101750000028DDD04FF49C72414601A8FAF740FE04
:1017600008225946484608F0C7FB28B9D6F828335E
:1017700023EA0703C6F8283301A8FAF74DFEC7E7A6
:1017800038B51C46094BB0F858031B685B6B15460F
:101790001A680144126818469047BDF81020411994
:1017A000204608F0B9FB012038BD00BF38250020D5
:1017B0002DE9F743DFF8549006460F4605244FF411
:1017C0007A7101A8FAF7F2FDD9F80080B6F858133B
:1017D000D8F8340003683944DB689847054630B1CF
:1017E00001A8FAF7EFFD284603B0BDE8F083D8F86A
:1017F0002800036801215B689847013C01A8FAF7BB
:10180000E1FD14F0FF04DAD1EDE700BF3825002038
:10181000034B1B68DB6A93F89C0080F00100704763
:10182000382500202DE9F04F2DED028B08EE103AFF
:101830002A4BD3F800900446D9F834000F460368C9
:10184000B4F858131B6885B039449046BDF840B0D1
:101850009847052500EB080A012103A8FAF7A6FD21
:10186000D9F83400036818EE102A1E6951465B4609
:10187000B047064640B103A8FAF7A4FD304605B0CC
:10188000BDEC028BBDE8F08FD9F828000368012178
:101890005B689847013D03A8FAF794FD15F0FF0532
:1018A000DAD12046FFF7B4FF0028E7D000F0D2F8E5
:1018B000D4F85C3341F28832C31A9342DED9C4F8BB
:1018C0005C0304F5597000F0B7FF5B460090424698
:1018D00039460348FFF798FBD0E700BF38250020C2
:1018E0006C42020870B51D46164B1B6813B11B6A8B
:1018F000DB0725D5144B1E68F46A94F84630C3B94B
:10190000124BA4F84400DB6884F84610E26163B12E
:101910009A6884F84720D96939B194F9483023B9D5
:10192000042204F1480000F099F8094B5B68C4E90F
:101930000835F06A1321BDE87040043008F01CB986
:1019400070BD00BF983F002038250020186200209D
:1019500000ED00E000B59BB0EFF309816822684616
:1019600008F0DAFAEFF30581074BC9B29A6BD86A2F
:10197000986A986A986A986A986A9B6A059B7B201D
:10198000FFF7B0FFFEE700BF00ED00E000B59BB041
:10199000EFF309816822684608F0BEFAEFF305818B
:1019A000064BC9B29A6B986A986A986A986A986A5C
:1019B0009B6A059BBF20FFF795FFFEE700ED00E067
:1019C00000B59BB0EFF309816822684608F0A4FADD
:1019D000EFF30581064BC9B25A6B986A986A986A08
:1019E000986A9B6A059BE320FFF77CFFFEE700BF38
:1019F00000ED00E0FEE70000FEE700007047000099
:101A00000FB483B504AC0F4F54F8048B0E4EFEF7A1
:101A1000BFFA4FF4A5722021FEF7A6FA42F2107524
:101A2000214640460194FFF7E7FA3846FFF7ECFA03
:101A30003368986A036829465B6898474FF4FA75DB
:101A4000EEE700BF75E30108382500204FF0804322
:101A5000586A704707F0BEBE07F0A0BEF8B50D4645
:101A6000074611462846164608F03AFF86420446C5
:101A70008CBF421C02462946384608F04DFA2046E3
:101A8000F8BD000070B5467B05460EBB4468836810
:101A900004EB8404A40804F50074E21A914288BFA0
:101AA000CC180C4B29681B68D86A0368621C1B6D34
:101AB000984718B901232B73304670BDAB68C5E950
:101AC0000004E21A0021184408F034FA0126F3E772
:101AD0000026F1E7382500200EB470B5017B85B0F3
:101AE000044619BBD0E901239A421BD0134B1E6850
:101AF0000AADD4E9012120680095521A099B03958B
:101B00000144F06AFAF78AFD00280FDBD4E90123CB
:101B1000D21A82420FD8411C2046FFF7B3FF00289B
:101B2000E7D103E0FFF7AEFF0028DFD105B0BDE845
:101B3000704003B070471844A060F7E738250020D4
:101B40001022002108F0F6B90148FFF7F9BF00BFE5
:101B5000883F002070B50446406A0D46164620B105
:101B6000FAF7DCFA0023A383A37705EB4500FAF725
:101B7000CFFA606228B100232577E67784F8203019
:101B8000012070BD81727047F0B4446A0E46114660
:101B90007CB1457F224600275FFA87FC65450DD959
:101BA00092F801C08C4506D192F800C0B44502D12C
:101BB0009370F0BC704701370332EDE7027FAA4211
:101BC00004D182680A48F0BCFFF71EBA05EB450550
:101BD0006655457F05EB450525446970427F02EB5C
:101BE00042021444A370437F01334377E1E700BF0F
:101BF000C042020813460A460021FFF7C5BF000095
:101C0000F0B587B004460E468DF80F208DF81410FD
:101C10008DF815200BB1FFF7EDFF2268002300932C
:101C2000156905A902222046A847A76905463FB1C4
:101C300030B10123606900930DF10F023146B847BE
:101C4000284607B0F0BD00002DE9FF419846037912
:101C50000B438DF80F300368CDF800801D691746DF
:101C600013460E4601220DF10F010446A847054612
:101C7000606908B9A3693BB135B100230093A46939
:101C800043463A463146A047284604B0BDE8F081B5
:101C9000F7B5437F04460BB901201CE090F82030D3
:101CA000C27F0133DBB29A4280F82030F4D800239F
:101CB000857F476A80F82030036905EB45057E196A
:101CC0005BB1795DC068984738B97B5BA4F8213077
:101CD000B37884F8233003B0F0BD717801230DF19F
:101CE00006022046FFF7B0FF68B1B2789DF80630D3
:101CF0009A4208D1A37F627F0133B3FBF2F102FB6A
:101D00001133A377C8E70DF107027178012320464C
:101D1000FFF79AFFB27818B19DF807309A42E9D0E0
:101D2000002371782046FFF76BFF7B5BA4F821301E
:101D30009DF8063084F823300020CCE7017170470D
:101D400070B500260446C0E9026601200D4607F082
:101D5000A9FCB04208BF3546206065602674204665
:101D600070BD000010B5037C044613B9006807F08D
:101D70009DFC204610BD000070B5057C04460E4653
:101D8000DDB9BFF35B8FC560BFF35B8FBFF35B8FC4
:101D90008560BFF35B8F43688B420CD0006807F00F
:101DA00085FC3146012007F07DFC206010B965609C
:101DB000284670BD66600125FAE70025F8E70000B7
:101DC00038B505460C4644B121462846FFF7D4FFF6
:101DD00020B904EB4404A408F5E7204638BD000010
:101DE0000023BFF35B8FC360BFF35B8FBFF35B8FD9
:101DF0008360BFF35B8F7047BFF35B8F0068BFF3F7
:101E00005B8F704770B505460C30FFF7F5FF05F1A5
:101E1000080604463046FFF7EFFFA04206D93046D9
:101E20006D68FFF7E9FF2544281A70BD3046FFF7BB
:101E3000E3FF201AF9E7000070B50546406898B145
:101E400005F10800FFF7D8FF05F10C0604463046FF
:101E5000FFF7D2FF8442304694BF6D680025FFF73C
:101E6000CBFF013C2C44201A70BD000038B50C4655
:101E70000546FFF7C7FFA04210D305F10800FFF7A2
:101E8000BBFF04446868B4FBF0F100FB1144BFF3EE
:101E90005B8F0120AC60BFF35B8F38BD0020FCE797
:101EA0002DE9F041144607460D46FFF7C5FF844271
:101EB00028BF0446D4B1B84658F80C6B4046FFF72B
:101EC0009BFF3044286040467E68FFF795FF331A39
:101ED0009C4203D86C600120BDE8F0816B60A41BBC
:101EE0003B68AB602044E8600220F5E72046F3E75A
:101EF00038B50C460546FFF79FFFA04210D305F109
:101F00000C00FFF779FF04446868B4FBF0F100FBB4
:101F10001144BFF35B8F0120EC60BFF35B8F38BDD2
:101F20000020FCE72DE9FF41884669460746FFF798
:101F3000B7FF6C4606B204EBC6060025B44209D0D2
:101F40006268206808EB050107F0E6FF6368083463
:101F50001D44F3E729463846FFF7CAFF284604B078
:101F6000BDE8F081F8B505460C300F46FFF744FF99
:101F700005F1080604463046FFF73EFFA042304612
:101F800088BF6C68FFF738FF201A386020B13046F0
:101F90002C68FFF731FF2044F8BD000073B51446EC
:101FA00006460D46FFF72EFF844228BF04460190E7
:101FB000DCB101A93046FFF7D5FF019B33B9326888
:101FC000C5E90233C5E9002401200CE09C4238BF7A
:101FD00001942860019868608442F5D93368AB6049
:101FE000241AEC60022002B070BD2046FBE700001E
:101FF0002DE9FF410F466946FFF7D0FF6C4600B25E
:1020000004EBC0050026AC4209D0D4F8048054F893
:10201000081BB819424607F07FFF4644F3E73046F5
:1020200004B0BDE8F081000038B50546FFF7E0FFD9
:10203000044601462846FFF719FF204638BD000038
:102040002DE9F74F10EE103A009210EE102A0729F2
:1020500028BF0721C3F316044FEAD37812024FEAD0
:10206000D35307460E4603F0FE0340F1A68001332A
:10207000DBB2FF2B32D044F40004DA0859495A4845
:1020800011F90290594951F8225003F00703A4FBBB
:102090000554C3F10F021133B2F1200104FA03F326
:1020A00025FA02F558BF44FA01F145EA03054FF05D
:1020B000000B58BF0D43144145F6F321CDF804B091
:1020C0004FF0300A2A1A64EB0103002B0DDB0AF1F2
:1020D000010A4FFA8AFA15461C46F3E714B948F08C
:1020E0000408C8E748F00808C5E700230A22F7F704
:1020F0009DFD019BD3B9BAF1300F06D109F1FF392B
:102100004FFA89F92A462346E5E7009BF3B1009A86
:1021100009F101035BB2013A012BACBFD2180132C5
:1021200002F0FF039E42009328BF1E460BF10103FD
:10213000BAF1390FDAB257FA83FC0ADC012396426E
:1021400007F802A0019319D99346B9E70136F6B210
:10215000ECE7A2EB0B0039213844CDF800C007F0C2
:10216000E9FEDDF800C0634630201946013B0A78DD
:10217000013252B23A2A13D00A700CE00A22A0FBB4
:102180000206400840EAC670281A02FB016164EBAF
:102190006104002CE7DA87F800800FFA89F01DE06F
:1021A000BB4208D1312309F101090B704FFA89F9BB
:1021B00048F01008EFE75870D7E7002B7FF45BAFCB
:1021C000002C7FF45AAF384648F00208721C00F821
:1021D000018BD2B2302107F0ADFE204603B0BDE83E
:1021E000F08F00BF7C43020800407A10FC420208D6
:1021F0009FED010A704700BF0000000000207047FB
:10220000002070470368DB681847000090ED010A62
:1022100070470000D0ED017AB1EE040A67EE807AD3
:102220009FED020A27EE800A704700BF0000803A47
:102230000120704770470000B1EE040A70470000AB
:1022400008B50820F9F75EFF18B1024B0360024B96
:10225000436008BDA44302087B148E3F014B03601A
:10226000704700BFC4430208704700007047000079
:102270000020704770470000704700007047000062
:1022800003689B6B184700000368DB6B184700006E
:102290007047000000207047704700000020704722
:1022A0009FED010A704700BF0000C8420020704740
:1022B00000207047002070477047000000207047E2
:1022C00000207047002070477047000070470000F2
:1022D0007047000000230B6001207047002070470A
:1022E00000207047704700007047000070470000F2
:1022F00070470000704700007047000000207047E2
:1023000070470000002070477047000070470000D1
:102310000020704700207047002070477047000081
:1023200000207047704700007047000070470000B1
:10233000704700007047000070470000322070476F
:10234000704700000F299CBF00EB4100428170479D
:102350000F299ABF00EB410040894FF4617070472C
:10236000102A0B4628BF102200F10A01520018461D
:1023700007F0D2BD70470000704700000020704792
:1023800000207047012070471046704700207047BA
:10239000014B0360704700BFC444020882B010B50F
:1023A000044602A8C4E9001240F8043F03C804F13F
:1023B000080383E80300DDE9050104F1100383E865
:1023C0000300DDE9070104F1180383E80300DDE9F8
:1023D000090104F1200383E803002046BDE8104012
:1023E00002B0704710B50A4492B2914208D0046816
:1023F0004B1C615C9BB209B1002010BD1946F4E78B
:102400000120FAE703680F3332D18368591C0FD1DA
:10241000036901332CD14268164B9A4228D1C36814
:10242000013325D1436901330CBF012004207047DB
:102430000E331DD103695A1C0BD143680D4A9342D8
:1024400016D1C2689A4213D14369013310D10220D8
:1024500070470D330CD14268064B9A4208D1C368CD
:10246000934205D14069984214BF0420032070476D
:102470000420704762B5861510B4BDF8044001947D
:10248000D0E90004A4465DF8044B60472DE9F04311
:10249000054685B088464FF0180900F1100602275E
:1024A0006B68023B4B4546D9009703AB4A46414611
:1024B0003046FFF7E1FF40B19DF80C3003F0030315
:1024C000012B09D0032B02D09BB1002001E0C5F8FD
:1024D0002C9005B0BDE8F0839DF80D305B09013309
:1024E00003EB430409EB44040234073424F00709E6
:1024F000D6E7BDF80C309DF80D20C3F38A035209CE
:1025000003EB430301325B0002EB42029BB2540037
:1025100003EB4202B2F5487FD7DC2A6800941344EB
:10252000414609F102023046FFF7A6FF0028CCD051
:1025300002344C44D9E7C5F82C900120C9E70000CB
:1025400010B4BDF804400194D0E90004A4465DF83D
:10255000044B60472DE9F047026B8AB004466AB924
:1025600090F82850039285F001051827009704ABD6
:1025700029461030FFF780FF039A08B900203FE09A
:10258000059E214B9E4203D0012384F83430F5E7A9
:1025900004A80392FFF736FF0128039AF4D16FF0E5
:1025A0000C0304F108086FF00E0A6FF00D09089390
:1025B00094F82810009704AB404607960996CDF88A
:1025C00010A0CDF81890FFF7BBFF0028D6D04FF031
:1025D000FF3309930893039A009704AB29464046BA
:1025E00005960796CDF810A0CDF81890FFF7A8FF34
:1025F0000028C3D040F22E43C4E90B7384F828505E
:102600000AB0BDE8F08700BF62B5861570B5044614
:1026100088B0D0E906030D4616469847A0B19EB192
:102620000A4B03934FF0FF336FF00E0205930793AD
:1026300004930693182302920093002202AB2946CA
:1026400004F10800FFF77CFF08B070BD62B5861585
:102650002DE9F04390F8343085B004460E46174615
:10266000002B3FD14FF001094FF00608002F5CD03E
:102670006368E26A9A1A236B08339A4236D3B6FB30
:10268000F8F59DF8083069F301038DF80830BDF8BE
:102690000820C5F30A0363F38C02ADF80820C2F3E7
:1026A00007226FF347128DF8092003EB43032268DA
:1026B00002EB430152F81330CDF80A308B88ADF8A5
:1026C0000E309DF80830E26A94F828106FF3010389
:1026D0008DF808300823009304F108006B44FFF7DD
:1026E0002FFF98B9002005B0BDE8F0832046FFF722
:1026F00031FF0028C3D1D4E9080398470028F1D05E
:10270000204600F04DF80028B9D1EBE7E36A083322
:10271000E36208FB1563C3F10603DBB2BB42E2DCF4
:102720001E44FF1AB6B2BFB2A0E70120DBE70000EB
:1027300037B505464FF44874062C2246C4F5487157
:10274000A8BF062289B292B22846CDE90012FFF74F
:1027500049FEDDE9001220B1063C231DECD1012029
:1027600004E02846FFF774FF0028F5D103B030BD20
:10277000002310B580F8343003630446FFF7D8FF18
:1027800060B194F82810012251402046FFF73EFF27
:1027900020B12046BDE81040FFF7DCBE002010BD90
:1027A00038B590F83550044645B1FDF7F1FB91225C
:1027B0004FF40011FDF7D8FB002038BD012380F84D
:1027C0003530FFF7D5FF84F83550F6E770B50025B2
:1027D000182688B080F8345080F82850C6622A46FF
:1027E00029460446FFF712FF10B9002008B070BD5B
:1027F00094F82820013A18BF012201212046FFF752
:1028000005FF0028F1D00B4B03936FF00E020593E8
:1028100002924FF0FF336FF00D020793049206937C
:1028200094F82810009602AB2A4604F10800FFF73E
:1028300087FEDBE762B5861510B50446D0E90803CC
:10284000984740B12046FFF7C1FF20B12046BDE8C0
:102850001040FFF76DBF002010BD00002DE9F04FC4
:10286000804693B005464FF4487258F8100BDFF8D5
:1028700018B1002107F05EFB06AF0026B9464FF005
:10288000180ACDF800A03B46002231464046FFF72B
:10289000F3FD044630B90024204613B0BDE8F08FA4
:1028A0000126EEE77B6803933846FFF7ABFD01385E
:1028B000C0B2022802D8039B5B4504D02846FFF72C
:1028C00085FF0446E8E71837002EE9D04846FFF7B1
:1028D00099FD07468DF814000CA8FFF793FD874279
:1028E00080468DF8150003D1012FE7D1002608E0BE
:1028F000032FFBD0032804D0022FF7D0831E5E42A3
:102900005E4112AB334413F8349CA9F10203012B4E
:1029100005D831462846FFF7B9FD0028CED086F00D
:10292000010112AB0B4413F8343C023B012B04D8D9
:102930002846FFF7ABFD0028C0D00023B9F1030FF4
:1029400085F834302B6315D0032F06D101220021E6
:102950002846FFF75BFE00289DD0B8F1030F06D193
:10296000012211462846FFF751FE002893D000238C
:102970002B6391E786F0010685F828602846FFF76B
:10298000D7FE0028E0D199E762B5861570470000B0
:1029900000207047B0F94C0070470000B0F94E00BD
:1029A00070470000012380F85430704780F85510BC
:1029B0007047000090F8543013B190F83000704721
:1029C0001846704737B590F8543004460D46ABB101
:1029D00090F83030122BA8BF122399420EDA00F182
:1029E0003401612201A804EB4504F9F7F9FC01A8C0
:1029F000A488F9F711FD204603B030BD0024FAE7A2
:102A000037B590F854500446A5B100F134014A227C
:102A100001A8F9F7E5FCD4E90A51226D0023994297
:102A200008BF9542C4E90A2301A814BF0125002567
:102A3000F9F7F2FC284603B030BD000073B590F8FA
:102A4000544005460E468CB1122A28BF122200F1CE
:102A50003401144601A87122F9F7C2FC6200291D55
:102A6000304607F059FA01A8F9F7D6FC204602B023
:102A700070BD00007047000013B50468009224691F
:102A80000B46A04702B010BD704700000020704701
:102A90000020704713B56C4684E8060000F114036B
:102AA00094E8030083E8050002B010BD00207047E1
:102AB00013B56C4684E8060000F10C0394E80300AB
:102AC00083E8050002B010BD0023C0E9033370475E
:102AD00082B002AB03E9060002B070477047000005
:102AE00000207047704700000020704700207047AA
:102AF00013B50346684680E80600DC6A03C818344C
:102B000084E80500D860196102B010BDC26A0023D4
:102B1000C2E90633C0E903337047000019B1012947
:102B200004D001207047C36B4363FAE7836BFBE774
:102B3000806A043070470000704700001FB502AC87
:102B400084E80C00009094E80C00806A03F0B0F870
:102B500004B010BD806A03F003B9000037B5074C1C
:102B60006D46206885E80C00F7F7DEFA20B995E895
:102B70000300203484E8030003B030BD9C3F0020F4
:102B800010B50446006C06F091FD606A034B2360AB
:102B900008B1F9F7C3FA204610BD00BFA4450208EA
:102BA00010B50446FFF7ECFF2046F9F7B3FA2046CC
:102BB00010BD000070B5044688B00D46B52103F085
:102BC00061F884F8405004F15C0005F0F1FE134B0D
:102BD0000494CDE905341420114B0793F9F792FAC8
:102BE000054698B194F840300E4E0C2202FB036665
:102BF00008AA12E9030001AB83E80300059B0093D8
:102C0000B279049B7179284602F020FBE561064801
:102C100006F094FEA067204608B070BD392B01086D
:102C20001D3001080C460208050000482DE9FF4749
:102C30001E46036890F844909B6CCDE90221012167
:102C400004469847054680B11FFA86F8A06ACDF879
:102C5000008002AB424603A903F098F8054640B94C
:102C6000236849469B6C20469847284604B0BDE837
:102C7000F087302383F31188DFF8BCA02D4FDAF8FA
:102C800000300399DA6A136B01331363E26A127935
:102C90000C235A43BA58002936D103211170E26A35
:102CA000127953433146029AF85804F0DFFEE36A82
:102CB0001B790C22534306F27121F8584901083060
:102CC00006F08EF9002383F31188013015D1DAF86C
:102CD0000030986A03685B69984730B9FDF758F986
:102CE000D6224FF48041FDF73FF9E36A1B790C22AD
:102CF00053430025F85805F097FCDDE90221A06A4E
:102D0000434603F069F8ABE7029803211170E26AC9
:102D100038B9127953433146039AF85804F08AFEC1
:102D2000C5E7107958433146DDE90232385804F0DE
:102D300067FEBCE70C460208382500202DE9F84F55
:102D40008246806A00AF0430BE6A0D46144698463B
:102D5000FEF7F0F820B900252846BD46BDE8F88FFB
:102D6000B44201D1454503D015B1B8F1000F0AD1E5
:102D70002946002E14BF3346234642465046FFF7ED
:102D800055FF0546E8E704EB060B0BF1070222F0BE
:102D90000702ADEB020DE94624B1224629466846FA
:102DA00007F0BAF82EB13246002109EB040007F013
:102DB000C1F85B464A4649465046FFF737FF05468D
:102DC0000028C8D0002EC7D0324609EB0401404687
:102DD00007F0A2F8C0E70000F0B583B00546806AAE
:102DE00000AF0430796016461C46FEF7A3F87968F8
:102DF00020B9002528460C37BD46F0BDE31D23F061
:102E00000703ADEB030D2246684607F085F8284618
:102E100023466A466946FFF709FF05460028E8D0C1
:102E200022466946304607F077F8E3E737B50446AF
:102E3000806A019204300D46FEF77CF840B1019B98
:102E40002A462946204603B0BDE83040FFF7EEBED3
:102E500003B030BD0138C3B2052B96BF084B094BF8
:102E600053F820304FF0000098BF5B088B4204D924
:102E7000072802D05B080130F8E7C000704700BFA8
:102E8000F445020800688909C36A1A79034B0C20CB
:102E900000FB02331879FFF7DDBF00BF0C460208C4
:102EA0002DE9F3410023C0E90333C0E90533037181
:102EB000037A1546022262F30203037291F840700E
:102EC000194B1A4A03600C2303FB0722037A127979
:102ED00095F8058080F8098062F3C703C0E90A15F8
:102EE000037229690446FFF7CFFF6969A0630646AC
:102EF0002046FFF7C9FF2A68E0633B460C4966633A
:102F0000CDF8008004F14000FEF768F8E36AD3E9E9
:102F10000612C4E90312D3E908232046C4E90523B5
:102F200002B0BDE8F08100BF384602080C46020836
:102F30008C45020870B5164E05463068F7F7F4F870
:102F4000E0B10025284670BD7C20F9F7DBF8044687
:102F50000028F6D03179FFF72DFE6B6823603379B6
:102F600084F840306C604820F9F7CCF8054600281A
:102F7000E8D0074A2146FFF793FFE3E76C6833790F
:102F8000002CE1D094F840209A42ECD02468F7E776
:102F90009C3F002010B50446084601212022084429
:102FA000FAF758F8E36AC0B25969B1FBF0F120466C
:102FB000FFF76AFFE06310BD38B590F8743004463F
:102FC000CBB1036F90F84050012B4FF090434FF07E
:102FD000200294BF5A831A83202101224FF090408F
:102FE00004F026FB0C235D43034B585905F000FB0E
:102FF000002384F8743038BD0C46020838B500F15F
:103000005C050446284605F015FD2046FFF7D4FF71
:103010002846BDE8384005F039BD0000FFF7EEBF97
:1030200010B590F87430044693B990F840300C22F3
:103030005343084A00F14401D05805F0CBFAA26F7F
:1030400020214FF0904004F0F3FA012384F874300B
:1030500010BD00BF0C4602082DE9F8430446806A03
:1030600004300E461746FDF765FF054618B194F883
:1030700044501EB115B32846BDE8F883002DFAD0A0
:10308000314A5FB9E36A1B790C214B43D3585B6823
:10309000D3E90210012383409BB20B83E36A1B79BF
:1030A0000C214B43D05805F0D3FA002384F8443068
:1030B000A36A0121D86902F01BF9DCE7A36ADFF8F3
:1030C0008880D86902F034FAE36A1B794FF00C0962
:1030D00009FB03F358F8030005F0B6FAD4E90A2314
:1030E0009B6823F00F03D364D4E90A239B6803F0A1
:1030F0000F031365A36A9D64D4E90A13606BDA6851
:103100000243A1F85420A36AA3F85650D4E90A3226
:10311000D2681A67A06AFFF74FFFA06AFFF780FF27
:1031200067B9E36A1B7909FB03F358F803305B685E
:10313000D3E9022101238B409BB25383012384F8FE
:103140004430354697E700BF0C4602080022FFF7DF
:1031500083BF0000084B094A09491A604FF4807286
:103160009A800022C3E902120649C3E90622C3E994
:103170000411C3E9082270479C3F0020ACE5010818
:103180000E08004840420F002DE9F8430446836AC8
:1031900094F8449001F271280D464FEA4818181D22
:1031A000B9F1000F3BD15B6849461B689847012283
:1031B00011462046FFF750FF302383F31188E36A5E
:1031C0002C4E1B790C277B430322F3581A70E36AB9
:1031D0001B797B432946F05804F0F6FBE36A1B7920
:1031E0007B434146F058083005F0FAFE054689F366
:1031F0001188421C05D1E36A1B795F43F05905F041
:1032000013FA012200212046FFF726FFA06A0430AE
:10321000FDF746FE681C18BF0120BDE8F883FDF7E6
:1032200089FE0028F9D0302383F31188E36A114E18
:103230001B790C277B430322F3581A70E36A1B792E
:103240007B432946F05804F0BFFBE36A1B797B43BC
:103250004146F058083005F0C3FE0023054683F3CD
:103260001188431CD6D1E36A1B795F43F05905F0FE
:10327000DBF9CFE70C460208407B704701617047DD
:1032800010B5074B074ADB680446DA61A37B33B904
:1032900023684FF47A719B6820469847F6E710BD83
:1032A000186200209446020838B50D4B0D4ADB68C1
:1032B0000446DA612368A27B9B6862B10A4D2368E9
:1032C00020469B684FF47A7198472B6858690368C9
:1032D0001B699847F3E742F2107120469847E9E7E7
:1032E00018620020434202083825002013B5044626
:1032F0000121C83005F006FD04F1D400012105F0DC
:1033000001FD154B0094B5224FF4FE61134805F002
:10331000CDFD134BC4F8B0000094B5224FF47C717E
:10332000104805F0C3FD104BC4F8B40000943A22D5
:103330004FF41F610D4805F0B9FD0D4BC4F8BC00FA
:1033400000943B224FF4BE610A4805F0AFFDC4F87B
:10335000C00002B010BD00BFD9370108985300204B
:1033600081320108B84900206D380108C83F0020AB
:10337000A9320108A84D002070B5437D04460D46D2
:103380004BB903681B6C984728B1B620FDF76AFF5C
:1033900040F20113A3822368294620469B68BDE8BA
:1033A0007040184708B5FDF7F1FF034BDB681B1AA7
:1033B0005842584108BD00BF186200202DE9F0476F
:1033C00004460D46FEF748FBDFF8689006460F46B8
:1033D000FEF742FB801B4FF0000361EB07014FF447
:1033E0007A72F6F773FCA84271F1000320D22368C9
:1033F0004FF47A719B6820469847A388AB42E7D880
:10340000236820461B6C98470028E1D0D9F800803B
:10341000D8F82C30FC2293F94CA083F84C20236878
:103420002046DB6C9847D8F82C3083F84CA0CFE7C7
:10343000BDE8F0873825002008B5302282F31188D6
:103440008368002B01DC05F083FC05F04FFC0023B2
:1034500083F3118808BD0000F7B5044600F1C806E3
:103460006D46304685E8060005F068FC94F8643047
:10347000DDE90007224604EBC30C62450DD0516A1A
:10348000814208D1916AB94205D1304603B0BDE806
:10349000F040FFF7D1BF0832EFE7072B0AD895E8D5
:1034A000030004EBC3022432013382E8030084F8F2
:1034B0006430EAE7034B04491B68986903681B689A
:1034C0009847E2E7382500209C46020808B50E4BD5
:1034D0001B68586A0368DB6C0C4698470B4B0C481A
:1034E000002C08BF184606F001FA72B6BFF34F8FE2
:1034F0000849094BCA6802F4E0621343CB60BFF38A
:103500004F8F00BFFDE700BF38250020020007B045
:10351000010007B000ED00E00400FA0510B5836972
:1035200004461BB9BDE8104006F058B8FEF792FA01
:10353000A369C01AE3699842F4D8012010BD0000C5
:1035400008B5437B13B10348FEF75AFA01234373CE
:1035500008BD00BFB446020805F046BC084605F0A9
:103560004DBC000029B10A2938BF0A21084605F0E0
:103570002BBD704710B503681B6C0446984740B1DB
:10358000637D33B100236375B420BDE81040FDF7BF
:1035900069BE10BDF7B5044600F1D4066D4630464D
:1035A00085E8060005F0CAFB94F8A830DDE90007BD
:1035B000224604EBC30C62450DD0916E814208D1C6
:1035C000D16EB94205D1304603B0BDE8F040FFF7F7
:1035D00033BF0832EFE7072B0BD895E8030003F160
:1035E0000D0204EBC202013382E8030084F8A83024
:1035F000E9E7044B04491B68986903681B6898470E
:10360000E1E700BF38250020F446020810B5084B5A
:103610000446402240F8243B002106F08BFC402267
:10362000002104F1680006F085FC204610BD00BFB3
:103630002047020810B50B4C1046002314F8132045
:103640008A4209D104EB4303FF225B78022118442C
:10365000F9F700FDC0B210BD01330E2BEED13A20B8
:10366000F9E700BF74470208F0B585B0074602AD20
:10367000082085E806001E4606F006F80446D8B184
:1036800095E803009DF9302084E803009DF82C1094
:103690003846FFF7CFFF0A9D094B009405F2F71556
:1036A0000246314625F0070006F01EF8054628B907
:1036B000204605F0FBFF284605B0F0BD0120FBE7E2
:1036C000C138010810B5044606F02AFAFEF7C2F91F
:1036D000C4F8AC0010BD000070B503681B6C044654
:1036E0000D46984738B12046FFF7ECFF4DB9236AE5
:1036F00013B90023A36170BD013B2362002BFAD1F3
:10370000F7E7FEF7A7F9A36943B1E269C11A8A4254
:1037100004D913441B1A9D4238BF1D46236AC4E9CD
:10372000060501332362236820469B69BDE870408B
:103730001847000010B5114806F046F93F2807D891
:10374000FCF726FC4FF6FF724FF40001FCF70CFC6F
:1037500005F0D2F9044678B1006A06F035F93F2841
:1037600006D8FCF715FC228F4FF40001FCF7FCFB98
:10377000204605F0D1F9EDE710BD00BF00010020A3
:10378000D0E9000318470000F8B590F8653004460A
:1037900003F0FF05F3B9012300F1C80680F8653096
:1037A000304605F0CBFA304694F86470FFF744FEDB
:1037B00004F12406AF4207DD736813B13046FFF70A
:1037C000DFFF01350836F5E7236903B19847002389
:1037D00084F86530F8BD000010B5104B104ADB6866
:1037E0000446DA612368A27B9B6822B94FF47A71A0
:1037F00020469847F6E723684FF47A719B68204685
:1038000098472046FFF7C0FF236820465B6998472A
:103810000028F0D02046FFF755FFECE718620020A3
:103820000C470208F8B590F8A930044603F0FF05EC
:10383000DBB9012300F1D40680F8A930304605F049
:103840007DFA304694F8A870FFF7F6FD04F168069B
:10385000AF4207DD736813B13046FFF791FF0135C2
:103860000836F5E7002384F8A930F8BD70B5124B8F
:10387000124ADB680446DA612368A27B9B6822B99E
:103880004FF47A7120469847F6E7002623684FF4F4
:103890007A719B68204698472046FFF7C3FFFEF7E2
:1038A000D9F8831BB3F57A7F0546EFD92046FFF799
:1038B00041FF2E46EAE700BF1862002014470208C5
:1038C00010B50446FFF75CFF2046BDE8104005F048
:1038D000EDBE000090F809017047000003695B79B4
:1038E00023B9406B0A23B0FBF3F070474FF4483024
:1038F00070470000406B7047037D03B1437D18465D
:103900007047000090F8ED20034602F0FF0012B16E
:1039100093F8EC00C0B27047002070470020704759
:10392000F8B590F80831476B1F330C4600EBC30124
:1039300050F833504E6877B103695B795BB903681F
:103940005B6998472044054BB3FBF7F35843281AAB
:10395000054666F1000628463146F8BD8096980077
:10396000C089704708B58430FEF74CFA003818BF9C
:10397000012008BD90F8EC303BB1054B026DDB68CF
:103980009A4202D17030FEF73DBA0020704700BF66
:103990001862002013B540F27F22044600F1D401E2
:1039A0006846F8F71DFD4FF4207204F1BC0101A830
:1039B000F8F716FD002384F8EC3084F8ED30236925
:1039C0005A7912B9186804F0CBFD002104F1700097
:1039D000FEF7D2F9002104F18400FEF7CDF901A829
:1039E000F8F71AFD6846F8F717FD02B010BD0000A1
:1039F00008B580F84C11806A082104F087FF012087
:103A000008BD000090F8ED20034602F0FF001AB157
:103A100003F18400FEF710BA704700002DE9F84367
:103A2000174604460D46FEF715F8DFF85C9006468B
:103A300000EB0708236820465B699847A84218D224
:103A40004FF4806004F036FFD9F80C30A4F85850D9
:103A50006365FDF7FFFF821BBA420AD2A8EB0003A1
:103A60004FF47A71A3FB01134FF4806004F06EFFF2
:103A7000E0E7236820465B69984785428CBF0020B9
:103A80000120BDE8F88300BF1862002010B5302384
:103A9000044683F311880B0707D5FCF779FA40F247
:103AA00032324FF00061FCF75FFAD4F8B8305A6850
:103AB000136823F00F031360D4F8B830197C1A6828
:103AC0000E238B405360FDF7C1FF0221C4F80C01A7
:103AD000A06A04F005FF002383F3118810BD0000E5
:103AE00070B503695A790446002A78D11D68036AC3
:103AF000002B08BF0021036880F80911DB6A984792
:103B000000286CD094F80931032B68D8DFE803F063
:103B100002322F68206A88B1012600F00F01324678
:103B200006FA01F120F00F0003F082FD236A23F072
:103B30000F0203F00F039E40B6B25683012384F8B0
:103B40000A31302383F311886B6D9A6812F4407F39
:103B500042D01A6822F001021A606A6D936823F459
:103B6000407393606A6D136843F0010333E00023F0
:103B7000C4E94333206A012600F00F01324606FAF9
:103B800001F120F00F0003F053FD236A23F00F0230
:103B900003F00F0306FA03F39BB2538384F80A6120
:103BA000302383F311886B6D9A6802F44072B2F58A
:103BB000007F11D01A6822F001021A606A6D9368C2
:103BC00043F4007393606A6D936823F48073936089
:103BD0006A6D136833431360002383F3118870BD4B
:103BE000236993F82920FF2A1BD0206AD20100F014
:103BF0000F030121994042F0020220F00F0003F070
:103C000017FD302383F311886B6D9A685204E3D457
:103C10001A6822F001021A606A6D936843F48043C7
:103C20009FE723682046DB6BBDE870400021184702
:103C300010B50446C06940B100F00F030121002215
:103C4000994020F00F0003F0F3FCA06950B100F0A0
:103C50000F030121BDE810400022994020F00F0021
:103C600003F0E6BC10BD000038B503695A7904467C
:103C70000D46002A38D10173186804F071FC012D3B
:103C800033D0022D35D02DB9E36B23F0805323F4CC
:103C9000B053E363236904F13801186804F052FC5F
:103CA00094F8643133B12369186804F5A8710430BD
:103CB00004F0E6FD002D14BF0123002384F86431D5
:103CC00009D0236918684FF40062202304F5A87115
:103CD000043004F0C1FD237D33B123691B685A6DA4
:103CE000136823F02003136038BDE36B43F4B05333
:103CF000CFE7E36B23F4007343F4A053C9E700005C
:103D0000037DA3B1D0F8B4305A68136823F00F03D1
:103D10001360D0F8B430197C1A680E238B405360BE
:103D2000D0F8B4305A68136823F001031360704769
:103D300038B503695A7904460D46D2B9186804F0BB
:103D40000FFC012DD4F8283114D0022D17D0D4F84F
:103D500028312364236904F13801186804F0F2FB68
:103D6000237D33B123691B685A6D136823F0200348
:103D7000136038BD23F40053C4F82831E7E743F457
:103D80000053F9E703695B791BB9806A042104F0E9
:103D9000BDBD7047F7B590F8ED3004460E461746A6
:103DA00003F0FF05BBB100F19C014FF4427201A882
:103DB000F8F716FB3A46314604F18400FEF7B2F8F4
:103DC00094F84C3105461BB1A06A042104F09EFD15
:103DD00001A8F8F721FB284603B0F0BD70B590F8B4
:103DE000093105460C46D3B9406AB8B1012600F046
:103DF0000F0106FA01F120F00F00324603F018FC23
:103E00006D6A05F00F0184EA060001F11003984085
:103E10008C4025F00F050443AC61304670BD002096
:103E2000FCE7000070B590F8093105460C46D3B99F
:103E3000006AB8B1012600F00F0106FA01F120F086
:103E40000F00324603F0F4FB2D6A05F00F0184EAFF
:103E5000060001F1100398408C4025F00F05044343
:103E6000AC61304670BD0020FCE70000164B10B579
:103E70000360164B80F832102C2201FB02330361E1
:103E80004FF461430446436300217030FDF758FF4F
:103E9000002104F18400FDF753FF04F19C00FDF7BD
:103EA0003DF804F1BC00FDF739F804F1D400FDF74A
:103EB00035F8002394F8322084F80931044B43F894
:103EC0002240204610BD00BF9C480208104802084E
:103ED000885B002013B5094C23686BB9009308492F
:103EE000084B3C224FF49E6005F0FEFB20602368E7
:103EF00013B90548FDF784FD02B010BDB45B002086
:103F000090470208B14B01089847020830B5836A10
:103F100085B004462BBB144B22691B685579D86ABF
:103F200013790093114A124B04F12C01002D08BFA4
:103F3000134606220391F8F791FB94F84C3103994C
:103F40000094002B18BFB5220A4B08BF3C224FF447
:103F50004C7005F0C9FBA062A36A13B90648FDF7CF
:103F60004FFD05B030BD00BF38250020BF47020817
:103F7000B8470208C54A0108C747020838B5D0F853
:103F8000B8500446EDB9302383F3118800690D4A17
:103F9000407B23460C2103F0B5F9C4F8B80085F343
:103FA0001188D4F8B8305A6823691B685B6D2833D0
:103FB00093602369D4F8B8001969BDE8384003F06C
:103FC00025BB38BD8D3A0108FFF7D8BF10B590F872
:103FD0005C3083F0010380F85C3090F85C3018337B
:103FE0000446402150F8230005F0E4FC94F85C30CE
:103FF000D4F8B4201833526854F82330D360D4F87E
:10400000B4305B6840225A60D4F8B4305B688A22CE
:104010001A60D4F8B4305A68136843F0010313608F
:1040200010BD00002DE9F04104468AB090461F46BD
:104030000E4689B957EA02030ED190F8ED305BB114
:1040400090F8EC3043B1034BDB6803650AB0BDE880
:10405000F08100BF18620020FFF73CFF23691A6857
:10406000002AF3D05B794FF4C870B6FBF0F0B0F5DE
:10407000007F38BF4FF40070002B0CBF4FF400736B
:104080004FF4806385B29F4238BF1F464FF494724D
:10409000454504F1D40104A838BF4546F8F7A0F916
:1040A000636F9D4207D0002384F8EC30294604F169
:1040B0007000FDF785FE636F1B09C4F89830C6B128
:1040C000636BB34200F04B819B4B1B689B6966633B
:1040D000A34200F0448104F170052846FDF792FEEA
:1040E000D4F820311844C4F820012846FDF778FEA2
:1040F000012694F83031E3B9E389D90519D4226E49
:1041000052B923699B793BB18B4B1B68D86A036812
:1041100040219B6C98472066626E52B923699B7957
:104120003BB1854B1B68D86A036840219B6C98475C
:104130006066A36E73B923691B7B5BB1E28912F4DD
:10414000007207D17C4B1B68D86A036840219B6CC6
:104150009847A06694F83031002B00F002810023CC
:10416000A382B4F86C20636BB2F57A7F04D9B3F5FF
:10417000E12F0DD800226275B3F5E13F08D823691D
:104180001A7B2AB1587B01F081F808B100236375CE
:10419000E289D4F8243112054CBF23F0005343F0D8
:1041A0000053C4F8243140F2671204F1BC0105A8A1
:1041B000F8F716F9D4F888309F4207D0002384F826
:1041C000ED30394604F18400FDF7FAFD1EB104F12B
:1041D0008400FDF705FE23695B79002B40F08E809B
:1041E000636B002B00F08A8094F8EE6094F8EE3058
:1041F000F6B203F0FF0503BB237DDBB1302383F36D
:10420000118820694D4AC07923460C2103F07AF8C1
:10421000C4F8B40085F31188D4F8B4305A6823691F
:104220001B685B6D243393602369D4F8B4009968EC
:1042300003F0ECF9012384F8EE30637D0BB3D4F87E
:10424000F030F3B93E4B0694CDE9073414203D4BD2
:104250000993F7F757FF054678B10AAA12E9030058
:1042600023695F7B01AB83E80300079B0093FF2278
:10427000069B3946284600F0E9FFC4F8F05005B91E
:104280006575636BA363217DD4F82831D4F82421AC
:104290002364D4F82C31E263636429B142F0100244
:1042A00043F04003E2636364637D1BB1636C43F0DE
:1042B00080036364244BC4E91234236904F1380198
:1042C000186804F03FF9237DC3B123691B685A6D58
:1042D000136823F02003136086B9D4F8B4305A6809
:1042E000136823F00F031360D4F8B430197C1A68F4
:1042F0000E238B4053602046FFF768FED4F88830C9
:1043000013B1012384F8ED30636F13B1012384F8F6
:10431000EC300E4BDB6823652046FFF7F7FD236882
:1043200094F80911DB6B2046984794F832307BB93A
:1043300094F8ED300CE000BF3825002061480108FA
:10434000C93F01089D430108013D01081862002092
:1043500005A8F8F761F804A8F8F75EF876E60026F5
:10436000C7E6226E1AB1636E003B18BF01232375A6
:10437000A36E003B18BF01236375F2E610B530232E
:10438000044683F31188D0F8B80003F037F800230F
:10439000C4F8B83083F3118810BD0000FFF7EEBFFA
:1043A0002DE9F74FD0F8F03004460E464BB346B334
:1043B00094F809112046F8F7D7F850B1636A43B171
:1043C00023F00F0203F00F03126922FA03F3DB0755
:1043D00017D404F19C0840F25532414601A8F7F782
:1043E000FFFF04F18407402E3246A16E28BF402211
:1043F0003846FDF7FDFD85B281462DB901A8F8F7D5
:104400000BF803B0BDE8F08F3846FDF7FBFC8642A1
:1044100028BF064601A8F7F7FFFFD4F8F00001F027
:1044200087F8022004F046FAD4F8F000C37C002B91
:1044300000F0A680636BB3F5E12F0FD8B4F86C10D1
:10444000033189B2B1F57A7FA4F86C1006D9002146
:10445000617503B0BDE8F04F00F04ABFFA214E4A43
:104460004B43B3FBF2F31FFA89F201339A4200D9AE
:104470009DB24FF0300B8BF31188D4F8B8305968E7
:104480000B6823F00F030B60D4F8B830197C186860
:104490004FF00E0A0AFA01F14160A06E294605F0BC
:1044A0008BFAD4F8B810A06E49683C4BC860D4F8B9
:1044B000B81049684D60D4F8B81049689A2008606F
:1044C000D4F8B8104868016841F001010160A91CE6
:1044D000606B5943324BB1FBF0F1324801F5FA7190
:1044E000994288BF0146002080F31188022004F021
:1044F0002DFA814610BB8BF31188D4F8B820506890
:10450000026822F00F020260D4F8B8201068127C12
:104510000AFA02F34360D4F8B8305B685B689D42E6
:1045200037D9ED1AADB21DB1FDF790FAC4F80C0100
:10453000022004F0B5F9002383F31188D4F8F000C9
:10454000C9F3400100F0D4FE002D3FF45AAF40F211
:10455000B132414601A8F7F743FF29463846FDF737
:1045600085FCD4F814312B44C4F81431D4F8183134
:104570002B44C4F8183101A8761BF7F74DFF16E756
:10458000B4F86C30002B3FF474AF013BA4F86C30EE
:104590006FE74D46CCE700BF40420F008096980081
:1045A0009F860100A086010013B5D0F8483104466B
:1045B000BBB900F59A7004F087F91823C4F84831A4
:1045C00023691868019003F0CBFF636C019823F016
:1045D000080304F13801636402B0BDE8104003F041
:1045E000B1BF02B010BD00002DE9F047044686B00F
:1045F0000D4640F2CA3200F19C0101A8F7F7F0FE27
:1046000094F8303123B1012D02D92046FFF7CCFFB9
:1046100004F184092A4602A94846FDF7BFFC4FF081
:104620000008824602AD4746C2451FDD2269537924
:10463000D3B910680268D669D5E90012B047061EE2
:1046400014DB05D0FDF702FA3744C4F80C01BFB201
:10465000083531464846FDF709FC55F8043C9E42B2
:1046600004D108F10108DFE70026F1E7D4F814319E
:104670003B44C4F81431D4F818313B44C4F8183121
:1046800001A8F7F7C9FE06B0BDE8F08770B504468B
:104690008430FDF7B7FB0146B8B1637D2046ABB16E
:1046A000FFF77EFE94F80931022B0ED1D4F8105199
:1046B0001DB9FDF7CBF9C4E94405637D4BB1D4F8CE
:1046C0000C31D3B1012384F8093170BDFFF78CFFA1
:1046D000E8E723691B689A6BE38913F4006FD4F849
:1046E0001431C2F580700CBF0C210821984204D20D
:1046F000A3F5807313448B42E4D8FDF7A7F9D4F8EF
:104700001031C01A0B4B9842DFD90B4B22691B6842
:104710000A4998690A4BD21A0A4B92105A43036805
:10472000D2B21B68984723682046DB6BBDE8704017
:104730000021184720A1070038250020E84702087B
:1047400010480208A38B2EBA10B5036A0446E3B1E1
:1047500090F80911F7F708FFB8B104F17000FDF700
:104760006BFB94F80A21D4F8983080B272B1984269
:104770000BD2226A002384F80A3122F00F010123B0
:1047800002F00F0293409BB20B8310BD103398428E
:10479000FBD9226A012322F00F0102F00F0284F8F4
:1047A0000A3193409BB24B83EFE7000070B5124B88
:1047B000026DDB689A42044619D190F8EC3003F0A0
:1047C000FF0593B100F170063046FDF71BFBD4F8EE
:1047D00020311844C4F820013046FDF701FB94F85D
:1047E0000A3133B92046FFF7AFFF284670BD0025D8
:1047F000FBE71D46F9E700BF1862002038B50D4BF6
:104800000546DB68006D984210D195F8EC306BB12D
:1048100005F17000FDF708FC044628B195F80A314F
:1048200013B92846FFF790FF204601E04FF0FF3014
:1048300038BD00BF1862002038B590F80851044612
:10484000FDF70AF985F0010504EBC505C5E93E0150
:1048500094F8083183F0010384F8083138BD000072
:1048600070B5037D0446002B4AD0D0F8B4305B68A5
:104870005D6890F85C601A6822F00F021A60D0F848
:10488000B430197C1A680E23C5F140058B40ADB2D7
:104890005360F6B2FFF79AFBADB118362A4654F8CA
:1048A000261004F17000FDF73DFBD4F81C31D4F85C
:1048B00020212B4415442D1AC4F81C31C4F8205172
:1048C0002046FFF7B9FF636D93B104F17000FDF767
:1048D00099FAB4F8583098420AD3302383F31188F8
:1048E0004FF48061606D03F0FBFF002383F31188B8
:1048F00094F80A3123B12046BDE87040FFF724BF89
:1049000070BD00002DE9FF4700F1700804464046E5
:10491000FDF792FA694602464046FDF7C1FA6E4637
:104920008146002704F5A87AB9450ADD2269537942
:1049300053B910680268156AD6E90012A847051E27
:1049400003DA04B0BDE8F087002594F864313BB188
:10495000504603F0B9FF10F0200F18BF4FF0FF359D
:10496000D4F848315BB929464046FDF7C1FAD4F87E
:104970001C312B44C4F81C312046FFF75DFF7368DF
:10498000AB4206F10806DCD80137CDE730B590F828
:10499000ED3085B00446002B51D0D0F8483100F1FD
:1049A000BC050BB340F2D742294603A8F7F718FD20
:1049B00004F59A7003F088FFD4F8483123EA000028
:1049C000C4F8480168B923691868019003F0C8FD6C
:1049D000636C019843F00803636404F1380103F049
:1049E000B1FD03A8F7F718FD94F83031DBB140F2C0
:1049F000F54204F1D40103A8F7F7F2FC2046FFF7D3
:104A000081FF636D63B104F17000FDF7FBF9B4F849
:104A10005830984204D3606D4FF4806103F076FF04
:104A200003A8F7F7F9FC40F2FD42294603A8F7F77F
:104A3000D7FC2046FFF72AFE03A8F7F7EDFC05B0E8
:104A400030BD0000F8B51E4D0446A36A3BB92B6883
:104A5000986A03684FF47A719B689847F5E70026D7
:104A60004FF47A7141F20C0003F070FF0546FCF739
:104A7000EDFF831BB3F57A7F2ABF06460027012787
:104A800029070AD594F84C31C3B1236D986B0130D6
:104A9000B52828BFB52004F07FFA94F8ED30002B3C
:104AA000DED06A0706D42FB9D4F84831002BD7D00E
:104AB000EB04D5D52046FFF769FFD1E73C20EAE7B4
:104AC0003825002008B5FFF7BDFF000037B590F886
:104AD000EC30044603B390F83031EBB900F1D40167
:104AE0004FF48B6201A8F7F77BFC237DB3B9204616
:104AF000FFF708FF636D63B104F17000FDF782F901
:104B0000B4F85830984204D3606D4FF4806103F0DC
:104B1000FDFE01A8F7F780FC03B030BDD4F8B43037
:104B2000002BE7D0302383F31188D4F8B4305B68CE
:104B30001A68D20734D45D68C5F1400515F0FF0549
:104B40001DD094F85C3018332A4654F8231004F131
:104B50007000FDF7E7F9D4F81C31D4F820212B447C
:104B600015442D1AC4F81C31C4F820512046FFF713
:104B700063FE94F80A3113B12046FFF7E5FDD4F83F
:104B8000B4305A68136823F00F031360D4F8B430BC
:104B9000197C1A680E238B4053602046FFF716FAE3
:104BA000002383F31188237D002BA3D19FE700000E
:104BB000104B70B5104C1D68A86A226803689B688A
:104BC0001AB94FF47A719847F6E7A86A0B4E036852
:104BD0004FF47A719B6898470B2456F8040B20B168
:104BE00090F8EC300BB1FFF771FF013C14F0FF04BB
:104BF000F3D1EAE738250020B45B0020885B002071
:104C000038B50446C8060D4604D5E06910B1022146
:104C100004F0C0FE690604D5A06910B1022104F0B9
:104C2000B9FEAA0604D5E06910B1012104F0B2FE74
:104C30002B0606D5A06920B1BDE83840012104F05B
:104C4000A9BE38BD2DE9F74F03690D4659790446D1
:104C500029B1B5FA85F0400903B0BDE8F08FC581F0
:104C6000D3F800809869D8F854205668976812687D
:104C700002F001091A7900F085FE2369E0611A79D2
:104C80005869012100F07EFE2369A0611A79D86974
:104C9000042100F077FE236920621A79186A042142
:104CA00000F070FE23686062DB6B94F80911204607
:104CB0009847D4E906A015F0080B1EBF524682465D
:104CC000104615F00403019303D0AB0718BF45F05D
:104CD0000305E907D4F8282161D542F4803246F46F
:104CE0008036C4F8282110B1022104F053FEAB072E
:104CF000D4F828215DD542F4003246F40036C4F8D9
:104D00002821BAF1000F03D00221504604F042FEE0
:104D1000D4F82831BBF1000F56D046F4004643F4D6
:104D20000043019AC4F82831D4F82C31002A50D01D
:104D300043F00803C4F82C3194F8303147F00807E9
:104D400063B9236918684FF48052182304F59A71E7
:104D5000043003F081FD012384F83031237D73B1E9
:104D6000D4F8B4305BB15A68136823F00F031360B2
:104D7000D4F8B430197C1A680E238B40536000239A
:104D8000A38229462046FFF73BFFD8F854305A68E3
:104D9000B24225D19A68BA4222D101205CE722F4BE
:104DA000803226F48036C4F8282100289FD00121C3
:104DB0009BE722F4003226F40036C4F82821BAF129
:104DC000000FA5D00121A0E726F4004623F40043FC
:104DD000A7E723F0080327F00807C4F82C31D0E731
:104DE000B9F1000F03D01A6822F001021A60D8F856
:104DF00054305E60D8F854309F60B9F1000FCCD0C9
:104E0000D8F85420136843F001031360C5E700008D
:104E1000004870473449020800207047014B0020C9
:104E200019707047B85B0020704700000020704781
:104E30007047000004F03EBC084609B104F036BCDF
:104E40007047000008B5134612780C2AA8BF0C2240
:104E500008461A70024905F05FF8012008BD00BF3E
:104E60009075FF1F1046194604F0DEBC04F0EEBC3E
:104E70002DE9F34742F6F8216846F7F797FA5348C9
:104E800001A9FBF797F8524B05461C6868B9A06961
:104E90004E4A03684F491B68984703246846F7F752
:104EA00091FA204602B0BDE8F087019B606B1F338A
:104EB00023F01F030193036800211B689847019AA0
:104EC00001460746284605F017F8A3691A681268D4
:104ED00038B91846404990472846FBF775F8012431
:104EE000DCE73E49184690470026B146019B4B45FA
:104EF00023D9606B03685FFA86F85B684146984780
:104F0000824620B92846FBF75FF80224C6E7A06A6C
:104F100003684FF47A711B699847606B03684146D8
:104F2000DB689847013630B9A0692D4903681B68D2
:104F300042469847E6E7D144D8E7A069234A036888
:104F400028491E68DFF8A8903B46B047606B0368AD
:104F500001215B6998474FF00108A06A03684FF48C
:104F60007A711B699847606B03682A461E69019B2A
:104F70003946B0470646A0690368D6B94246D3F819
:104F800000A049460A23D047A06A036864215B68F1
:104F900008F101089847B8F10B0FDED1606B036888
:104FA00031465B699847A0690F4903680A221B686C
:104FB000BFE71B680D499847606B036800215B6978
:104FC00098472846FBF700F8002467E79CE60108AD
:104FD000382500204C4902085F490208764902083A
:104FE0007F49020890490208CC490208C2490208D8
:104FF000A34902082DE9F04F254B9DB093F890206E
:105000000F9293F89120109293F89220119293F8B6
:105010009320129293F8952093F89470139293F83A
:105020009620149293F89720159293F898B093F8DD
:1050300099A093F89A9093F89B8016AB0C4605467E
:1050400014491722184605F037FC139A0792149A50
:105050000692159A05920F9A0492109A0392119A49
:105060000292129A0C4B0897CDE900020026CDE976
:105070000989322221462846CDE90BAB8DF86F60B5
:10508000F7F7ECFA012084F831601DB0BDE8F08F2D
:105090000075FF1F29E10108EC49020804F062BD18
:1050A0002DE9F0471B4A1C4CDFF87480DFF874A030
:1050B000DFF8749086B010460F4604F085FC154A60
:1050C0001649A41A034600943846FCF705FD03F080
:1050D00013FD0446D4B1256AE269A36B05924545E8
:1050E000284614BF661BAAEB0806049304F06CFC68
:1050F000DDE90432CDE90106494638460095FCF762
:10510000EBFC204603F008FD0446E3E706B0BDE8EB
:10511000F08700BF0001002000070020244A020899
:105120000007002000230020574A0208084600F02C
:10513000F1B800002DE9F04188B00D4604A805A99A
:1051400004F0F0FA1549DFF8588006462846FCF7C7
:10515000C3FC00242746E0B286421CD9CDE906777D
:1051600010B1049B03EB441007AA06A903F04AFB05
:1051700005990C2262438818D0E901300290079803
:105180000190069800908A589B0A41462846FCF7F1
:10519000A3FC0134DFE708B0BDE8F0817C4A0208D7
:1051A000874A020808460AB904F072BA012A01D1F6
:1051B00004F074BA022AF7D0012004F073BA000098
:1051C00070B50C4615462AB9084604F06FFA2E460B
:1051D000304670BD104619B9BDE8704004F054BAAD
:1051E00004F052FA06460028F2D054F8042CAA42E1
:1051F00028BF2A46214604F08FFE204604F056FAC6
:10520000E6E7000070B50C4615460026AE4204D213
:10521000F7F728FFA0530236F8E7EB0704D5F7F7B6
:1052200021FF2C4404F8010C012070BDF7F7E0B910
:1052300038B5054D00242846013403F0B9FB102C85
:1052400005F12005F7D138BDC05B002082B010B554
:10525000914203934FF00003C0E90033C0E90233E9
:1052600004460174427484BF02744174DDE9030191
:1052700084E80300DDE9050104F1080383E8030085
:105280002046BDE8104002B0704700000020704783
:105290000F2838B50AD8074B03EB40152846AC68F1
:1052A00003F0C8FB14B1AB689C4201D1002038BDAB
:1052B0000120FCE7C05B00200F2938B504461546E5
:1052C00010D8094800EB411003F0E0FB55B1074B43
:1052D0001B683BB1227C02EB420203EB82039A681B
:1052E00001329A6038BD00BFC05B0020BC5B00206B
:1052F00013B5002304460A4683740191417CFFF7ED
:10530000DBFF019A217C204602B0BDE81040FFF788
:10531000D3BF00002DE9F04F354E2DED028B3368E1
:105320008BB007461BB9CC20F6F7F2FE306031494E
:105330009FED318ADFF8C4803846FCF7CDFB0025AD
:105340004FF00C09326809FB05F4EBB2115902EB7E
:10535000040C31B9DCF8041019B9DCF80810002984
:105360003DD0111991ED007A52F804E0DCF8040008
:10537000DCF8081007910EEB0001013107EE901ADE
:10538000B8EE477AF8EE677A27EE087ADCF804A0E0
:1053900052F804B0C7EE277A0722B3FBF2F2C2EB51
:1053A000C20CA3EB0C0301330132DBB2D2B209937E
:1053B000089217EE900AF4F799F8079B0093CDE94D
